:020000040800F2
:1080000000800120FD6C01080D0301080F03010829
:108010001103010813030108150301080000000003
:10802000000000000000000000000000170301082D
:1080300019030108000000001B030108DD8100088E
:10804000416D0108416D0108416D0108416D010854
:10805000416D0108416D0108416D0108416D010844
:108060001D8E0008416D0108416D0108416D010838
:10807000416D0108416D0108416D0108416D010824
:10808000416D0108416D0108416D0108219400080E
:10809000A992000865930008416D0108E58E00086B
:1080A000416D0108416D0108416D0108416D0108F4
:1080B000416D0108416D0108416D0108416D0108E4
:1080C000416D0108416D0108416D0108416D0108D4
:1080D000416D0108416D010839910008416D0108A9
:1080E000416D0108416D0108416D0108416D0108B4
:1080F000416D0108416D0108416D0108416D0108A4
:10810000416D0108416D0108416D0108416D010893
:10811000416D0108416D0108416D0108B58E0008EF
:10812000416D0108416D0108416D0108416D010873
:10813000416D0108416D0108416D0108416D010863
:10814000416D0108416D0108416D01088DB70008BE
:10815000416D0108416D0108416D0108416D010843
:10816000416D0108416D0108416D0108416D010833
:10817000416D0108416D0108416D0108416D010823
:04818000416D010844
:1081880010B5054C237833B9044810B10448AFF34F
:1081980000800121217010BDC005002000000000F2
:1081A800C479010808B5064B1BB106480649AFF368
:1081B80000800648016811B1054B03B1984708BD16
:1081C80000000000C4790108C4050020BC05002097
:1081D80000000000684620F007018D4601B5124BEB
:1081E8001A787AB15A6801325A60104B1A6801320B
:1081F8001A600F4B1A6812B11A68013A1A60002205
:10820800094B00E001221A700A4B1A683AB11A6841
:10821800013A1A601B6813B9074B01221A70BDE8AE
:1082280001408546704700BFDC050020E05400206F
:10823800C04A0020C44A0020C84A0020074B41F623
:108248004B525A60064AF02182F8231000229A60A5
:108258006FF0040007221A600AF030BD10E000E059
:1082680000ED00E0014B5868704700BFDC050020B6
:108278002DE9F341654F012001460024022509F04C
:108288009BFA0F23384669460126009348F21008E6
:108298008DF804408DF806408DF807408DF805509C
:1082A80009F0D2F838466946CDF800808DF80640C6
:1082B8008DF807408DF804608DF8055009F0C4F872
:1082C800A7F818804FF480733846694600938DF8F4
:1082D80006408DF807408DF804508DF8055009F0D8
:1082E800B3F821464FF4800009F0BCF907F5806720
:1082F8002846314609F060FA40F6FC73384669466C
:1083080000934FF480588DF804408DF806408DF89E
:1083180007408DF8055009F097F838466946CDF8BA
:1083280000808DF806408DF807408DF804608DF8C0
:10833800055009F089F8A7F81880042007F5806728
:10834800314609F039FA4AF2C23338466946009391
:108358008DF804408DF806408DF807408DF80550DB
:1083680009F072F844F2080338466946DFF8A48039
:1083780000938DF806408DF807408DF804608DF85D
:10838800055009F061F84FF4804308203B833146DB
:10839800788309F011FA4FF68C73404669460093CA
:1083A80010278DF804408DF806408DF807408DF8A9
:1083B800055009F049F8404669468DF806408DF8A1
:1083C800074000978DF804608DF8055009F03CF8D7
:1083D80038463146A8F81A7009F0EEF98DF80640CB
:1083E8008DF807400A4C4FF6FF7320466946009304
:1083F8008DF804608DF8055009F026F84FF47F4396
:108408006383FF232383BDE8FC8100BF0000024093
:1084180000100240000C0240C90802F047BF0728BC
:1084280020D8DFE800F004070A0D1013161B4FF4DC
:10843800807210E04FF400720DE04FF480620AE0A1
:108448004FF4006207E04FF4805204E04FF400520A
:1084580001E04FF48042044B5A837047024B4FF4BB
:1084680000425A83704700BF00100240072820D8F6
:10847800DFE800F004070A0D1013161B4FF4807292
:1084880010E04FF400720DE04FF480620AE04FF400
:10849800006207E04FF4805204E04FF4005201E01C
:1084A8004FF48042034B1A837047024B4FF400424B
:1084B8001A8370470010024038B50546002445FA73
:1084C80004F3DB07E0B202D5FFF7D0FF01E0FFF7C6
:1084D800A6FF0134082CF2D138BD08B507282ED8DC
:1084E800DFE800F004060B10151E232800200FE01B
:1084F800144B1869C0F3802008BD124B1869C0F3EB
:10850800C02008BD0F4B1869C0F3003008BD042017
:1085180001F038FCB0F5006F34BF0020012008BD21
:10852800084B1869C0F3403008BD064B1869C0F302
:10853800803008BD034B1869C0F3C03008BD002067
:1085480008BD00BF000C024007282DD8DFE800F066
:1085580004090E13181D2227144B5869C0F3002074
:108568007047124B5869C0F3402070470F4B586949
:10857800C0F3802070470D4B5869C0F3C020704786
:108588000A4B5869C0F300307047084B5869C0F36C
:1085980040307047054B5869C0F380307047034B33
:1085A8005869C0F3C030704700207047001002407F
:1085B80010B50020FFF7C8FF041C18BF01240120D4
:1085C800FFF7C2FF10B144F00204E4B20220FFF743
:1085D800BBFF08B144F004040320FFF7B5FF08B15E
:1085E80044F008040420FFF7AFFF08B144F010047A
:1085F8000520FFF7A9FF08B144F020040620FFF783
:10860800A3FF08B144F040040720FFF79DFF08B11D
:1086180044F08004204610BD034B202208B15A8341
:1086280070471A83704700BF00100240082008B541
:1086380001F0A8FB592805D9074B1A7852B901222D
:108648001A7008BD082001F09DFB542802D8024B7F
:1086580000221A7008BD00BFE4050020044B1878FA
:108668000138C0B201288CBF00200120704700BF2C
:10867800E4050020044B1878012802D102221A7060
:1086880070470020704700BFE4050020012808D08B
:1086980002D302280FD109E0084B1869C0F3402023
:1086A8007047064B1869C0F380207047034B186960
:1086B800C0F3C02070470020704700BF000402408C
:1086C800022808B513D80B4BC200195C0A4B9A183C
:1086D80053F8300021B95368000C40EA034008BD44
:1086E8005168002342F210720CF0D0FF08BD002040
:1086F80008BD00BFBA4A0020404C0020022830B50F
:1087080022D872B6114CCB170A4604EBC001C1E956
:10871800002354F830404D6822042B0443EA1443E4
:10872800C1E900230A4A002342F82030094A0128F7
:1087380042F8203003D0022803D0074A02E0074A53
:1087480000E0074A536262B630BD00BF404C0020CB
:10875800F44B0020084D00200004014000080040B0
:10876800000C00400020704702289CBF014B43F8D2
:1087780020107047344C002001282CD002D3022846
:108788007AD151E03D4B11F0040F9A680BD0C8061E
:1087980002D542F0040208E022F004029A60DA6886
:1087A80042F0040205E022F004029A60DA6822F03E
:1087B8000402DA60324BC1F3C0021A70314BC1F3C4
:1087C800401211F001011A702F4B02D001221A70C9
:1087D800704719707047294B11F0040F9A680BD035
:1087E800C80602D542F4807208E022F480729A60CA
:1087F800DA6842F4807205E022F480729A60DA68DE
:1088080022F48072DA601E4BC1F3C0025A701D4B0D
:10881800C1F3401211F001015A701B4B02D0012222
:108828005A70704759707047144B11F0040F9A68CA
:108838000BD0C80602D542F0200208E022F0200240
:108848009A60DA6842F0200205E022F020029A607D
:10885800DA6822F02002DA60094BC1F3C0029A708C
:10886800084BC1F3401211F001019A70064B02D077
:1088780001229A7070479970704700BF003C014010
:10888800B74A0020BA4A0020B44A00202DE9F04F28
:10889800CD4E8FB000240225C023304609A9099384
:1088A8008DF828508DF82A408DF829508DF82B40E6
:1088B80008F0CAFD30460621032208F048FEC34FDF
:1088C80003223046072108F042FE0121284608F01D
:1088D800A3FF384609F06EFA03A809F053FB4FF6D8
:1088E800FF7B384603A9ADF80C40CDF810B0ADF8C1
:1088F8001440ADF80E4009F007FB22462346032139
:10890800384609F07BFF06A809F0B6FD4FF00808C5
:10891800384606A94FF00409ADF8208009F020FE7A
:10892800384606A9ADF8189009F01AFE41F65F6CB2
:1089380061463846CDF800C009F0BDFE7C62384675
:10894800012107F5803709F074FBC023384609A9CF
:1089580009938DF828508DF82A408DF829508DF804
:108968002B4008F071FD384606212A4608F0EFFD35
:108978002A463846072108F0EAFDA7F5FE37012107
:10898800484608F03DFF384609F014FA03A809F0F4
:10899800F9FA384603A9ADF80C40CDF810B0ADF897
:1089A8001440ADF80E4009F0AFFA224623460321E1
:1089B800384609F023FF06A809F05EFD384606A9E7
:1089C800ADF8208009F0CCFD384606A9ADF818901E
:1089D80009F0C6FDDDF800C03846614609F06BFEB7
:1089E8007C623846012107F5FC3709F022FB032396
:1089F800384609A9099301938DF828508DF82A4023
:108A08008DF829508DF82B4008F01EFD3846214678
:108A18002A4608F09CFD2A463846012108F097FDB1
:108A2800A7F5FA370121404608F0EAFE384609F072
:108A3800C1F903A809F0A6FA384603A9ADF80C4015
:108A4800CDF810B0ADF81440ADF80E4009F05CFA5E
:108A5800019B224619463846234609F0CFFE06A850
:108A680009F00AFD384606A9ADF8208009F078FD1E
:108A7800384606A9ADF8189009F072FDDDF800C077
:108A88003846614609F017FE7C623846012109F034
:108A9800D0FA2946012009F029F9CDF82C90DFF801
:108AA800389101270BA88DF831808DF830408DF86A
:108AB800327008F0EFFBD9F808300DA823F0040352
:108AC800C9F80830D9F80C30C24623F00403C9F8B5
:108AD8000C3006238DF835308DF834808DF836400B
:108AE8008DF837700AF0A0F84146384609F0FEF8CC
:108AF8004FF480730BA80B938DF831808DF83040BC
:108B08008DF8327008F0C6FBD9F80830052123F437
:108B18008073C9F80830D9F80C30384623F48073CC
:108B2800C9F80C3009F0E2F84FF020080BA8CDF88E
:108B38002C808DF830408DF831A08DF8327008F017
:108B4800A9FBD9F808300DA823F02003C9F808308C
:108B5800D9F80C301E4E23F02003C9F80C30DFF88A
:108B68007C9017238DF8343007238DF835308DF835
:108B780036408DF837700AF057F8D9F810102046AB
:108B880021F07F433360090EFFF7F6FDD9F8301066
:108B9800384621F07F437360090EFFF7EDFDD9F8E1
:108BA8005010284621F07F43B360090E094EFFF7A5
:108BB800E3FD3946404608F023FE304609F0FAF84E
:108BC80041F270730CE000BF00080240000401404D
:108BD800344C002000140040003C0140A84C002008
:108BE800304603A90493ADF80C40ADF81440ADF835
:108BF8000E4009F089F9304639463A4609F04AFDEF
:108C08003046394609F015FA37230DA88DF8343067
:108C18008DF835508DF836708DF837700AF004F8F5
:108C28000FB0BDE8F08F012870B5424B0CD002D3CD
:108C380002281AD111E0404A1178404A526A09B113
:108C4800C2F580321A6010E03B4A51783C4A526AB9
:108C580009B1C2F580325A6007E0374A9178394A3B
:108C6800526A09B1C2F580329A60324A364B52F8DC
:108C7800204053F820108C4252F8204053F820101E
:108C880020DD611AB1F5004F30494FEAC0060E44A5
:108C980051F830100C4671680D4608DA52F8201069
:108CA80053F820302A4ACB1A52F8202034E053F8DF
:108CB800201052F82030264ACB1A52F8202003F50B
:108CC80080331AE08C422DDA53F8204052F82010F5
:108CD8004FEAC006611AB1F5004F1C490E4451F81D
:108CE80030100C4671680D460CDA53F8201052F813
:108CF8002030174ACB1A52F820205343E41A65EB68
:108D0800E3750DE052F8201053F82030104ACB1AC2
:108D180052F8202003F580335343E41845EBE375FC
:108D2800C6E90045034B53F82020074B43F82020A1
:108D380070BD00BFF44B0020B44A0020000401407D
:108D480000080040000C0040084D0020404C002066
:108D5800344C0020174B1A691B6912F0080F14BF16
:108D680000200120DA06144B58BF40F002001B69AE
:108D780058BFC0B21B04114B58BF40F004001A6919
:108D880051071A691B6958BF40F00800120758BFFD
:108D980040F010001906094B58BF40F020001A692E
:108DA8001B69D20558BF40F040009B0558BF40F0F2
:108DB800800070470004024000080240000C024096
:108DC800034B08B1034A00E0034ADA60704700BF6A
:108DD80000ED00E00400FA050100FA050C49002343
:108DE8004FF0FF3203F1200041F8202003F160002A
:108DF8000133082B41F82020F4D100231946044AF6
:108E08009A180133F02B82F80013F8D1704700BF8D
:108E180000E100E0684620F007018D4601B5042016
:108E280008F0A0FA0D4B002119600D4B0D48196090
:108E380000220023C0E900230B4B59620B4B1B781F
:108E480043B90B4B9A6822F004029A60DA6822F060
:108E58000402DA60BDE8014085467047F44B002003
:108E6800084D0020404C002000040140B74A002073
:108E7800003C0140012808D002D302280FD108E0A5
:108E8800084B186900F0080007E0074B00201B6931
:108E98007047044B186900F00400C0B27047002006
:108EA800704700BF0000024000080240684620F0FA
:108EB80007018D4601B50121074809F00BFC002088
:108EC800FFF7B1FE0120FFF7AEFE0220FFF7ABFE71
:108ED800BDE801408546704700140040684620F010
:108EE80007018D4601B54FF4807008F02DFAD8B10E
:108EF8004FF4807008F036FA1D4B002159601D4B65
:108F08001D48596000220023C0E902231B4B596207
:108F18001B4B5B7843B91B4B9A6822F480729A60AA
:108F2800DA6822F48072DA60202008F00DFAD0B1F5
:108F3800202008F017FA0E4B002199600D4B0E48BF
:108F4800996000220023C0E904230F4B59620C4B9F
:108F58009B7843B90B4B9A6822F020029A60DA6832
:108F680022F02002DA60BDE801408546704700BF64
:108F7800F44B0020084D0020404C00200008004021
:108F8800B74A0020003C0140000C0040034B4FF45E
:108F9800804208B11A8370475A837047000802401C
:108FA800C0B202F0A9BAC0B202F098BA70477047CE
:108FB800704700BF70B5044688B0584809F04CFCAB
:108FC8004FF40030012108F01BFC0820012108F0B3
:108FD800F3FB022600252023514805A905938DF8A7
:108FE80018608DF81A508DF819608DF81B5008F02C
:108FF8002BFA40234A4805A905938DF818608DF887
:109008001A508DF819608DF81B5008F01DFA444865
:109018000521072208F09BFA41480621072208F09B
:1090280096FA01A809F0C8FC0B2C25D8DFE804F053
:109038002406090C0F1215181B1E20224FF4615329
:109048001CE04FF4964319E04FF4E14316E04FF467
:10905800164313E04FF4614310E04FF496330DE0EC
:109068004FF4E1330AE04FF4613307E02D4B05E09C
:109078002D4B03E02D4B01E04FF4165301A927486F
:10908800019309F03DFC2623002401258DF81C30AE
:1090980007A806238DF81D308DF81E408DF81F5047
:1090A80009F0C2FD1D4840F2FF3109F086FD282174
:1090B80022461A4809F062FD2A46184840F22771EC
:1090C80009F05CFD2A46154840F2266109F056FD74
:1090D8002A46124840F2255109F050FD22460F4811
:1090E80040F2244109F04AFD22460C4840F6460168
:1090F80009F044FD2246094840F66A1109F03EFD90
:1091080060212246054809F039FD054B10225A8393
:109118000248294609F071FC08B070BD00440040BF
:10912800000C024090D0030020A1070040420F002D
:10913800684620F007018D4619B529490B889B061A
:109148001BD5284B5B69D80601D58B8815E0264BC3
:109158001A6858680132202A08BF0022824205D0C6
:109168001C6888881919C0B208721A601F4B0A2235
:109178001A601D4B9A6A1E4B1A60194803881A0612
:109188001AD51B4B1A68BAB9174BDC6A196B8C4293
:109198000ED0144910240C83196B5C1894F83440D1
:1091A800013184801963196B202905D11A6303E002
:1091B80040F2277109F0E2FC094803885B060BD5E9
:1091C80040F2266109F01DFD074B1A6BDB6A9A42D3
:1091D80002D1044B10225A83BDE8194085467047D6
:1091E80000440040000C0240E8050020C44A00206A
:1091F800C04A00200A4BDA6A196B0132202A08BFDC
:1092080000228A420AD0D96A591881F834000548E0
:10921800DA6240F22771012209F0B0BC704700BF42
:10922800E8050020004400400A4B59681A6891423A
:109238000CD05A6899180132097A5A605A68017034
:10924800202A05D100225A6001207047002070476B
:1092580001207047E8050020014B9862704700BF65
:10926800E8050020034B187810B100221A7001207D
:10927800704700BFC84A002072B6034B00225A60EC
:109288001A6062B6704700BFE805002010B50446B2
:1092980001E0FFF7AFFF14F8010B0028F9D110BD6A
:1092A800684620F007018D4671B5284D284B2C687B
:1092B8001B680134082C08BF002400219C4287B099
:1092C80024483CD001AA07F07FFC9DF80C302A689E
:1092D800042B214B03EB021206D1012151702A689D
:1092E80003EB0213029A05E0002151702A6803EB90
:1092F8000213019A5A609DF80D30174A022B134B3E
:10930800196802EB011201D1012100E000219170DE
:109318001B689DF80E10104A1B010C48D1540DF122
:109328000E010023056811F8016F02EB0515ED1811
:109338000133082B2E72F5D1044B1C6001E007F0B5
:1093480089FC07B0BDE8714085467047584B00203E
:10935800CC4A002000640040D84A0020684620F02B
:1093680007018D4671B5284D284B2C681B680134C0
:10937800082C08BF002401219C4287B024483CD017
:1093880001AA07F021FC9DF80C302A68042B214B18
:1093980003EB021206D1012151702A6803EB021374
:1093A800029A05E0002151702A6803EB0213019A22
:1093B8005A609DF80D30174A022B134B196802EBBF
:1093C800011201D1012100E0002191701B689DF874
:1093D8000E10104A1B010C48D1540DF10E01002348
:1093E800056811F8016F02EB0515ED180133082B1C
:1093F8002E72F5D1044B1C6001E007F02BFC07B07E
:10940800BDE8714085467047584B0020CC4A002083
:1094180000640040D84A0020684620F007018D46C5
:1094280031B52B4B2B4A1968126886B0914205D189
:1094380029480121002207F093FC44E01968274AD3
:1094480002EB0111497851B104211B688DF80C1009
:109458000021019102EB03125368029307E01B6895
:109468008DF80C1002EB031253680291019318490E
:109478001A4B0A680DF10E0003EB021292781C4693
:10948800002A14BF022200228DF80D200A6812015A
:109498009A5C8DF80E2000220D680D4B04EB051523
:1094A800AD182D7A0132082A00F8015FF4D11A6844
:1094B80001321A601A68082A01D100221A60064887
:1094C80001A907F0EAFA06B0BDE8314085467047C1
:1094D800D44A0020D04A0020006400405C4B0020A1
:1094E8002DE9F04101388AB00E461546072829D8DB
:1094F800DFE800F020181612100E0C040223ADF855
:1095080010300B238DF81430012322E003231AE0D6
:10951800062318E00C2316E00F23ADF8103015E0F1
:109528001E2310E03C23ADF810300F238DF81430C3
:1095380007230EE07823ADF810300C238DF8143093
:10954800032306E00823ADF810300F238DF81430FC
:1095580002238DF815308A4800238DF8133007F060
:109568003FF901214FF0007008F04AF90820012165
:1095780008F022F90323002408200121079302237D
:109588008DF820308DF821308DF822408DF8234059
:1095980008F012F97B4807A907F056FF0922794815
:1095A800214607F0D4FF01210922764807F0CFFFB2
:1095B8000127734804A98DF812408DF816408DF8DC
:1095C80017708DF818408DF819408DF81A708DF8BD
:1095D8001B7007F01FF9B6F5006F8DF80A408DF87B
:1095E8000B408DF80C704FF6FF730DDA7201ADF871
:1095F8000020ADF80240ADF80430ADF80630ADF803
:1096080008408DF80D700BE0ADF80040ADF8024051
:10961800ADF80430ADF80630ADF808408DF80D40CF
:10962800684607F063F9012300228DF80A308DF8A7
:109638000B208DF80C3095B1B5F5006F0FDA690184
:10964800ADF802204FF6FF72ADF80010ADF8042017
:10965800ADF80620ADF808308DF80D300EE0114653
:10966800ADF80020ADF802204FF6FF72ADF80420E7
:10967800ADF80620ADF808308DF80D10684607F0F3
:1096880035F902238DF80A307313F60046F0040604
:1096980000270124ADF8026068464FF6FF76ADF862
:1096A80000308DF80B708DF80C40ADF80460ADF803
:1096B8000660ADF808708DF80D4007F017F94FF007
:1096C8000303BD42B8468DF80A308DF80B708DF84B
:1096D8000C4010DD6B13ED0045F00405ADF80030CB
:1096E800ADF80250ADF80460ADF80660ADF808407A
:1096F8008DF80D400CE00423ADF80070ADF8023091
:10970800ADF80460ADF80660ADF808408DF80D704E
:10971800684607F0EBF8012414230726002509A85A
:109728008DF824308DF825608DF826508DF8274067
:1097380009F07AFA152309A88DF824308DF82560E8
:109748008DF826508DF8274009F06EFA132309A8E2
:109758008DF824308DF825608DF826508DF8274037
:1097680009F062FA02212246054807F0F9FA04488E
:109778001021224607F0F4FA0AB0BDE8F08100BFD4
:1097880000640040000C0240F0B5437887B00746FB
:10979800426833B104238DF80C3000230292019300
:1097A80003E08DF80C3001920293BB780DF10E02A4
:1097B800002B14BF022300238DF80D303B788DF861
:1097C8000E300023F918097A0133082B02F8011F1B
:1097D800F8D1114801A907F060F9042817D10F4DF5
:1097E8000F4B2C681B680134082C08BF00249C42CE
:1097F8000FD02E680B4B03EB061697E80F0086E890
:109808000F00012104480A462C6007F0A9FA01203C
:1098180000E0002007B0F0BD00640040D04A0020FE
:10982800D44A00205C4B002070B50D4B0D4C05460A
:1098380022681B689A420FD026680B4B03EB06136D
:1098480001360FCB85E80F0026602368082B05D169
:1098580000232360012070BD002070BD012070BD71
:10986800584B0020CC4A0020D84A00202DE9F04F60
:1098780001218BB04FF4805007F0CEFF6A4D0120D4
:1098880000240226E023014608938DF826408DF82F
:1098980027408DF824608DF8256007F08DFF284655
:1098A80008A907F0D1FD052128460A4607F04FFE12
:1098B800DFF8808128460621052207F048FE0522A8
:1098C8002846072107F043FE012520234FF4827A1A
:1098D8004FF4007B404603A9ADF81830ADF80C40B2
:1098E800ADF81040ADF81A40ADF81C40ADF80EA028
:1098F800ADF81260ADF81450ADF816B008F090F855
:109908004046294608F027F929464FF4804007F0D9
:1099180077FF08F554484FF46043304629460893CA
:109928008DF826408DF827408DF824608DF8256045
:1099380007F042FF404608A907F086FD40460D2182
:10994800052207F004FE40460E21052207F0FFFD20
:10995800052240460F21A8F5E63807F0F8FD102348
:10996800404603A9ADF818300193ADF80C40ADF8A6
:109978001040ADF81A40ADF81C40ADF80EA0ADF897
:109988001260ADF81450ADF816B008F049F840462A
:10999800294608F0E0F8254F29464FF4004007F023
:1099A8002FFF4FF4E0520420294608928DF82640F4
:1099B8008DF827408DF824608DF8256007F0FCFEAF
:1099C800384608A907F040FD38460A21062207F064
:1099D800BEFD38460B21062207F0B9FD38460C219A
:1099E800062207F0B4FDADF80C40ADF81040ADF814
:1099F8001A40ADF81C400E4C019B204603A9ADF857
:109A08000EA0ADF81260ADF81450ADF816B0ADF870
:109A1800183008F005F820462946B14608F09BF8AA
:109A28000BB0BDE8F08F00BF000002400008024004
:109A3800003C00400030014070B504460D46164613
:109A4800042876D8DFE800F003090D120600022288
:109A58003A4B09E00122394B01E0394B10225A8375
:109A680009E0384B4FF480525A8315E0344B4FF4D9
:109A780000425A8321E03448022108F0FDF800280A
:109A8800F9D03148294608F0C1F82F48012108F0DB
:109A9800F3F80028F9D020E02C48022108F0ECF86F
:109AA8000028F9D02948294608F0B0F827480121AC
:109AB80008F0E2F80028F9D00FE02548022108F064
:109AC800DBF80028F9D02248294608F09FF82048FA
:109AD800012108F0D1F80028F9D0D6B1042C28D8F3
:109AE800DFE804F003090D1206000222134B09E017
:109AF8000122124B01E0124B10221A8310E0114B85
:109B08004FF480521A830DE00D4B4FF400421A8334
:109B18000AE0042C0FD8DFE804F00503050703006A
:109B2800094802E0094800E0094808F06CF8C0B2AA
:109B380070BD002070BD002070BD00BF0010024045
:109B4800000002400004024000300140003800409C
:109B5800003C004000000000F8B50BF059FB0AF08B
:109B68003BFF00222E4B0AF08BFF21A3D3E90023F1
:109B78000AF086FF04460D4622462B461CA1D1E971
:109B880000010AF0C9FD1CA3D3E9002306460F46CD
:109B9800204629460BF09EF802460B4630463946C9
:109BA8000BF098F80BF02EFA0AF016FF00221D4B66
:109BB8000BF090F80DF048FA11A3D3E900230AF04E
:109BC8005FFF11A3D3E900230AF0A8FD02460B4664
:109BD8000FA1D1E900010BF07DF80FA3D3E9002311
:109BE8000AF09AFD0BF00EFA0BF030FDF8BD00BF3D
:109BF8006666666666660A409A99999999990140D7
:109C0800C3F5285C8FA272400000000000FEAA4045
:109C18009A999999FD6F2F41C3F5285C8F1271406D
:109C28000000303F000024402DE9F04101219CB0A4
:109C38004FF4800007F0C0FD01214FF4807000252B
:109C480007F0EAFD032633231AA948481A938DF82A
:109C58006F508DF86C6007F0F7FB1AA94448DFF8DD
:109C680020818DF86F501A968DF86C6007F0ECFB28
:109C780001214FF4800007F09FFD01214FF480700F
:109C880007F0CAFD404607F05BF93A4B01240293FE
:109C9800394B062703934FF4806307934FF400630F
:109CA80008934FF4005309934FF480730A93404686
:109CB8004FF4003301A90B930195049506950C9573
:109CC8000E950F9505970D9407F0C6F92146404665
:109CD80007F0FDF916A8169517951895199506F029
:109CE800F3FB1095129513951495244D10A9284649
:109CF8008DF844408DF845408DF8547006F0B5FB5A
:109D08002846214606F0AEFC28460A21224623466C
:109D180006F026FC28460E210222234606F020FCE7
:109D280028460F213246234606F01AFC2846082109
:109D38000422234606F014FC28462346092105225E
:109D480006F00EFC3A46234628460B2106F008FC8E
:109D58002846214606F08FFC2846214606F0CEFB11
:109D6800284606F04BFC1CB0BDE8F0810008024014
:109D7800000402404C2001403C0600200020014025
:109D8800106402400B2820D8DFE800F0061F1F1FD0
:109D9800091F1F1F0D15181B0D4B188801E00C4BD0
:109DA800588880B270470A4B588940F2712380B2B4
:109DB800584300137047064B988804E0044BD88832
:109DC80001E0034B188980B2C6E60020704700BF47
:109DD8003C060020AFF300800C4B072202FB00304A
:109DE80090F800380B7090F801384B7090F80238F2
:109DF8008B7090F80338CB7090F804380B7190F89A
:109E080005384B7190F806388B717047480600206A
:109E1800254938B500224FF400635A540133B3F58D
:109E2800804FFAD14FF40064002006210122FFF789
:109E380003FE002005210246FFF7FEFD0020012257
:109E48000146FFF7F9FD8007F3D5002002210246FD
:109E5800FFF7F2FD0020C4F307210246FFF7ECFDEF
:109E68000020E1B20246FFF7E7FD0025A5F13F011A
:109E78004A4242EB0102002001460135FFF7DCFDB2
:109E8800402DF3D1002005210246FFF7D5FD002023
:109E980001220146FFF7D0FDC307F3D44034B4F5DF
:109EA800804FC1D138BD00BF48060020F7B507254F
:109EB800454300200C4602460321FFF7BDFD05F58A
:109EC80000650020C5F307210246FFF7B5FD002015
:109ED800E9B20246FFF7B0FD002001460246FFF74F
:109EE800ABFD0746002001460246FFF7A5FD0646E2
:109EF800002001460246FFF79FFD05460020014667
:109F08000246FFF799FD8DF803000020014602463E
:109F1800FFF792FD8DF80400002001460246FFF786
:109F28008BFD8DF80500002001220146FFF784FD16
:109F380023788DF80600BB4210D16378B3420DD167
:109F4800A378AB420AD1DDF80300D4F80330C3EBA1
:109F5800000CDCF1000040EB0C0000E00020FEBD2E
:109F680038B51B4B04460D46195500200621012221
:109F7800FFF762FD002005210246FFF75DFD002086
:109F880001220146FFF758FD8207F3D50020022180
:109F98000246FFF751FD0020C4F307210246FFF7F0
:109FA8004BFD0020E1B20246FFF746FD002029469E
:109FB8000122FFF741FD002005210246FFF73CFD85
:109FC800002001220146FFF737FDC307F3D438BD4F
:109FD8004806002038B50725454305F500650C46B9
:109FE80028460978FFF7BCFF681C6178FFF7B8FFBF
:109FF800A81CA178FFF7B4FFE81CE178FFF7B0FFD1
:10A00800281D2179FFF7ACFF681D6179FFF7A8FFCC
:10A01800A179A81DBDE83840A2E72DE9F843164606
:10A02800424A044688460023121803E018F8031031
:10A03800D1540133B342F9D1002006210122FFF7A0
:10A04800FBFC002005210246FFF7F6FC0020012258
:10A058000146FFF7F1FC8307F3D5002002210246F1
:10A06800FFF7EAFC0020C4F307210246FFF7E4FCEF
:10A078000020E1B20246FFF7DFFC0025771E44E02E
:10A08800013414F03F0918F8051006D0C7EB050E87
:10A09800DEF1000242EB0E0200E00122D2B2002003
:10A0A800FFF7CAFCB9F1000F2ED1BD422CD2002017
:10A0B80005210246FFF7C0FC002001220146FFF7F8
:10A0C800BBFC10F00100F2D106210122FFF7B4FC1D
:10A0D800002005210246FFF7AFFC002001220146BF
:10A0E800FFF7AAFC8007F3D5002002210246FFF7FC
:10A0F800A3FC0020C4F307210246FFF79DFC0020C3
:10A10800E1B20246FFF798FC0135B542B8D100200C
:10A1180005210246FFF790FC002001460122FFF7C7
:10A128008BFCC107F3D4BDE8F88300BF48060020C4
:10A13800014B185C704700BF4806002010B5054C5D
:10A148000023201802E0C45CCC5401339342FAD1B6
:10A1580010BD00BF48060020F7B5002003210246C5
:10A16800FFF76AFC002001460246FFF765FC002065
:10A1780001460246FFF760FC504D002443F6FF7687
:10A18800A11B4A4242EB010200200146FFF754FCA2
:10A1980060550134B4F5804FF2D100200521024604
:10A1A800FFF74AFC002001220146FFF745FC10F0AA
:10A1B8007104F2D1FEF756F840F2CF7607463F4DCC
:10A1C80006E095F8FF47A4F14202544244EB02042A
:10A1D800FEF748F8C01B0028B8BF4042B04202DC76
:10A1E800002CEED000E01CB1354B1B78002B4FD073
:10A1F80040F2FF700021FFF7B3FEFFF709FE0020D1
:10A2080030494022FFF709FF4FF480702E49B422ED
:10A21800FFF703FF40202D492022FFF7FEFE4FF4F1
:10A22800DA702949B422FFF7F8FE60202749202276
:10A23800FFF7F3FE4FF41A702349B422FFF7EDFE3F
:10A24800802022492022FFF7E8FE02AD002345F8CE
:10A25800043D4FF4C3642046042229460434FFF722
:10A26800DCFEB4F5FF6FF6D102AD002345F8043DDE
:10A278004FF4A7642046042229460434FFF7CDFE94
:10A28800B4F5C36FF6D140F2FF704221FFF768FEC4
:10A29800002040220B49FFF751FF402020220C49A3
:10A2A800FFF74CFF602020220A49FFF747FF802074
:10A2B80009492022FFF742FFFEBD00BF48060020E3
:10A2C800304C0020040000202077010800770108A6
:10A2D800A84C0020C84C0020E84C002000000000DA
:10A2E8002DE9F04113780646C3F34117032F0D46B5
:10A2F800144631D0464A02EB4712127B62BBD9079B
:10A308002AD45F2B28D8434AD25D2ABB13F09F0377
:10A3180001D0082B20D1DFF8048118F8073083B961
:10A328003B4B03EB4713D97F21B13846FEF774F84E
:10A33800032304E0597A3846FEF76EF8022308F83A
:10A348000730DFF8DC8018F807302BB1384601F009
:10A35800D3F8002308F80730002221780420FFF7FB
:10A368006BFB2870002261780420FFF765FB68709A
:10A378000022A1780420FFF75FFBA87001220420C7
:10A38800E178FFF759FBE8702378DA073ED45F2BB2
:10A398003CD803F01E02082A04D0142A2CD0062A1E
:10A3A80034D11AE0242171435B090C2000FB03130C
:10A3B800A678E578184A45EA0625D550A3781B07FC
:10A3C80024D52678760900FB061693596FEA0353BD
:10A3D8006FEA13539351BDE8F081242256435B0979
:10A3E8000C2202FB0363A178E2780B4E42EA0122B9
:10A3F800F3185A60BDE8F08124214E435B090C2113
:10A4080001FB0363044EE278F3181A72BDE8F08189
:10A41800A84C0020604D0020584C00205D4D0020C5
:10A42800634D002007B513788DF800108DF80130C2
:10A43800537801A98DF8023093786A468DF8033075
:10A44800FFF74EFF0EBD07B58DF802309DF81030AE
:10A458008DF800108DF8012001A96A468DF80330A7
:10A46800FFF73EFF0EBD07B500238DF800108DF8ED
:10A4780001308DF80320131201A96A468DF80230C5
:10A48800FFF72EFF0EBD5F29F7B506460D461446A9
:10A4980058D811F01E07C1F3411202D0022F51D132
:10A4A8001DE0032101FB00222E491301C818CC50DE
:10A4B8004368C3EB040EBEF1000FB8BFCEF1000E27
:10A4C800BEF5000F09DB9C42CCBF274C274C01EBA3
:10A4D80002121C190123137334E0077332E00327B7
:10A4E80007FB00271F483901431824F07F4C5C60A4
:10A4F80003F1080EC3F808C04358191B0029B8BF58
:10A508004942B1F5000F1ADBA342CCBF164B174BDB
:10A518005201E3188DF800201A148DF801201A1240
:10A528008DF80220304601A96A468DF80330FFF7FE
:10A53800D7FE0C4B03EB071701233B7302E0002304
:10A548008EF8043023148DF801303046231201A907
:10A558006A468DF800508DF802308DF80340FFF7F9
:10A56800BFFEFEBDA44D0020FFFF7F00010080FF5D
:10A5780011F01E0307B501D0022B03D10022FFF70B
:10A5880082FF0CE000238DF800106A4601A98DF8BF
:10A5980001308DF802308DF80330FFF7A1FE0EBDB3
:10A5A800012104200A46FFF747BA13B541F001011B
:10A5B80014468DF8041001AA6946FFF791FE9DF82C
:10A5C80001309DF8000023709DF8023063709DF8FB
:10A5D8000330A3701CBD07B541F001018DF80410CC
:10A5E80001AA6946FFF77CFE9DF803309DF802003A
:10A5F80043EA0020030544BF6FEA00506FEA105099
:10A608000EBD73B54D01EDB245F01503164601A90F
:10A618006A4604468DF80030FFF762FE9DF8053063
:10A6280045F014058DF801309DF80630204601A943
:10A638006A468DF800508DF802308DF80360FFF7F8
:10A648004FFE7CBD73B54D01EDB245F015031646BE
:10A6580001A96A4604468DF80030FFF741FE9DF8CF
:10A66800053045F014058DF801309DF80730204677
:10A6780001A96A468DF800508DF802608DF8033004
:10A68800FFF72EFE7CBD2DE9F74F4FEA40185FFA21
:10A6980088F84FEA4159002048F0180101AAFFF74D
:10A6A80084FF9DF805404FEA5959250904F00F0425
:10A6B800AC4248460EDB0AF06DF9641B06460120E1
:10A6C80000FA04F00F460AF075F90022324B0AF03E
:10A6D800D7F90FE00AF05EF92C1B0646012000FAB4
:10A6E80004F00F460AF066F902460B4600202A4994
:10A6F8000AF0F0FA02460B46304639460AF0EAFA02
:10A708000AF080FC0AF068F921A3D3E900230AF0D3
:10A71800B7F90AF077FC0AF05FF900221F4B0AF03C
:10A72800AFF94FF0FF3582468B462E4600240127AD
:10A7380000E0064607FA04F00AF03CF90B46024628
:10A74800594650460AF09CF90AF034FCA0F18003FF
:10A75800802B28BF304638BF254601340E2CE8D15F
:10A7680000248DF8050048F01201204601AA8DF852
:10A7780004408DF80650FFF755FE204648F00C01BE
:10A788004A46FFF770FE2046BDE8FE8FAFF3008013
:10A7980004560E2DB29DEF3F00006040000020409F
:10A7A800B4234343F7B54A08032606FB023606F5E9
:10A7B8008077044638460D46FFF7BAFC8DF804004A
:10A7C800781CFFF7B5FC8DF8050006F58170FFF7DA
:10A7D800AFFC45EA44148DF80600E1B2002001AA56
:10A7E800FFF720FEFEBD37B50D4641EA401101AA2C
:10A7F8000446C9B20020FFF7D8FEB4235C436D08B5
:10A80800032303FB054404F580759DF804102846CE
:10A81800FFF7A6FB681C9DF80510FFF7A1FB04F5E0
:10A8280081709DF80610FFF79BFB3EBD10B5C4B2C2
:10A838002146640100200222E4B2FFF7E2FE44F060
:10A8480008010020FFF794FE44F00A010020BDE84B
:10A8580010408DE637B5440144F01604E4B20D46C5
:10A8680001AA21460020FFF7A0FE9DF8053015F04B
:10A87800010F14BF43F0400323F040038DF8053067
:10A888009DF8053015F0020F14BF43F0100323F0B4
:10A8980010032146002001AA8DF805308DF8060026
:10A8A800FFF7C0FD3EBD37B5440144F01604E4B2DD
:10A8B8000D4601AA21460020FFF777FE9DF80530D6
:10A8C80015F0010F14BF63F07F0303F07F038DF8C9
:10A8D80005309DF8053015F0020F14BF43F0200332
:10A8E80023F020032146002001AA8DF805308DF8B9
:10A8F8000600FFF797FD3EBD07B5410141F016017F
:10A9080001AAC9B20020FFF750FE9DF80530C3F335
:10A918008010DA0648BF40F002000EBD07B54101BD
:10A9280041F01601C9B2002001AAFFF73EFE9DF8CA
:10A938000530D809990648BF40F002000EBD70B531
:10A94800104C04EB00139A682646914209DD8A1AD6
:10A95800C2F18074A2425D6801DCAA1809E02C1BD0
:10A968000AE00ADA521AC2F18074A2425D6802DC77
:10A97800AA1A5A6001E02C195C6006EB001081608D
:10A9880070BD00BFA44D002037B541F001030C464F
:10A9980001AA694605468DF80430FFF7A1FC9DF829
:10A9A80002109DF80130090241EA03419DF8033085
:10A9B8001943080248BF41F07F415F2C1AD8C4F3FD
:10A9C800411314F01E0402D0022C13D106E0032216
:10A9D80002FB0535084B2D0159590BE0032202FBF8
:10A9E800053521F07F41E8B2FFF7A9FF024B03EBE1
:10A9F8000515696808463EBDA44D002073B51C4B7B
:10AA0800587E10F0010004D00020682140F2211285
:10AA180002E068214FF49072FFF735FD0020022311
:10AA280000937E2102460346FFF70DFD00241BE03C
:10AA3800E9B230460135FFF7B3FE1D2DF8D1750197
:10AA4800EDB245F00C010020FFF79EFF01463046AD
:10AA5800FFF719FE0134002045F0160143F2FF12FA
:10AA6800FFF701FD032C02D00025E6B2E0E77CBD2C
:10AA78000400002038B50D4668210446FFF784FF1E
:10AA880015B140F0010201E020F0010220466821E2
:10AA9800BDE83840F7E47FB54301044643F00303BB
:10AAA80003AA002002A98DF80C30FFF719FC9DF8C5
:10AAB8000A109DF80930090241EA03419DF80B305C
:10AAC80020461943154DFFF73AFF2001291801F1D7
:10AAD80008031A7902B3124A0C2606FB0422127ADA
:10AAE800D2B928584968451A002DB8BF6D42B5F546
:10AAF800000F05DB8842CCBF0A480B48081800E065
:10AB08001A716401C0F30742C0F30723C0B2009072
:10AB1800E1B20020FFF797FC7FBD00BFA44D0020E5
:10AB2800584C0020FFFF7F00010080FFAFF300803A
:10AB3800F8B50F4B0E461D5CC1F3074100222846AD
:10AB4800FEF77AFF0B4C0702C6F3072100222846BE
:10AB58002760FEF771FF07433F02F1B22846012242
:10AB68002760FEF769FF07433F092760F8BD00BF6C
:10AB7800507701084846002010B5124B0022C1004A
:10AB88005A605A18527B12B14FF400725A605B181F
:10AB98009B7B0C4A1BB1536843F480735360094C88
:10ABA800C300E218D17B0F2901D90F21D173E31813
:10ABB800D97B636819436160FFF7BAFF6368236252
:10ABC80010BD00BF484600202A4B032110B501FBE9
:10ABD800003292F925403F2C02DD3F2482F82540BF
:10ABE80001FB003393F925203F3202DAC12283F8B2
:10ABF8002520204B032202FB003292F826101F2941
:10AC080002D91F2182F826104FF440225A600322ED
:10AC180002FB003393F82430012B03D1154B4FF47A
:10AC280050225A60134B032103EBC00292F83420E0
:10AC380001FB003122B991F8252002F07F0206E0DD
:10AC480091F8251002F0030201F07C010A435968CB
:10AC5800084C41EA02225A60032303FB004393F89D
:10AC68002610636819436160FFF762FF6368A36495
:10AC780010BD00BF48460020274B052110B501FB39
:10AC8800003292F84C40012C02D9012482F84C4041
:10AC980001FB003393F84D20032A02D9032283F8DD
:10ACA8004D201D4B052101FB003292F84E400F2C20
:10ACB80002D90F2482F84E4001FB003393F84F204D
:10ACC800032A02D9032283F84F20134C052303FBE0
:10ACD800004292F850100F2902D90F2182F8501023
:10ACE80003FB004393F8501093F84C2041F42021C3
:10ACF80041EAC23193F84D2041EA423193F84E209F
:10AD080093F84F3041EA022141EA43116160FFF7AD
:10AD18000FFF6368E36510BD4846002038B5234B34
:10AD28004FF460225A60C200991891F8341011B19A
:10AD38004FF4702159609A1892F82E1092F82D400D
:10AD4800090341EA84315C682143596092F82F3045
:10AD5800012B03D1154B41F480615960134BC1009D
:10AD68005C185A6894F8305094F8314042EA052249
:10AD7800012C5A6004BF42F080025A605B1893F8B5
:10AD880032300A4A012B03D1536843F04003536021
:10AD9800064C04EBC00393F83310636843EA0111CF
:10ADA8006160FFF7C5FE6368236638BD484600202A
:10ADB800524B0B2110B501FB003292F86440032C72
:10ADC80002D9032482F8644001FB003393F866201B
:10ADD800032A02D9032283F86620484B0B2101FB82
:10ADE800003292F868400F2C02D90F2482F868408C
:10ADF80001FB003393F86920072A02D9072283F858
:10AE080069203E4B0B2101FB003292F86A400F2C5F
:10AE180002D90F2482F86A4001FB003393F86D20B1
:10AE28000F2A02D90F2283F86D2034490B2202FB26
:10AE3800001393F86E400F2C02D90F2483F86E404C
:10AE480002FB001292F86430DB0343F400244C60E8
:10AE580092F8651019B1294A43F404235360274B2B
:10AE68000B2202FB003292F867201AB15A6842F4AA
:10AE780000525A600B2279B902FB003292F868102E
:10AE880092F86640C90141EAC4215C6892F86920D9
:10AE9800214341EA02121DE002FB003292F86C30B5
:10AEA80016491BB14B6843F480534B60134B0B227C
:10AEB80002FB003292F86E1092F86D405A6842EA2E
:10AEC800C41201F0070442EA041209075A6002D5C5
:10AED80042F400625A60094C0B2303FB004393F8C9
:10AEE8006B2022B993F86A20636813436360616832
:10AEF800FFF71EFE6368C4F8883010BD484600207E
:10AF08002E4A2DE9F84FA2F1400A00210AF109085A
:10AF18000D460C464FF001094FF0050E03260B466F
:10AF2800022708F11F0CA2F15C0B0AEB040004F8DD
:10AF38000A9080F801E080F802E008EB050005F8C7
:10AF48000860033446708370C370037180F80590FD
:10AF58008771C3710CEB010001F80C301770437056
:10AF68008370C370037153700BEB0500D37093703B
:10AF78001771567182F806E0D37113729672537284
:10AF8800083505310B32092C43718371C371CCD15B
:10AF98000025ECB22046FFF76FFE2046FFF714FEAF
:10AFA8002046FFF7BBFE2046FFF7E6FD01352046A9
:10AFB800FFF7FEFE032DECD1BDE8F88FAC4600206C
:10AFC800044B042903EBC003D97301D000225A7340
:10AFD800D2E500BF48460020034B03EBC00359737A
:10AFE80009B10422DA73C7E548460020024B03EB97
:10AFF800C0039973C0E500BF48460020024B03EB2D
:10B00800C000C07B704700BF48460020024B03EBDE
:10B01800C000407B704700BF48460020024B03EB4E
:10B02800C000807B704700BF48460020034B0B22BE
:10B0380002FB003383F86410BAE600BF48460020DC
:10B04800034B0B2202FB003383F86510B0E600BF08
:10B0580048460020034B0B2202FB003383F867109D
:10B06800A6E600BF48460020034B0B2202FB003334
:10B0780083F866109CE600BF48460020034B0B226D
:10B0880002FB003383F8681092E600BF48460020B0
:10B09800034B0B2202FB003383F8691088E600BFDC
:10B0A80048460020034B0B2202FB003383F86A104A
:10B0B8007EE600BF48460020034B0B2202FB00330C
:10B0C80083F86C1074E600BF48460020034B0B223F
:10B0D80002FB003383F86D106AE600BF4846002083
:10B0E800034B0B2202FB003383F86E1060E600BFAF
:10B0F80048460020034B0B2202FB003090F8640006
:10B10800704700BF48460020034B0B2202FB00306B
:10B1180090F86500704700BF48460020034B0B229B
:10B1280002FB003090F86700704700BF48460020D7
:10B13800034B0B2202FB003090F86600704700BFFB
:10B1480048460020034B0B2202FB003090F86800B1
:10B15800704700BF48460020034B0B2202FB00301B
:10B1680090F86900704700BF48460020034B0B2247
:10B1780002FB003090F86A00704700BF4846002084
:10B18800034B0B2202FB003090F86C00704700BFA5
:10B1980048460020034B0B2202FB003090F86D005C
:10B1A800704700BF48460020034B0B2202FB0030CB
:10B1B80090F86E00704700BF48460020034B0522F8
:10B1C80002FB003383F84C1056E500BF48460020C8
:10B1D800034B052202FB003383F84D104CE500BFFA
:10B1E80048460020034B052202FB003383F84E102B
:10B1F80042E500BF48460020034B052202FB00330E
:10B2080083F84F1038E500BF48460020034B05225D
:10B2180002FB003383F850102EE500BF484600209B
:10B22800034B052202FB003090F84C00704700BF2A
:10B2380048460020034B052202FB003090F84D00E1
:10B24800704700BF48460020034B052202FB003030
:10B2580090F84E00704700BF48460020034B052277
:10B2680002FB003090F84F00704700BF48460020AE
:10B27800034B052202FB003090F85000704700BFD6
:10B2880048460020034B032202FB003383F82410B6
:10B298009AE400BF48460020034B032202FB003318
:10B2A80083F8251090E400BF48460020034B032292
:10B2B80002FB003383F8261086E400BF48460020CE
:10B2C800034B032202FB003090F82400704700BFB4
:10B2D80048460020034B032202FB003090F925006A
:10B2E800704700BF48460020034B032202FB003092
:10B2F80090F82600704700BF48460020024B03EB39
:10B30800C00383F82D1009E548460020024B03EBE3
:10B31800C00383F82E1001E548460020024B03EBDA
:10B32800C00383F82F10F9E448460020024B03EBD2
:10B33800C00383F83010F1E448460020024B03EBC9
:10B34800C00383F83110E9E448460020024B03EBC0
:10B35800C00383F83210E1E448460020024B03EBB7
:10B36800C00383F83310D9E448460020064B10B5D3
:10B3780003EBC00383F834100446FFF7CFFC2046E4
:10B38800BDE8104020E400BF48460020024B03EB14
:10B39800C00090F82D00704748460020024B03EB90
:10B3A800C00090F82E00704748460020024B03EB7F
:10B3B800C00090F82F00704748460020024B03EB6E
:10B3C800C00090F83000704748460020024B03EB5D
:10B3D800C00090F83100704748460020024B03EB4C
:10B3E800C00090F83200704748460020024B03EB3B
:10B3F800C00090F83300704748460020024B03EB2A
:10B40800C00090F834007047484600202DE9F04706
:10B41800314F98463B1893F88C3004460D46164633
:10B42800DDF820A0DDF82490042B1AD8DFE803F01B
:10B4380003080D121700FFF7BBFC3B19012212E0AD
:10B44800FFF76CFC3B1902220DE0FFF715FC3B19D6
:10B45800032208E0FFF7B8FB3B19042203E0FFF7DB
:10B468008BFB3B19002207EBC40483F88C2094F86B
:10B478003320194B012A0DD002D3022A23D111E01F
:10B4880015B11B689B0C2B70EEB1134B1B689B0A04
:10B49800337018E0B8F1000F15D01B689B0AC8F884
:10B4A800003010E0B8F1000F04D01B68DB0B5B0123
:10B4B800C8F80030BAF1000F05D0074B1B68C3F37A
:10B4C80084238AF80030B9F1000F03D0024B1B68BF
:10B4D80089F80030BDE8F08748460020054B0B226C
:10B4E80002FB003393F86B201AB9012283F86B2012
:10B4F8005EE4704748460020054B0B2202FB0033F0
:10B5080093F86B201AB1002283F86B2050E470473F
:10B518004846002006281DD8DFE800F004070A0E78
:10B52800111418000C4B1B680EE00B4B1B6A0BE048
:10B53800094BD3F8883007E0074BDB6D04E0064B76
:10B548009B6C01E0044B1B6E0B607047024B93F839
:10B558006B300B60704700BF48460020704770474B
:10B568007047704770477047704712230B80014837
:10B57800704700BF4400002004230B800048704738
:10B5880056000020002070470020704700207047B8
:10B5980070B5084C0022236806E03F2B03D8865C70
:10B5A800E5182E71013301328A42F6D1014A002092
:10B5B800136070BDD846002010B5044C0A460448F4
:10B5C800214608F041F8204610BD00BF9B610020CD
:10B5D8003F78010810B5044C0A460448214608F093
:10B5E80033F8204610BD00BF9B6100204D7801084C
:10B5F80010B5044C0A460448214608F025F82046B0
:10B6080010BD00BF9B6100205878010810B5044C9C
:10B618000A460448214608F017F8204610BD00BF26
:10B628009B6100206078010810B5044C0A46044864
:10B63800214608F009F8204610BD00BF9B61002094
:10B6480078780108202802D0212822D112E08A78AF
:10B658004878120442EA002208780F4B0243C8785F
:10B6680042EA00629A610A791A774A795A778A799E
:10B678009A770EE0084B9A69100A0A704870100C05
:10B68800120ECA701A7F88700A715A7F9B7F4A719E
:10B698008B710020704700BF44000020F7B5274C8D
:10B6A8004FF4C0530026032700932046022369461F
:10B6B8008DF804308DF805708DF806608DF80760F8
:10B6C80005F0C2FE20460B210A2205F040FF0A229F
:10B6D80020460C2105F03BFF01254FF4007320465E
:10B6E800694600938DF805708DF804608DF8065052
:10B6F8008DF8076005F0A8FE0A222046092105F00A
:10B7080026FF4FF480632046694600938DF8065063
:10B718008DF807508DF8057005F096FE0A210A4647
:10B72800204605F014FF29464FF4804006F074F8CF
:10B738008020294606F04CF8FEBD00BF00000240FC
:10B7480007B54FF4C06007F065FA43238DF804305D
:10B758000322012301A88DF805308DF806208DF805
:10B76800073007F061FA0EBD782358430723B0FB72
:10B77800F3F0002301338342FCD970474FF47A7306
:10B788005843F1E7684620F007018D4601B50348A4
:10B7980008F052FDBDE8014085467047D44D0020B1
:10B7A8000023F0B5094C0A4F40F2FF751E460AE027
:10B7B800226810F803C007F802C00132AA4288BF05
:10B7C8003246226001338B42F2D1F0BD944A002008
:10B7D8009B590020074910B50A684AB10023043173
:10B7E8005C5CC45401339342FAD1024B00211960C6
:10B7F800104610BDD8460020084B1B68082B0BD9F3
:10B808000023064A111D595CC1540133092BF8D194
:10B81800002313600120704700207047D84600209D
:10B8280007B5054B054803F120023C33009301217D
:10B83800034B07F069FB0EBD44000020D44D0020E7
:10B8480058010020014808F0CBBC00BFD44D0020AF
:10B8580010B5844A91781346022900F03C810329E7
:10B8680000F04081002940F0E48153784D2B00F02E
:10B87800AE8022D8452B6BD00ED8422B55D005D898
:10B88800402B44D0412B40F0D28145E0432B51D08E
:10B89800442B40F0CC8153E0482B73D005D8462B7D
:10B8A8005BD0472B40F0C38163E04B2B7DD000F287
:10B8B8008880492B40F0BB816AE0542B00F0D88087
:10B8C80011D8512B00F0A38006D84F2B00F08480AC
:10B8D800502B40F0AC8194E0522B00F0A880532B01
:10B8E80040F0A581ABE0832B00F0E18006D8552B12
:10B8F80000F0CA80572B40F09A81D1E0852B00F0E8
:10B90800E080C0F0D880FF2B40F09181DFE0554BFC
:10B9180040F2FF70D97804E0524B0020D978524B9E
:10B928001970BDE81040FEF71BBBD1784E4B0120C3
:10B938005970F6E74B4B0420D9784B4B1971F0E757
:10B94800484B4949D3F803301C2041F81C3F0BE011
:10B95800D178454B05205971E3E7424B4249D3F86A
:10B9680003300C2041F80C3F0422BDE81040FEF7DC
:10B9780054BB3C4B3C4CD3F80330214641F8083FBC
:10B98800082064E0D3783849262001F8263F79E07A
:10B99800344BDA78344B0AB9DA7503E033490122BB
:10B9A800DA754A60D97D1720BBE72E4B2E4CD97823
:10B9B8000320E170FEF7D4FAE078BDE81040FDF707
:10B9C8004BBC284B0220D978274B9970A9E7D1782E
:10B9D800254B15205975A4E7224B234CD3F80310A7
:10B9E8001920C9B26176FEF7BBFA607E10F001003B
:10B9F80002D00020012100E00146BDE81040FFF719
:10BA080039B8184B1620D978174B997589E7164B12
:10BA1800197D1C4611F0010F04D0D378DB0701D43F
:10BA2800FEF7F6F90F4B1420D978217579E70D4BFD
:10BA38000D49D3F80330202041F8203F94E7094B03
:10BA4800094CD3F80330214641F8103F1020042256
:10BA5800FEF7E3FA6079A1682269BDE81040FDF7B6
:10BA68003FBD00BFC853002004000020E45400205C
:10BA7800D2F80330012B00F2DC80D3786F491A200A
:10BA880001F81A3F012270E76D4BD3F80320012A11
:10BA980000F2CF80DB7869491B2001F81B3FF1E7F2
:10BAA800674B6649DB78272001F8273FEAE7D2F899
:10BAB8000320644B03E0624BD3F80320624B1A6007
:10BAC80010BD5F4BD3F803205E4B5A6010BD5C4B32
:10BAD800DA785E4BAFE051785D4BD2F8032043F83B
:10BAE800212010BD52782E2A00F2A180DFE812F042
:10BAF8002F00380041009F009F009F009F009F007B
:10BB08009F004A004F0054009F009F009F009F0025
:10BB18009F009F009F009F009F009F009F009F0025
:10BB28009F009F009F0059005D00610068006C0045
:10BB380070009F009F009F009F009F009F0077005C
:10BB48007C00810086008B00900095009A00D3F855
:10BB58000320404B1A60FCF785FB3A4B986010BDF8
:10BB6800D3F803203B4B5A60FCF77CFB354BD8607D
:10BB780010BDD3F80320374B9A60FCF773FB314BA9
:10BB8800186110BDD3F80320324BDA6010BDD3F82A
:10BB98000320304B1A6110BDD3F803202D4B5A6196
:10BBA80010BDD3F80310002006E0D3F803100020DE
:10BBB80011E0D3F803100120BDE81040FEF74ABE9B
:10BBC800D3F80310012006E0D3F803100220F3E7AE
:10BBD800D3F803100220BDE81040FEF764BED3F886
:10BBE80003201C4B9A6110BDD3F80320194BDA616E
:10BBF80010BDD3F80320174B1A6210BDD3F80320E9
:10BC0800144B5A6210BDD3F80320124B9A6210BD30
:10BC1800D3F803200F4BDA6210BDD3F803200D4B85
:10BC28001A6310BDD3F803200A4B5A6310BD0322D0
:10BC380000E00422084B1A7010BD00BF0400002069
:10BC4800C85300201C470020E0540020DE54002088
:10BC5800FC540020144D0020E454002037B5444B18
:10BC68001A7D9AB9434AD2F80320511C4FF00A01B1
:10BC780004D1414A12685143996101E04A439A61EB
:10BC8800FCF7F0FA3A4B0122D8611A75394C6378FF
:10BC9800042B6CD8DFE803F00328303E1100FCF7D2
:10BCA800E1FA334BDA69801A9A690028B8BF404232
:10BCB800904259D900221A7559E0A07803F07EFD08
:10BCC8002B4C08B9207536E0A369002B4BD0FCF744
:10BCD800C9FAE369C01AA3690028B8BF404298426C
:10BCE80041D90023237538E00020FEF759FCA578D8
:10BCF8006D0040FA05F518E000207C2101AAFEF746
:10BD080054FCA57802236D0003FA05F59DF806306A
:10BD18001D400CE000207C2101AAFEF746FCA57816
:10BD28009DF806306D0043FA05F515F00105104C35
:10BD380006D000232375114B1A6822F0100210E078
:10BD4800A36983B1FCF78EFAE369C01AA3690028D6
:10BD5800B8BF4042984206D92575084B1A6842F088
:10BD680010021A6003E0024B1A6A013A1A623EBDD9
:10BD78001C470020C8530020D0540020D053002076
:10BD880010B51F4B9A78012A1CD003D3022A1D4CE8
:10BD980021D11BE05878082802D8FCF79EFB0EE05A
:10BDA8000A2803D1174B00225A6016E00B2802D14B
:10BDB800FCF7D8FC03E0FF280FD1FCF7F9FB114B87
:10BDC80058600AE05878FDF7DDFFF8E75878FCF787
:10BDD800BBFB606001E0042323700B4B1B7873B13D
:10BDE800084B5A68094B1A60094B22B91A6842F085
:10BDF80008021A6010BD1A6822F008021A6010BD05
:10BE0800C8530020E4540020DF540020D054002000
:10BE1800D053002038B5204B5A78812A3AD19A78E5
:10BE2800922A37D19A79A32A34D15A79B42A31D1AE
:10BE38001A79C52A2ED1DB78D62B2BD1174B1C2289
:10BE48001A83FFF7FFFCFCF70DFA40F2E7340546CA
:10BE5800FCF708FA401B0028B8BF4042A042F7DDB3
:10BE680072B6FCF7BBFF0E4B00241C6021460D4840
:10BE780005F02DF90B4805F063F804F0E9FA05F030
:10BE8800FBF94FF0804005F095FF2046BDE83840AB
:10BE9800FCF796BF38BD00BFC85300200010024011
:10BEA80010E000E0106402402DE9F04706460D4618
:10BEB8001446002949D0002847D0814245D057016F
:10BEC800FFB247F0060841460020FEF75DFD47F047
:10BED8000C0182460020FEF757FD8146304609F0E6
:10BEE80097F90646284609F093F90146304609F0C5
:10BEF8009BFA0746504609F08BF9394609F094FA3F
:10BF080009F0A4FB0546484609F082F9394609F0CC
:10BF18008BFA09F09BFB0646002808BF01260C494E
:10BF28003846002D08BF012509F068FB18B12046E6
:10BF38003146FEF7A8FB002041462A46FEF7A3FA41
:10BF4800044B1C19012384F82430BDE8F08700BF96
:10BF58000000A0411C47002070B50D4D04462D1867
:10BF680095F824309BB1C6B20A4B710141F0060125
:10BF780053F82420C9B20020FEF775FA064B304664
:10BF880053F82410FEF77FFB002385F8243070BD9A
:10BF98001C470020FC580020F05400202DE9FF47E2
:10BFA800994B98781A46022803D95B78022B40F0FF
:10BFB800B8815378944C032B00F2B181DFE813F079
:10BFC8000400410092009101FFF7C6FFA1788F4B52
:10BFD80000255D548E4B28465D544901C9B2D4F8FA
:10BFE8000320FEF750FAA17828462A46FEF709FBF7
:10BFF800884EA37806EB43139B7F002B00F09481B7
:10C008002C46814DB046AB789C4215D008EB4313C3
:10C01800B27F9B7F9A420FD12046E7B2FFF79CFF81
:10C028007901C9B2D5F803200020FEF72CFA0020C8
:10C0380039460246FEF7E5FA01342036032CE2D1F0
:10C0480072E1FFF789FFA178704B00255D54704BB2
:10C0580028465D54490141F00201C9B2FEF794FC3B
:10C06800D4F80330A178C6184901C9B22846324627
:10C07800FEF709FA2A46A1782846FEF7C2FA664B67
:10C08800A2785E60634B03EB4212927F002A00F0B5
:10C098004B815D4E1C469846B07885421DD008EB12
:10C0A8004013A27F9B7F9A4217D1EFB24FEA4719FC
:10C0B8005FFA89F9FFF750FF49F002010020FEF707
:10C0C80063FCD6F803304946C2180020FEF7DBF9B6
:10C0D800002039460246FEF794FA01352034032D34
:10C0E800DAD121E110F0C0051DD1022800F2198132
:10C0F800D4F80330444E142B00F31381032202FBBF
:10C108000303464A52F82340FFF726FFB1783F4B16
:10C1180028465D543E4B22465D544901C9B2FEF79C
:10C12800B2F9B178F6E0402D40F0AA80D4F80320A7
:10C13800142A00F3F6800024009401940294234604
:10C1480040FA03F1CD0706D504AD29190134032CB3
:10C1580001F8043C02D00133032BF1D14FF003085E
:10C16800ADF104070025DFF8B49008FB02F815E0EC
:10C1780003ABEE5C01353046FFF7EEFE710141F08E
:10C188000201C9B20020FEF7FFFB464459F82630E9
:10C19800C01A0028B8BF404247F8040FA542E7DBA1
:10C1A800012C47DD022C0CD1009B01998B4203DD49
:10C1B8009DF80D2018463BE008469DF80C201946CE
:10C1C80036E0032C36D1009E019D029CAE420EDD66
:10C1D800A64209DD9DF80D2030462946FFF764FE8A
:10C1E8009DF80E2030460DE09DF80C2018E0A54281
:10C1F8009DF80C2014DD28463146FFF755FE9DF8C2
:10C208000E202846214613E0C85300201F4C00206A
:10C21800A04C0020A84C0020E4540020D453002057
:10C2280020463146FFF740FE9DF80D20204629465E
:10C23800FFF73AFE3D4EDFF8FC90DFF8FC80002463
:10C24800B37843FA04F2D10716D5D6F803200321B0
:10C2580001FB024236490025E7B2CD54790159F86D
:10C268002220C9B2284608F80350FEF70CF92846E0
:10C2780039462A46FEF7C5F90134032CE0D153E0CC
:10C28800802D51D1294ED6F80330142B49DCDFF824
:10C29800A490DFF8A4800024B37843FA04F3DA0703
:10C2A8001BD5D6F80330032202FB0343204659F876
:10C2B80023A0E7B2FFF750FEB3781D4A00257901A5
:10C2C800D554C9B22846524608F80350FEF7DBF8A1
:10C2D800284639462A46FEF794F90134032CDBD167
:10C2E80022E0030620D4D4F80330032202FB030221
:10C2F800104B002553F82260FFF72EFEA1780E4B55
:10C3080028465D540A4B32465D544901C9B2FEF7CE
:10C31800BAF8A17828462A46FEF773F904E0032202
:10C3280000E00422054B1A70BDE8FF87C8530020BF
:10C33800A04C0020D45300201F4C0020E4540020BF
:10C3480013B5B04C63782246A52B00F05E8259D80D
:10C35800852B00F0E18027D8072B00F017810FD834
:10C36800032B00F0D98005D8012B00F0AC8000F237
:10C37800B680A4E0052B00F0EE8000F2F780D3E051
:10C38800812B00F0A08009D80D2B00F02481802B90
:10C3980000F095800C2B40F0288307E1832B00F0F8
:10C3A800C38000F29C803BE1952B00F0768115D884
:10C3B8008C2B00F0608108D8872B00F03D81C0F0FD
:10C3C800CA808A2B40F011833EE1932B00F0038151
:10C3D80000F2EC808D2B40F0088358E1A12B00F08F
:10C3E800F08109D89A2B00F08381A02B00F0E1811D
:10C3F800992B40F0FA8268E1A32B00F0F08100F25B
:10C40800F581E5E1B62B00F0A48226D8AD2B00F02B
:10C418004B820FD8A92B00F0248205D8A72B00F057
:10C42800128200F21782FFE1AB2B00F0288200F2A3
:10C438002D821DE2B12B00F05D8205D8AF2B00F0F4
:10C44800418200F2468236E2B32B00F06282C0F0ED
:10C458005882B52B40F0C98272E2C82B00F0768171
:10C4680015D8C12B00F05B8108D8B82B00F090825A
:10C47800C0F08582C02B40F0B88287E0C32B00F063
:10C488005D81C0F05381C72B40F0AF826EE0D22BA4
:10C4980000F09B8209D8CC2B00F06981D12B00F0E9
:10C4A8008D82C92B40F0A18279E2D52B00F07081F2
:10C4B800D62B00F07581D42B40F097825FE1514B69
:10C4C8009978490104E04F4B9978490141F00201FC
:10C4D800C9B2D3F803200020FDF7D5FF88E2494C04
:10C4E8000020A178D4F80320490141F00801C9B21D
:10C4F800FDF7B9FFA178D4F80320490141F00601FE
:10C50800002AB8BF5242C9B20020FDF7ACFF3E4A2C
:10C51800A378D31801221BE09178D2F803204901AF
:10C5280041F00A01C9B283E0364C0020A178D4F862
:10C538000320490141F00601C9B2FDF794FFA37831
:10C54800D4F80310314A42F823102F4AD318002296
:10C5580083F824204CE22B4CD4F80310A078FEF783
:10C5680092F8A378D4F80310294AECE7254B294A16
:10C57800987801211154D978274B03EB401359724D
:10C58800264B1B5C022B40F03382F5E11D4B214A00
:10C59800987801211154D9781F4B03EB40139972F5
:10C5A8001E4B1B5C002B40F02382E5E1154C01AAD1
:10C5B800A1780020490141F01401C9B2FDF7F5FF47
:10C5C800D4F803209DF8053012B143F0020316E0B9
:10C5D80023F0020313E00B4C01AAA17800204901C3
:10C5E80041F01401C9B2FDF7E0FFD4F803209DF82B
:10C5F800053012B143F0010301E023F001038DF887
:10C6080005302EE0C85300201C470020FC580020AD
:10C61800F0540020584D0020A84C00205D4D00200B
:10C62800AF4B9978490141F00401D3F80320C9B20E
:10C638000020FDF718FFDBE1A178D4F803204901B9
:10C6480041F00E01C9B2F3E7A54C0020A17801AA78
:10C65800490141F01401C9B2FDF7A7FFE3788DF84D
:10C668000630A178490141F01401C9B2002001AA9D
:10C67800FDF7D8FEBCE1A0789A4BE17803EB4013B4
:10C68800D972C1F10801C9B2FEF79AFCB0E1944B26
:10C698009978490141F01A01C7E7A17801AA49012F
:10C6A80041F01401C9B20020FDF77FFFD4F8032040
:10C6B8009DF8053012B143F0040301E023F00403B0
:10C6C8008DF80530864B9978CCE7854C01AAA1787E
:10C6D8000020490141F01801C9B2FDF766FFE27870
:10C6E8009DF8053002F00F0223F00F0313430FE00B
:10C6F800A17801AA490141F01801C9B20020FDF74B
:10C7080054FF9DF80530E27803F00F0343EA021363
:10C71800A1788DF80530490141F01801A5E7A27804
:10C72800704B03EB4213E2781A7261E16C4B9A7812
:10C73800D3F803106B4B5201995059E1A278694B19
:10C7480003EB4213D4F803205A6051E1A078664BFA
:10C7580001221A54634BD4F8032003EB4013DA7711
:10C76800624B1B5C032B40F04381E17804E1A27823
:10C778005C4B03EB4213D4F80320DA8138E1584BC1
:10C78800584A9978D3F8033002EB411253612FE1EC
:10C79800A278544B03EB4213D4F803209A7727E18D
:10C7A8004F4B504A9978D3F8033002EB41129383E8
:10C7B8001EE14B4BD3F803109878C9B2FEF70CFC76
:10C7C80016E1D4F80310A078C9B2FEF70FFC0FE108
:10C7D800D4F80310A078C9B2FEF728FC08E1D4F811
:10C7E8000310A078C9B2FEF72BFC01E1A078FEF790
:10C7F8008BFCD4F803100346C9B2A07813B9FEF72E
:10C8080033FCF5E0FEF758FCF2E0A078FEF77CFC7C
:10C81800D4F803100346C9B2A07813B9FEF72EFC6A
:10C82800E6E0FEF75DFCE3E0A078FEF76DFCD4F8E7
:10C8380003100346C9B2A07813B9FEF729FCD7E064
:10C84800FEF744FCD4E0D4F80310A078C9B2FEF790
:10C8580029FCCDE0D4F80310A078C9B2FEF7AEFCED
:10C86800C6E0D4F80310A078C9B2FEF7B1FCBFE067
:10C87800D4F80310A078C9B2FEF7B4FCB8E0D4F835
:10C888000310A078C9B2FEF7B7FCB1E0D4F80310E2
:10C89800A078C9B2FEF7BAFCA278154B03EBC20325
:10C8A800D4F803205A71A3E0D4F80310A078C9B2D1
:10C8B800FEF7E8FC9CE0D4F80310A07849B2FEF734
:10C8C800EBFC95E0D4F80310A078C9B2FEF716FD8A
:10C8D8008EE0D4F80310A078C9B2FEF717FD87E000
:10C8E800C8530020A84C0020584D00205D4D002062
:10C8F800044C0020D4F80310A078C9B2FEF70EFD4E
:10C9080076E03C4BD3F803109878C9B2FEF70EFDD9
:10C918006EE0A078384A4301D118497AA72903D88C
:10C92800D3189B7AA72B05D9D4F80310012904D072
:10C9380004225BE0D4F80310C9B2FEF707FD57E004
:10C948002C4B2D4A9978D3F8033002EB41129361AE
:10C958004EE0A078D4F80320284B43F8302022B9C1
:10C9680003EBC0035979FEF751FC224B244A98780F
:10C97800125C012A3CD1D978FBF74EFD38E01D4BFB
:10C988001E4A9978D3F8033002EBC10213712FE0E5
:10C99800D4F80310A078C9B2FEF75CFB28E0154B69
:10C9A8009878D978144B03EB40131A6922F07F4228
:10C9B80042EA01621A61FBF7DFFE19E00D4B987835
:10C9C800D3F80310FBF79AFE12E0A0780A4BD4F8CC
:10C9D800031003EB40131A6921F07F4102F07F42F4
:10C9E8000A431A61FBF7C0FE02E00322054B1A70E6
:10C9F8001CBD00BFC8530020A84C0020044C0020D8
:10CA08005D4D0020E45400202DE9FF47DFF8009336
:10CA1800BC4C99F80030642263702270D9F8030086
:10CA2800222B606001F0CB8357D80F2B01F00F81C8
:10CA380026D8072B00F0428410D8032B00F0318150
:10CA480006D8012B00F0A980022B41F00586E6E00C
:10CA5800052B00F06D8100F2788165E10B2B01F068
:10CA68003E8006D8092B00F0E38600F2E58600F048
:10CA780072BD0D2B01F06B8001F2A58001F04AB860
:10CA8800192B01F0E88113D8152B01F0438107D841
:10CA9800132B01F0E080142B41F0DE8501F017B96B
:10CAA800172B994B01F0BD8101F2C88101F0B6B98D
:10CAB8001E2B01F0098209D81B2B01F0F181C1F06E
:10CAC800DC811C2B41F0C88501F0EDB9202B01F069
:10CAD800AE8201F20F8301F050BA812B01F0188465
:10CAE8002ED8412B01F0FA8315D8252B01F0AA8303
:10CAF80007D8232B01F07183242B41F0AD8501F079
:10CB080073BB272B01F0CE83C1F0A883402B41F0E3
:10CB1800A38501F0E0BB452B01F0EC8306D8432B3D
:10CB280001F0E28301F2E38301F0DBBB472B01F064
:10CB3800E783C1F0E283802B41F08E8501F0E3BBEF
:10CB4800882B01F08D8412D8842B01F01F8407D81C
:10CB5800822B01F0F683832B41F07E8501F0F6BB32
:10CB6800862B01F02C8401F2998401F023BC8C2BD4
:10CB780001F0F38406D88A2B01F0D48401F2E8840A
:10CB880001F0B8BCF22B01F05B85FF2B01F05B854F
:10CB98008D2B41F0618501F008BD99F80230022B18
:10CBA80038D85A4E5A4FDFF87091DFF870A1002438
:10CBB800BB789C4207D0554A02EB43139B7F1BB3BB
:10CBC800B27F9A4220D1012304F809305FFA84F831
:10CBD800504B002541464FEA4818E55428460222A2
:10CBE8005FFA88F804F80A50FDF70BFD48F00601D3
:10CBF800284640F2FF72FDF736FC48F00801D7F8E6
:10CC080003202846FDF72FFC01342036032CCFD112
:10CC180001F025BD3B4B04221A7001F020BD3C4FAA
:10CC2800BB78022B38D8394EDFF8EC90DFF8ECA04F
:10CC38000024BB789C4207D0344A02EB43139B7F05
:10CC480023B3B27F9A4221D1012304F809305FFA55
:10CC580084F8304B002541464FEA4818E5542846E9
:10CC680002225FFA88F804F80A50FDF7CAFC48F077
:10CC78000601284640F2FF72FDF7F5FBD7F80320BE
:10CC880048F0080152422846FDF7EDFB01342036F2
:10CC9800032CCED101F0E3BC1A4B04221A7001F028
:10CCA800DEBC99F80230022B3AD8184EDFF86C80B7
:10CCB800DFF860A0002499F802309C4207D0134A9C
:10CCC80002EB43139B7FBBB1B27F9A4214D100257C
:10CCD800E7B2384604F8085004F80A5002F066FD36
:10CCE800284639460222FDF78CFC790141F00801FB
:10CCF800C9B22846FDF73CFC01342036032CDAD1B2
:10CD080001F0ADBCE45400201C470020A84C0020D2
:10CD1800C85300201F4C002040470020A04C002092
:10CD28000423237001F09BBCFFF738F901F097BC8E
:10CD380099F80230022B03D8FFF702FB01F08FBCF1
:10CD4800B04B04221A7001F08ABCAF4DAD4CA878E4
:10CD5800022800F29A826B78A42B00F01B827CD800
:10CD6800842B00F00A8136D8082B00F0228115D8D0
:10CD7800032B00F0068105D8012B00F0F48000F2A7
:10CD8800FC80EDE0052B00F00681C0F00281062B47
:10CD980000F00581072B40F0748205E10D2B00F0AF
:10CDA800208109D80A2B00F04981C0F025810B2B7E
:10CDB80000F032810C2B2BE0812B00F0D48003D8BB
:10CDC800802B40F05E82CBE0822B00F04681832BE3
:10CDD80040F05782DDE0952B00F05F811BD88A2B4D
:10CDE80000F0438108D8862B00F0D580C0F0C980B8
:10CDF800872B40F0468234E18D2B00F0468103D822
:10CE08008C2B40F03E823BE1932B00F0EA80942B80
:10CE180040F03782D8E09D2B00F0CB800ED89A2BBB
:10CE280000F0558103D8992B40F02B8242E19B2BCF
:10CE380000F0F2809C2B40F02482FFE0A12B00F050
:10CE4800A08103D8A02B40F01C8297E1A22B00F010
:10CE58009B81A32B40F0158299E1B72B00F0F68156
:10CE680037D8AD2B00F0CF8116D8A82B00F0BA81A7
:10CE780005D8A62B00F0A68100F2B18195E1AA2B76
:10CE880000F0B681C0F0B181AB2B5E4C00F0B381ED
:10CE9800AC2B40F0F681B1E1B22B00F0C3810CD885
:10CEA800AF2B00F0B681C0F0B181B02B554C00F02B
:10CEB800B381B12B40F0E581B1E1B42B00F0B98129
:10CEC800C0F0B381B52B00F0B881B62B40F0D98102
:10CED800B8E1CC2B00F01D8120D8C32B00F00D81C8
:10CEE8000ED8C02B60D0474D03D8B82B40F0C9816D
:10CEF800B1E1C12B00F0F780C22B40F0C281F7E00E
:10CF0800C72B4CD003D8C42B40F0BB81FAE0C82B08
:10CF180000F0FA80C92B40F0B481A0E1D22B00F0D8
:10CF2800A8810ED8CF2B00F0FD8003D8CE2B40F07F
:10CF3800A881F3E0D02B00F00A81D12B40F0A18129
:10CF480094E1D52B00F00B8103D8D42B40F09981C4
:10CF580000E1D62B00F00881FE2B40F0928108E119
:10CF68004001C1B203E0410141F00201C9B2002011
:10CF7800FDF70AFD234B586089E1410141F00801A2
:10CF880002E0410141F00A01C9B20020FDF723FB8C
:10CF9800F0E71E4B00E01E4B53F8202063E11D4BC9
:10CFA80003EB4010427A5EE11A4B03EB4010827AA1
:10CFB80059E10020FDF7F4FA134B9B785B0040FA27
:10CFC80003F000F00100D5E7410141F0140101AA86
:10CFD800C9B20020FDF7E9FA9DF80520C2F3400226
:10CFE80041E1410141F0140101AAC9B20020FDF755
:10CFF800DCFA9DF805202DE00130C0B2FBF76DFA90
:10D00800B8E700BFE4540020C8530020FC580020B3
:10D01800F0540020A84C002000207C2101AAFDF734
:10D02800C4FAAA4B9A780223520003FA02F29DF836
:10D0380006301A420CBF0022012214E101AA002086
:10D048007C21FDF7B2FAA14A9DF806309278520089
:10D0580043FA02F202F0010205E1410141F0040144
:10D0680092E7410141F00E018EE7410141F01401C0
:10D07800C9B2002001AAFDF798FA9DF80630FEE033
:10D08800FDF7BCFFC0F10800D1E0410141F01A01F1
:10D09800C9B20020FDF79FFAC9E0410141F014012F
:10D0A800C9B2002001AAFDF780FA9DF80530C3F344
:10D0B8008003E4E0410141F0180101AAC9B200204F
:10D0C800FDF773FA9DF8052002F00F02CBE041014D
:10D0D80041F0180101AAC9B20020FDF766FA9DF8CF
:10D0E80005201209BFE07A4B03EB4010037AC6E033
:10D0F800774B40011B586B60C9E0754B03EB401040
:10D108004368BCE0734B0AE0714B03EB4010C37FEC
:10D11800B5E06F4B03EB4010C389B0E06E4B53F89A
:10D128002030ACE06D4B0022195C626011B16C4993
:10D1380001244C601A546B4B195C1A4621B1684B98
:10D14800596841F002015960002313549FE0664B6F
:10D158001B5C94E05E4B03EB401043698FE05C4B33
:10D1680003EB4010837F8AE0594B03EB4010838B1D
:10D1780085E0574B03EB4010027B74E0FDF746FF58
:10D1880055E0FDF74BFF52E0FDF7B4FF4FE0FDF728
:10D19800BBFFEFE6FDF7B8FF0346A87813B9FDF724
:10D1A800C7FF44E0FDF7ECFF41E0FDF7ADFF4C4C55
:10D1B800464B18B99878FDF7C5FF38E09878FDF721
:10D1C800F3FF34E0FDF7A0FF454C404B18B99878C1
:10D1D800FDF7C2FF2BE09878FDF7DCFF27E0FDF7AD
:10D1E800C5FF24E0FEF71CF821E0FEF723F81EE057
:10D1F800FEF72AF81BE0FEF731F818E03B4B03EB8B
:10D20800C00043793BE0FEF75BF810E0FEF762F8F8
:10D218000DE0FEF7BBF80AE0FEF7C0F807E0FEF7FE
:10D22800C5F804E0FEF7CAF801E0FEF7D7F8606039
:10D238002DE02F4B1B5C636029E0254B03EB40106E
:10D2480083691CE0294B53F830200CE0274B03EB93
:10D25800C000037913E0FDF761FF686017E01C4B1D
:10D2680003EB4010C27C1E4B5A6010E0FBF728FA13
:10D2780080E6174B03EB4010036923F07F4363609C
:10D2880005E0174B03221A7001E004232370194BA1
:10D298001B78002B01F0E381114B5A68164B1A607A
:10D2A800164B2AB91A6842F008021A6001F0D7B979
:10D2B8001A6822F008021A6001F0D1B999F8020040
:10D2C80002281DD90423237001F0C9B9C8530020CE
:10D2D800A84C0020E44B0020244C0020A04C002047
:10D2E800E45400201F4C0020A34C0020044C0020D4
:10D2F800004C0020DF540020D0540020D0530020E0
:10D3080099F801309A2B21D8992B80F08B80822BA9
:10D3180070D00BD8062B4CD003D8042B3FD0052B4C
:10D328000AE0072B53D00C3B012B0CE08C2B66D06A
:10D3380005D8832B33D0862B40F0088134E08D2B21
:10D348006BD0933B022B00F201814EE0C82B00F01A
:10D358009B8010D8C12B78D005D8B52B67D0C02BAF
:10D3680040F0F48033E0C32B00F0838077D3C72BE1
:10D3780040F0EC801DE0D42B00F0B08006D8CC2B18
:10D3880000F09080D22B40F0E18099E0D62B00F09D
:10D39800C180C0F0B180FE2B40F0D880C8E00621E3
:10D3A800FDF721FA01F05BB90C21FDF71CFA01F039
:10D3B80056B9D34B420199180931D318CA1A023009
:10D3C80002EB4010597AFCF7CBFD01F048B9CC4B81
:10D3D800420199180A31D318CA1A023002EB4010D8
:10D3E800997AFCF7BDFD01F03AB91421FDF7FBF974
:10D3F80001F035B90421FDF7F6F901F030B9C04B59
:10D40800420199180B31D318CB1A023003EB4010A4
:10D418000122FCF702FE01F022B91A21FDF7E3F917
:10D4280001F01DB91821FDF7DEF901F018B9430123
:10D4380003F11802B249D31A0230511803EB401015
:10D448000422FCF7EAFD01F00AB9AD4B03EB4013E7
:10D4580040014830197AFCF783FD01F000B9A8496A
:10D46800042201EB401102304001FCF7D6FD01F027
:10D47800F6B8A349042201EB4011400104314430BD
:10D48800FCF7CBFD01F0EBB89D4B420199181F3119
:10D49800D318CB1A023003EB40100122FCF7BDFD74
:10D4A80001F0DDB8964B420199180E31D318CB1A0A
:10D4B800023003EB40100222FCF7AFFD01F0CFB8B9
:10D4C800430103F110028E49D31A0230511803EBBD
:10D4D80040100422FCF7A1FD01F0C1B8884B4201BD
:10D4E80099181431D318CB1A023003EB40100422D8
:10D4F800FCF793FD01F0B3B8814B420199181E3136
:10D50800D318CB1A023003EB40100122FCF785FD3B
:10D5180001F0A5B87A4B420199181C31D318CB1ADF
:10D52800023003EB40100222FCF777FD01F097B8B8
:10D53800734B420199180C31D318CB1A023003EB04
:10D5480040100122FCF769FD01F089B86D4B0322F8
:10D558001A7001F084B899F802006B4D022804D9BA
:10D56800684B04221A7001F07AB86B789A2B24D889
:10D57800992B80F0BF80822B00F09B800BD8062B64
:10D5880076D003D8042B41D0052B0BE0072B7DD098
:10D598000C3B012B0EE08C2B00F0908005D8832BE0
:10D5A80034D0862B40F03F8147E08D2B00F09D80E2
:10D5B800933B022B00F2378176E0C72B58D011D865
:10D5C800C12B00F0B78006D8B52B00F0A580C02B82
:10D5D80040F029815AE0C22B00F0B680C32B40F0FE
:10D5E8002281BBE0D42B00F0E08006D8C82B00F0E5
:10D5F800C080CC2B40F01781C9E0D62B00F0F18019
:10D60800C0F0E180FE2B40F00E81F8E03E4C062190
:10D61800FDF7C6F8A5780020690141F00601C9B2F6
:10D62800FCF7D9FF394B3A4A43F82500A378D318B9
:10D63800002283F8242001F012B8334C0C21FDF7A6
:10D64800AFF8A5780020690141F00C01C9B2FCF7D8
:10D65800C2FF304B2E4A43F82500A078002112184B
:10D6680082F8241053F82010FDF70DF800F0F7BFEA
:10D67800234B44011A190932E418131B023003EB37
:10D688004010FCF755FD607200F0E9BF1C4B4401E7
:10D698001A190A32E418131B023003EB4010FCF786
:10D6A80047FDA07200F0DBBF1421FDF779F800F008
:10D6B800D6BF0421FDF774F800F0D1BF104C430128
:10D6C800E1180B311B19CB1A023003EB4010012271
:10D6D800FCF734FDA87804EB4014E17AC1F10801A5
:10D6E800C9B2FDF76DFC00F0BABF1A21FDF758F872
:10D6F80000F0B5BF1821FDF753F800F0B0BF00BF28
:10D70800A84C0020E4540020C8530020FC580020F6
:10D718001C470020F0540020430103F11802A649D9
:10D72800D31A0230511803EB40100422FCF706FD0F
:10D7380000F095BFA04C04EB401440014830FCF7C2
:10D74800F7FC207200F08BBF9B49042201EB4011CB
:10D7580002304001FCF7F2FC00F081BF9649042238
:10D7680001EB4011400104314430FCF7E7FC00F0C4
:10D7780076BF914B420199181F31D318CB1A02304A
:10D7880003EB40100122FCF7D9FC00F068BF8A4B7C
:10D79800420199180E31D318CB1A023003EB40100E
:10D7A8000222FCF7CBFC00F05ABF834B42019918C8
:10D7B8001431D318CB1A023003EB40100422FCF7C3
:10D7C800BDFC00F04CBF7C4B420199181E31D318A8
:10D7D800CB1A023003EB40100122FCF7AFFC00F03B
:10D7E8003EBF754B420199181C31D318CB1A023031
:10D7F80003EB40100222FCF7A1FC00F030BF6E4C96
:10D808004301E1180C311B19CB1A023003EB40100D
:10D818000122FCF793FCAB7804EB4314207BFBF765
:10D82800B5FB00F01CBF654B03221A7000F017BF50
:10D83800FEF70EF800F013BF99F80220604B022A99
:10D848005E4C00F0D380032A00F0D580002A40F017
:10D858002D815B78502B74D023D8462B56D0224686
:10D868000DD8422B48D005D8402B3CD0412B40F056
:10D87800B9803FE0442B534944D045D83FE04B2B77
:10D8880053D0214606D8482B45D041D3492B40F0E8
:10D89800A98044E04D2B4ED04AD34F2B40F0A280B4
:10D8A8004CE0812B64D022460FD8542B52D004D898
:10D8B800522B44494AD04BD846E0572B52D0802BA4
:10D8C80052D0552B40F08E8047E0852B214661D001
:10D8D80003D8832B58D05AD853E0FE2B69D07BD875
:10D8E800F02B7FD161E040F2FF70FCF721FC334B55
:10D8F8005860DDE0334B5DE0324B5B78D2E00B796A
:10D908005360D5E0CB69FBE74B79F9E72D4B99E0FC
:10D918002C4B9B68F4E72B4B93F82630F0E7294B08
:10D92800DB7D003318BF012341E0264BDB78B9E0EB
:10D93800244B9B78E4E7234B5B7DE1E7214B5B7E3F
:10D9480035E0204B9B7DADE00B7DD9E70B6AD7E72F
:10D958000B69D5E71B4B9B7EA4E01A4BDA7E174B6D
:10D968005A60A5E0174B00E0174B93F82730C7E73C
:10D97800154B93F82730A3F10402534243EB0203FB
:10D9880090E0114B1B6ABBE70F4B1B68B8E70F4BC6
:10D998001B680CE00C4A0E4953684B4303F540538F
:10D9A8003933536023F000437CE00A4B1B784B600B
:10D9B8007EE0084B1B78A3E7A84C0020E454002025
:10D9C800C8530020040000201C470020E054002019
:10D9D8006D4EC641504D00208F4B1B78003318BF49
:10D9E80001238DE78D4B03221A7061E05A788C4B26
:10D9F80053F8223056E05B782E2B55D8DFE803F039
:10DA0800181B1E5454545454542124275454545409
:10DA180054545454545454545454542A2C2E30327C
:10DA2800365454545454543B3E4144474A4D500094
:10DA38007C4B1B6836E07B4B5B6833E0794B9B681B
:10DA480030E0784BDB682DE0764B1B692AE0754B9C
:10DA58005B6927E0002006E0002008E0012002E0E2
:10DA6800012004E00220FCF747FF02E00220FCF757
:10DA780055FF60601CE06B4B9B6913E0694BDB69E9
:10DA880010E0684B1B6A0DE0664B5B6A0AE0654B69
:10DA98009B6A07E0634BDB6A04E0624B1B6B01E0A7
:10DAA800604B5B6B636003E0032300E00423237097
:10DAB8005D4B1B78002B00F0D285584B5A685B4BA6
:10DAC8001A605B4B2AB91A6842F008021A6000F023
:10DAD800C6BD1A6822F008021A6000F0C0BD99F8A5
:10DAE8000230022B12D199F80130372B0AD84C4951
:10DAF80003F5A770800001EB83010422FCF78DFA7F
:10DB080000F0ADBD0323237000F0A9BD04232370EA
:10DB180000F0A5BD99F80230022B13D1454B5B7874
:10DB2800372B0AD83E4903F5A770800001EB830123
:10DB38000422FCF703FB00F092BD384B03221A7055
:10DB480000F08DBD354B04221A7000F088BD99F89D
:10DB58000200022832D8374C6378012B21D003D336
:10DB6800022B2E4C26D120E001F018FEA178324A73
:10DB78000023DFF8CCC0314E01271D4602EB4114CB
:10DB8800994205D0907F30B194F81E80804502D12B
:10DB980003F80C709D5501332032032BF0D100F0AF
:10DBA8005EBD01F003FE00F05ABD01F007FE6060A3
:10DBB80000F055BD0323237000F051BD174B04221C
:10DBC8001A7000F04CBD99F8023013B1022B39D10C
:10DBD80003E0FAF721FD00F042BD164B5B78072BF6
:10DBE8000AD820B91846FAF71AFC00F038BD1846CA
:10DBF800FAF73CFC00F033BDFF2B08D1431C0ABFE9
:10DC08000A4BC0B21878FAF757FC00F028BD034B4E
:10DC180003221A7000F023BDDE540020E4540020D3
:10DC2800FC540020144D0020DF540020D054002064
:10DC3800D0530020C8530020A84C00201F4C0020BF
:10DC4800404700209A4B04221A7000F008BDFEF7E6
:10DC580097F800F004BD99F80120964B092A27D8B7
:10DC6800DFE802F005080B0E12181B1E21251A68A2
:10DC780010181CE01A68101A19E01A68504316E0C8
:10DC88001A6892FBF0F012E01A6892FBF0F100FBC0
:10DC980011200CE01A68104009E01A68104306E0E9
:10DCA8001A68504003E01A68D2431A6000E018600E
:10DCB8001A68814B2AB91A6842F008021A6000F003
:10DCC800CEBC1A6822F008021A6000F0C8BC794B72
:10DCD8001A68794B8242196804DD41F0040121F089
:10DCE800030108E00BBF21F0060121F0070141F014
:10DCF800010141F0020119606F4B2AB91A6842F01C
:10DD080008021A6000F0ABBC1A6822F008021A6018
:10DD180000F0A5BC99F801300C2B00F2A084DFE8D4
:10DD280003F0071019222B343E475059626B7400D8
:10DD3800614B1B68190740F19284604B186200F030
:10DD48008EBC5D4B1B681A0700F189845B4B186217
:10DD580000F085BC584B1B68DB0740F18084574BAB
:10DD6800186200F07CBC544B1B68D90700F177841B
:10DD7800524B186200F073BC4F4B1B685A0740F1B6
:10DD88006E844E4B186200F06ABC4B4B1B6813F054
:10DD9800050F00F06484494B186200F060BC464BE4
:10DDA8001B689B0740F15B84444B186200F057BC2A
:10DDB800414B1B68990700F05284404B186200F0F1
:10DDC8004EBC3D4B1B68DA0640F149843B4B186258
:10DDD80000F045BC384B1B689B0640F14084374B2C
:10DDE800186200F03CBC344B1B68590640F137847C
:10DDF800324B186200F033BC2F4B1B681A0640F1F7
:10DE08002E842E4B186200F02ABC2B4B1B68DB05B6
:10DE180040F12584294B186200F021BC186200F0FB
:10DE28001EBC9A6A072A00F21A841C6A03EB820154
:10DE38000132CC629A62186200F011BC9B6A1F4AD8
:10DE4800002B00F00C84013B936202EB8303DB6A36
:10DE5800136200F004BC99F801302E2B03D8184A3D
:10DE68000121D154FBE3FF2B04D1144B012283F889
:10DE78004C20F4E303232370F1E3124B5B782E2B41
:10DE880003D80F4A0021D154E9E3FF2B04D10B4BEF
:10DE9800002283F84C20E2E3054B03221A70DEE3EC
:10DEA800FDF7DCFEDBE3054B002283F82720D6E3F1
:10DEB800E4540020D0540020D05300201C470020F8
:10DEC800744D0020C853002099F80130142B51D804
:10DED80099F80220022A19D8032101FB0325A64C30
:10DEE80044F82500A548807E002800F0B883002B60
:10DEF80000F0B583581E01FB002000F5C3708000B8
:10DF080004EB85010422FCF788F8A8E3FF2A2DD149
:10DF18008BB100249A4F0325974E15E008EB0500B6
:10DF2800791904220435FCF778F80C2DF6D10C3455
:10DF3800FC2C02D193E3904E0C2404F5C068002514
:10DF480008F10C08A719E9E779780422481E05FBAF
:10DF5800004005FB014100F5C370800006EB81011C
:10DF68000134FCF75AF8032CEED178E3854B0422F0
:10DF78001A7074E30323237071E399F80130804F1A
:10DF8800142B50D8BA78022A1AD8032101FB03238C
:10DF9800794951F823207B4B5A607B4B1B78002B27
:10DFA80000F05D83794B1A60794B22B91A6842F008
:10DFB80008021A6053E31A6822F008021A604EE356
:10DFC800FF2A2CD183B1002403256B4E15E008EB02
:10DFD8000500791904220435FCF7B0F80C2DF6D1A8
:10DFE8000C34FC2C02D13AE3634E0C2404F5C068CF
:10DFF800002508F10C08A719E9E779780422481EDA
:10E0080005FB004005FB014100F5C370800006EBED
:10E0180081010134FCF792F8032CEED11FE3594B30
:10E0280004221A701BE3574B03221A7017E399F85E
:10E038000160142E5AD8524DAC7821062BD54E4E7D
:10E048004E4F0024AB7843FA04F3DA070DD561018B
:10E0580041F00201C9B2002095F80180FCF794FC58
:10E06800032303FB084846F82800BB7E7BB16B7886
:10E078006BB10321581E01FB004001FB034100F571
:10E08800C370800006EB81010422FBF7C6FF013450
:10E09800032CD7D1E3E2022C24D8610141F002011C
:10E0A800C9B20020FCF770FC032202FB0644334B84
:10E0B80031499B7E41F82400002B00F0D0826B7818
:10E0C800002B00F0CC82AC78581E02FB004002FB0B
:10E0D800034300F5C370800001EB83010422FBF7C2
:10E0E8009CFFBCE2274B04221A70B8E2254B03229E
:10E0F8001A70B4E299F80120244B0A2A51D8DFE8B3
:10E1080002F0060B11161C24292E33374B00214A26
:10E11800196812688A1803E01E4A196812688A1A70
:10E128001A603EE01B491A6809684A43F8E7194A29
:10E138001968126891FBF2F2F2E7164A1968126838
:10E1480091FBF2F002FB1012EAE7124A11681A6812
:10E158000A40E5E70F4A11681A680A43E0E70D4AE2
:10E1680011681A684A40DBE70A4B1A68D243D7E7B6
:10E178001A68084BD4E700BFD453002004000020DD
:10E18800C8530020E4540020DF540020D05400205D
:10E19800D0530020EC540020A64A1968106811607A
:10E1A8001860A54B1A68A54B22B91A6842F00802F4
:10E1B8001A6054E21A6822F008021A604FE29E4B75
:10E1C8001B68C9F8033099F80230022B02D8FEF711
:10E1D800B7F844E20423237041E2974B1B68C9F85F
:10E1E8000330FDF735FB3AE2954B5B78052B00F2DF
:10E1F8003682DFE803F003090F151B218F4B1A68DD
:10E2080002F00F021A602AE28C4B1A6822F0100200
:10E218001A6024E2894B1A6822F020021A601EE272
:10E22800864B1A6822F040021A6018E2834B1A687B
:10E2380022F080021A6012E2804B1A6822F480727F
:10E248001A600CE299F801302E2B04D87D4A02EBB3
:10E258008303186503E20323237000E2794B764AAF
:10E26800D3F80C111160D3F81011724A1160D3F869
:10E278001421D3F818111A62704A1160D3F81C21BE
:10E2880071491A75D3F82021DA61D3F824219A61EB
:10E2980093F82821885C08B101208854002283F86B
:10E2A8002C21DCE199F80220022A10D8644B597815
:10E2B8004FF00303142907D803FB01235E4A634880
:10E2C800126840F82320CAE1614A1370C7E1604B25
:10E2D80004221A70C3E100F059FFC0E100F05EFFAC
:10E2E800BDE100F05CFFBAE100F05AFFB7E100F0D1
:10E2F80058FFB4E100F056FFB1E100F054FFAEE181
:10E3080000F052FFABE14F4B002283F82720A6E133
:10E3180099F8013013B1012B10D104E0494B0122C7
:10E3280083F827209BE1B0F5006F04D2454A82F8B4
:10E338002730106293E10423237090E103232370B4
:10E348008DE1404B022283F8272088E13D4B0022D3
:10E358003D4C83F84C2083F82C2103F14C014FF0FD
:10E36800FF351046A054013200232F2A41F8045FDC
:10E37800F8D1344A82F827301362936213752E4A13
:10E3880013602C4A13602D4A136068E1314B1B7DE2
:10E398009B070CD4B0F5006F38BF2A4A4FF004032E
:10E3A8003ABF82F82730C2F83001237057E10823BA
:10E3B800237054E1234B002283F827204FE1264B9A
:10E3C80001221A70234A254B9178B0F5006F197015
:10E3D80003D2147D14F0010409D000225A709A70F7
:10E3E800DA701A715A719A71DA71197237E101A9E2
:10E3F800FBF7F2FC194B9DF804201C725A709DF82B
:10E4080005209A709DF80620DA709DF80A201A7186
:10E418009DF809205A719DF808209A719DF80720E7
:10E42800DA710122D05C197A01324118082A19726E
:10E43800F8D114E1EC540020D0540020D05300202F
:10E44800C85300201C470020744D0020D4530020DE
:10E45800E454002004000020D4540020D5540020A7
:10E4680099F801307BB97F4A012111707E497F4AB2
:10E47800897811707E490968013311F8010B082B5E
:10E488009854F9D1EBE0012B40F0E9800C22E271BD
:10E49800637126220723A2712371E0E0754B5B7834
:10E4A800032B00F2DC80DFE803F0020F1B20724A26
:10E4B800724B92F82710D971117DD2F830219971D9
:10E4C800110A59711A71CAE06B4A6C4B92F82710FD
:10E4D800D971117D126A9971110A59711A71BEE0C8
:10E4E800674B1A68654B5A60B9E0664B1A68634B0C
:10E4F8005A60B4E05F4B5A78002A40F0B0809978AF
:10E50800002940F0AC8040F2D243984240F0A78006
:10E5180040F2FF70FBF724FDFBF77AFC0120FAF7C5
:10E528004FFC9CE099F80120574B003218BF01229C
:10E538001A7099F80320554B1A704F4B93F83421F1
:10E54800534B1A70534A00231370534A137086E0D2
:10E55800494B012283F8352181E099F8015015B122
:10E56800012D1FD10FE0042240F2FB7003A9FBF735
:10E57800E5FDD9F80320039B9A4202D10123636089
:10E588006DE065606BE099F802302A2B06D140F205
:10E59800FB7042490422FBF740FD60E0374B032241
:10E5A8001A705CE00323237059E0324B5B78032B2D
:10E5B80042D8DFE803F00902313D2F4A0023D2F8A0
:10E5C800381102F59C7224E02B4BD3F83821092A24
:10E5D80007D803EB82010132C1F83C01C3F83821A6
:10E5E8003DE0264B09221A7039E052F8044F844264
:10E5F8000ED12B4A013902EB830203E05068013344
:10E6080042F8040B8B42F9D31B4BC3F8381126E0B0
:10E6180001338B42E9D122E0174A0023C2F838318E
:10E62800194602F59E7299500433282BFBD116E047
:10E63800124B0A225A6012E0104B03221A700EE0A5
:10E64800FDF7E8FB0BE040F2D243984207D10A4BB2
:10E65800012283F8642102E0084B02221A70BDE807
:10E66800FF8700BFD454002004000020D5540020A8
:10E6780000000020C85300201C470020E45400205C
:10E68800D0540020EC540020F04B0020234C0020F4
:10E698005C4D0020224C0020A34D0020CB530020CD
:10E6A80058480020474900232DE9F0410B604649AE
:10E6B800464A0B6046494748136293620B601375DC
:10E6C80082F84C3082F82C314FF0FF344C32194626
:10E6D800C15401332F2B42F8044FF9D10024DFF83D
:10E6E8000C813D4F25466E01F6B246F0060100202A
:10E6F800FCF74AF946F00C0144F808000020FCF742
:10E7080043F90135E0510434032DECD1334D002495
:10E71800E97AE0B2C1F10801C9B20134FCF750FC52
:10E728002035032CF4D100232D491A465A500433BE
:10E73800B3F5806FFAD12B4B9B7E6BB915E008EBD4
:10E748000500791904220435FBF7F8FC0C2DF6D1E5
:10E758000C34FC2C02D108E0234E0C2404F5C068CC
:10E76800002508F10C08A719E9E71E4BDC7E64B9FF
:10E778001B4E4FF4A76506EB84012846042201349A
:10E78800FBF7DCFC0435382CF5D1164A1379012B3C
:10E7980008D0112B05D0A3F121014B4243EB010313
:10E7A80000E00123094C84F86531537D13B1F9F772
:10E7B80055FF08B9002300E0012384F82730BDE89D
:10E7C800F08100BFD0540020EC5400201C470020EA
:10E7D800D0530020744D0020F0540020A84C002095
:10E7E800FC54002004000020D4530020FC580020D2
:10E7F800F7B50F4E05460C4696E803008DE8030072
:10E808000C496F46C1F803300B4B8A7000220D701B
:10E818004C701A70FEF7F8F831787368074A82F876
:10E8280066119DE8030086E803001846FEBD00BF98
:10E83800E4540020C8530020DF5400201C47002067
:10E84800014B93F8660170471C47002073B51F4DB4
:10E85800034602AA0C4695E8030002E9030059782A
:10E868001B4A0026117099785170D97891701979DE
:10E8780091715979517199791171DB79D370154B6F
:10E888001E70FEF7C1F8144B1A7872B922702B78F3
:10E898006270A3706B78E370EB792371AB79637165
:10E8A8006B79A3712B79E37109E0012A07D10B4A2F
:10E8B800334612F8011FE1540133082BF9D1034BF9
:10E8C80002AA12E9030083E803007CBDE454002097
:10E8D800C8530020DF540020D4540020D554002011
:10E8E8002DE9F04F9C4B99B01B789C4913B991F8CE
:10E8F80067316BB19A4B1B78062B09D00A2B07D0CE
:10E908000F2B05D01F2B03D0944B002283F8342102
:10E9180091F83431914A591EC9B201293DD8012BC9
:10E9280014BF082307238F498DF81C3092F86831EB
:10E938008D4AC86812788DF81D30002308908DF82C
:10E948001E30C2B98B688DF82B208DF82430874B88
:10E9580019788DF8251059788DF82610D9798DF801
:10E96800271099798DF8281059791B798DF8291075
:10E978008DF82A300AE0012A08D17D490DF12302D9
:10E988000133585C082B02F8010FF9D107A8FAF7F0
:10E99800FBFE002840F0AD80DBE3032B724922D157
:10E9A80092F86541002C7DD10B788BB96D4D6F4C79
:10E9B800A8786E7823788619F6186378F618E379BC
:10E9C800F618A379F6186379F6182379F61817E07C
:10E9D800012B40F08E80664D605D0134FAF70AFC29
:10E9E800092CF9D185E0042B26D15E4D5F4CA8781F
:10E9F8006E78002301228619637022706360B6184E
:10EA0800FAF7F8FB6878FAF7F5FB2078FAF7F2FBE3
:10EA18006078FAF7EFFBE079FAF7ECFBA079FAF700
:10EA2800E9FB6079FAF7E6FBF6B22079FAF7E2FB40
:10EA38003046FAF7DFFB5CE0072B37D192F86531F7
:10EA4800002B2FD10A781ABB464B9E785F78474B2C
:10EA58008DF848601D785C78BE19D8798DF84A50D1
:10EA6800AD1999798DF84B4064195A798DF84C0095
:10EA780000191B798DF84D1009188DF84E20521881
:10EA88008DF84F309B188DF849708DF850302CE078
:10EA9800012A2AD1364A985C12A958540133092B05
:10EAA800F9D122E0314801F011FC22E0082B20D1F5
:10EAB8002E4A00230120537010705360294A8DF8A4
:10EAC8004A00917852788DF848108DF849208A18B4
:10EAD80012188DF84B308DF84C308DF84D308DF87C
:10EAE8004E308DF84F308DF8502012A80921FCF7D0
:10EAF80057FE204B1B78002B00F08A801E4B1F4CC2
:10EB08001B78013B062B7ED8DFE803F004043A7D2E
:10EB18007D7D5D00134A1949936809788DF8343072
:10EB280080238DF835308A238DF8363000238DF810
:10EB380037308DF838308DF839308DF82D308DF824
:10EB48002E30D3688DF83A100BA807218DF82C10B9
:10EB58000C93FAF719FE56E0DE5400201C470020FB
:10EB6800C853002004000020D4540020E45400209E
:10EB7800D5540020A34D00205C4D0020224C0020DD
:10EB88009D4D2378A8786E7886190A36F618FAF714
:10EB980031FB6878FAF72EFB8020FAF72BFB8A20E6
:10EBA800FAF728FB0020FAF725FB0020FAF722FBEA
:10EBB8000020FAF71FFBF6B22078FAF71BFB304665
:10EBC800FAF718FB1FE08C4B227898785978802345
:10EBD8008DF8551041180A318DF856308A238DF872
:10EBE80054008DF857308DF85B200023521815A873
:10EBF80009218DF858308DF859308DF85A308DF834
:10EC08005C20FCF7CDFD7D4A002313707C4A13700D
:10EC18007C4C7D4A002384F83431137084F86731C2
:10EC280094F8643113B10120FAF7CAF894F8352141
:10EC3800744B52B193F86521D2F1010238BF00221A
:10EC480083F86521002283F8352107A8FAF7ECFD3F
:10EC5800002842D09DF81C30062B3ED96B4B9DF8FE
:10EC6800242008991A709DF825205A709DF82620AE
:10EC78009A709DF827209A719DF828205A719DF85E
:10EC880029201A719DF82A20DA709DF81D205D4B05
:10EC980083F86821584A1269914202D1012283F807
:10ECA8006721F9F7DFFA5A4B00221860594B1A709E
:10ECB8009DF81C20534B072A14BF0222012283F817
:10ECC800342193F82720531EDBB2012B524B02D973
:10ECD800052A40F0E880002206E14A4C94F8655184
:10ECE8002646002D73D10DF15F00FAF79DFA002832
:10ECF8006DD0FAF7B7FA08B184F86951414B9DF81D
:10ED08005F0093F8692199180132D2B2092A81F873
:10ED18006A0183F8692140F0ED80002283F86921B7
:10ED2800354A93F86A315178994207D092F82710FA
:10ED3800002900F0DF808B4240F0DC8092F8272029
:10ED48009A4203D12F4B012283F8672100231A46E8
:10ED58002C4C04F5B571595C01335218082BD2B20A
:10ED6800F6D194F8723193422DD1284B94F86B2147
:10ED78001A7094F86C215A7094F86D219A7094F86E
:10ED88006E219A7194F86F215A7194F870211A7152
:10ED980094F87121DA70F9F765FA204B204A186067
:10EDA80094F8271000231370032284F834214A1E94
:10EDB800D2B2012A84F86931174A02D9052918BF45
:10EDC8000123137096E0042384F8343192E096F816
:10EDD80065310C4C33B30D4801F031F910B3F9F734
:10EDE80041FA0E4B0E4A186000231370032284F870
:10EDF800342194F827204EE004000020224C002003
:10EE0800A34D00201C470020D4540020C8530020E4
:10EE18004C4D0020E04B0020DF540020544D0020D2
:10EE28005B4D0020AA4E96F86541002C43D10FADEA
:10EE38002846FCF7E1FC00283DD023462A5D013432
:10EE48009B18082CDBB2F9D19DF844209A422ED1A8
:10EE5800A04B9DF83D201A709DF83E205A709DF8F1
:10EE68003F209A709DF840209A719DF841205A7170
:10EE78009DF842201A719DF84320DA70F9F7F2F9EB
:10EE8800954B964A186000231370914A072182F81F
:10EE9800341192F82720511EC9B201291946904B06
:10EEA80003D9052A01D001221EE0197022E0884BFF
:10EEB80083F834411EE096F82730854C013BDBB2DD
:10EEC800012B17D8236AB3F5006F0FD2F9F7C6FBE9
:10EED80060B1206A7F49431C2362FAF77DFF09234A
:10EEE80084F834317E4B01221A7003E0784B0022FB
:10EEF80083F82720764C94F82730042B234604D136
:10EF0800744E3278110640F1F98093F834313BB1F0
:10EF1800042B05D0082B03D0062B01D0FDF774FD78
:10EF28006B4C94F83431092B40F0A780F9F79AF923
:10EF38006C4BA2681B68801A0028B8BF40429842F0
:10EF480009D9694B1A78012A01D102221A70F9F7F6
:10EF580089F95F4B9860F9F785F95D4A614BD2688A
:10EF68005B68801A0028B8BF4042984209D95E4BB6
:10EF78005A78012A01D102225A70F9F773F9544BD1
:10EF8800D860F9F76FF9524A564B12699B68801A94
:10EF98000028B8BF4042984209D9534B9A78012AB1
:10EFA80001D102229A70F9F75DF9494B1861484B73
:10EFB80093F84C20002A60D093F82C1100295CD1DA
:10EFC8004A4A93F828A11268D3F80C910192484A4A
:10EFD800D3F8108112681C6A0292464AD3F814C109
:10EFE8001268D3F818710392DA69187D04929A6945
:10EFF800D3F81C61D3F82051D3F824B10592CDF889
:10F0080000A00A46DFF8E0A01AF80230022B1BD154
:10F01800DFF8E4A05AF82230B3F1FF3F0FD0D1B2A5
:10F0280006460091A446DDF814B0049D039F1C46D3
:10F03800DDF80880DDF804900121002004E0DFF805
:10F04800A8A000230AF8023001322F2ADAD1204B77
:10F05800009AC3F80C91C3F810811C62C3F814C15C
:10F06800C3F818711875C3F81C61C3F82051C3F8A8
:10F0780024B183F8282183F82C11154A92F83431E9
:10F08800092B06D192F82730022B02D1052382F8EA
:10F098002730D2F838110E4B00295AD093F8342172
:10F0A800092A56D193F82720012A52D1186A00223A
:10F0B80003F59C7353F8044FA04204D1044B052276
:10F0C80083F8272045E001328A42F3D141E000BFAE
:10F0D8001C470020C8530020544D00205B4D0020E1
:10F0E800DF540020144D0020744D0020D05400201F
:10F0F800EC540020D05300206C47002094F83431A1
:10F108003BB3042B25D0082B23D0062B21D0124D3E
:10F11800D4F830016A70D6F80330B0F5006F6B6030
:10F1280012D23146FAF756FFD4F830013146FAF7D1
:10F13800BDFE30B1D4F830310133C4F83031652325
:10F1480000E007232B7004E007232B70002384F8CA
:10F15800273019B0BDE8F08FE4540020704710B58F
:10F16800F9F780F8074C2368C01AB0F5FA7F07D979
:10F17800054B5A6982F040025A61F9F773F820602A
:10F1880010BD00BF085900200010024008B5F9F76B
:10F19800E1FD014B586008BDE454002070477047FA
:10F1A8007047704770477047704700BF2DE9F74FA9
:10F1B80004464FEA440A02274FF0010B07FA0AF700
:10F1C8000BFA0AFB4601F5B2002045F07C0101AAC2
:10F1D800FBF7EBF99DF80630022C07EA03070BEA68
:10F1E800030BB84B1E4496F80880994608F07F0830
:10F1F80001D8601C00E0A01CC0B2F9F76EF909EB59
:10F20800441999F908300646002B03DAD0F10106B3
:10F2180038BF002608F1FF33072B00F2B982DFE878
:10F2280013F008000800080008006601660166017E
:10F238006601A54E335D013B0E2B00F2A982DFE883
:10F2480013F00F003E00550062007B00830093001E
:10F25800A800D70013011801A702360147018E0242
:10F2680045F0140101AA0020FBF79FF99DF805302D
:10F2780006EB840645F00605736000202946FBF777
:10F28800AAF90222306121460020FBF7BAF9A8F159
:10F2980002080020294640F2FF72FBF7E4F85FFA03
:10F2A80088F8002003222146FBF7CCF9B8F1010FBA
:10F2B800854F01D8022300E004233B5568E206EBA2
:10F2C80084035A68002002F00402002A14BF0522B1
:10F2D80001222146FBF7B6F97A4A6301D25845F074
:10F2E80008010020FBF7BFF8032323E0BBF1000F60
:10F2F80000F04E8245F002010020FBF745FB734BFE
:10F3080043F8240030E106EB84035A68002002F039
:10F318000402002A14BF062202222146FBF792F9B2
:10F32800684A6301D25845F0080152420020FBF7B1
:10F338009AF8052333552BE2002F00F02982204646
:10F34800FBF774FA0623F5E7002021460322FBF7B2
:10F3580079F95C4B45F0080103EB44135A68002027
:10F36800FBF781F8072206E2002F40F0118245F0F2
:10F378000805384629463A46FBF775F8514B384692
:10F3880003EB44135A6829465242FBF76CF80822EB
:10F39800F1E1002F00F0FC8145F002010020FBF7AD
:10F3A800F3FA06460020024645F00801FBF75BF831
:10F3B800464B002053F824202146921B43F8242072
:10F3C8000322FBF73FF93F4B6701DB195A6845F009
:10F3D80006010020FBF747F8F9B200203246FBF798
:10F3E80052F8002002462146FBF70BF90922C2E138
:10F3F8000020FBF7D5F840FA0AFA1AF0010F00F0DE
:10F40800C781002045F0080602463146FBF72BF875
:10F41800002002222146FBF7F4F8002045F0020103
:10F428000246FBF730F8650100200246E9B2A8F170
:10F438000308FBF728F85FFA88F800212046F9F757
:10F448005DF9B8F1010F00F29581002021460222F2
:10F45800FBF7D7F81B4B00205D196A68314652420A
:10F46800FBF701F80A2286E1002F00F091810B23B7
:10F4780060E7002F40F08C8145F002013846FBF729
:10F4880083FA45F0080106463A463846FAF7EBFF94
:10F4980061010222C9B296FBF2F23846FAF7F3FF8D
:10F4A8003A4638462146FBF7ACF80D2263E10020C6
:10F4B800FBF776F840FA0AFA1AF0010F00F06881B3
:10F4C8000E2337E7A84C002090480020E44B00208A
:10F4D80006EB840745F0060100203A69FAF7C3FFF6
:10F4E8003A7900202146FBF7ADF8002322E7A94A24
:10F4F800135D9146013B0E2B00F24A81DFE813F0C1
:10F508000F00360058006B008E004801A10048012A
:10F518004801D500E200B90008013E012F0145F07D
:10F528001401002001AAFBF740F89DF8053009EB0B
:10F538008409C9F80430002002222146FBF761F84B
:10F54800002045F0060140F2FF72FAF78CFF002018
:10F5580003222146FBF776F8B8F1060F02D0B8F17E
:10F56800080F01D1022206E1042204E1B8F1060FD6
:10F578000CD109EB8409D9F80420002002F0040218
:10F58800002A14BF05220122214605E0B8F1080F20
:10F5980004D1002021460322FBF754F87E4A630178
:10F5A800D25845F008010020FAF75DFF0322E2E097
:10F5B800A8F10503DBB2012B08D8BBF1000F05D079
:10F5C800B8F1060F734B35D10422D5E0002E00F0B8
:10F5D800DF800C23DAE0B8F1050F0CD109EB8409C0
:10F5E800D9F80420002002F00402002A14BF0622E1
:10F5F8000222214605E0B8F1070F04D10020214678
:10F608000322FBF71FF8644A6301D25845F008014A
:10F6180052420020FAF727FF0522ACE0A8F10503C3
:10F62800DBB2012B08D83FB1B8F1050F594B01D116
:10F638000222A1E00F229FE0002E00F0A9800723FC
:10F64800A4E0002E40F0A48009EB84035A683046F9
:10F6580002F00402002A14BF052201222146FAF70B
:10F66800F1FF4D4B45F0080103EB441330465A684F
:10F6780017E0002E40F08C8009EB84035A6830466E
:10F6880002F00402002A14BF062202222146FAF7D9
:10F69800D9FF414B45F0080103EB44135A68304643
:10F6A8005242FAF7E0FE0A2370E0002E70D045F0CF
:10F6B80002010020FBF768F9364B03EB8402D061A6
:10F6C8000B2259E0002E63D145F002013046FBF7CA
:10F6D8005BF9314B6701DB1945F006012D4D5A687E
:10F6E80080465E733046FAF7CEFE05EB8403DA698E
:10F6F8000223904498FBF3F2F9B23046FAF7C3FEBE
:10F70800304621463246FAF77CFF0D232B553FE061
:10F718000020FAF745FF40FA0AFA1AF0010F37D02D
:10F728000E23002009F8043045F008010246FAF7D4
:10F738009AFE002021460222FAF763FF002045F0D6
:10F7480002010246FAF79FFE002061010246C9B293
:10F75800FAF799FE20460021F8F7D0FF18E00020BC
:10F7680021460222FAF74DFF002045F00801024623
:10F77800FAF779FE0E22074B1A5509E009EB8403C4
:10F788001A7900202146FAF75DFF002309F80430B2
:10F79800BDE8FE8F90480020A84C0020024B1A5C60
:10F7A8000AB901221A54704790480020024B1A5C8B
:10F7B8000AB10F221A54704790480020014B185C78
:10F7C800704700BF90480020F8B50024064D074F49
:10F7D8002646E655E0B2A97A0134F8F71DFE203531
:10F7E800032CF6D1F8BD00BFA84C00205D4D0020C9
:10F7F8002DE9F043974B85B01A7832B96FF0004283
:10F808005A609A60DA6001221A701C7C5CB9E0B216
:10F81800F8F763FE8F4B03F11102A0540134082C52
:10F82800F5D101221A748C4FDFF864828B4E27249D
:10F838000025E8B2F8F751FEEB5D834215D0AB1D09
:10F84800E85558F82330022B05D0032B08D0012B9C
:10F858000BD150B104E040B9325D012A05D103E073
:10F86800335D012B01D10223335501350134082DB5
:10F87800DFD17B4EF369C3B17A4C2578ADB9F8F77F
:10F88800F1FC794B1B68C01AF3690028B8BF4042E5
:10F8980098420AD92846FAF7C9FF0120FAF7C6FFA5
:10F8A8000220FAF7C3FF012323706D4E336AC3B1F8
:10F8B8006E4C2578ADB9F8F7D5FC6D4B1B68C01AAE
:10F8C800336A0028B8BF404298420AD92846FAF756
:10F8D800ADFF0120FAF7AAFF0220FAF7A7FF0123DC
:10F8E80023705C4D634B687E03EB40131C7B6CB14B
:10F8F800614A624B82180092614A00218218019283
:10F9080003EB80030A46FBF781FD0BE3F8F7AAFC3B
:10F91800EB69C01A0028B8BF40420A2840F30283A6
:10F92800697E2046490141F00A01C9B2FAF753FE3F
:10F938000446687EFBF7AFF8687E0C2242435149C3
:10F948008B181D7A0DB18D5800E05D684E4B1B5C1D
:10F95800032B00F2D280DFE803F00257183E002C98
:10F9680000F0CB80434B3B4E03EB4013D97F464D11
:10F9780021B1F8F751FD737E032204E0597AF8F7B4
:10F988004BFD737E0222EA54B7E044B9410141F0CD
:10F998000801C9B22046FAF71EFE00283FD02D4EB6
:10F9A800344B707E03EB4013D97F002900F09E8012
:10F9B80084EAE472A2EBE472002DB8BF6D42AA4259
:10F9C80002D0002C40F08C80304B53F830108A4223
:10F9D80080F08C800FE084EAE472A2EBE472002DE0
:10F9E800B8BF6D42AA4201D0002C7FD1274B53F8F3
:10F9F80030108A4264D203EBC0031979F8F70CFD82
:10FA0800144B01215B7E6FE0002C43D1410141F092
:10FA18000801C9B22046FAF7DEFD00283AD1F8F706
:10FA280021FC0C4D0A266B7E05EB83025268801A76
:10FA3800104A0028B8BF404202EB4312918B714331
:10FA480088425ADD917A1846F8F7E6FC6B7E0E4A32
:10FA5800D45452E0B8480020C9480020744D002012
:10FA6800040000205B4D0020544D0020E04B002096
:10FA78004C4D0020A84C0020004C0020244C0020B5
:10FA8800A34C0020584C00205D4D0020044C002061
:10FA9800144D00200F4E104B707E03EB4013D97F9E
:10FAA80021B384EAE473A3EBE473002DB8BF6D427D
:10FAB800AB4200D0A4B9094A52F83020934215D37A
:10FAC800054B03EB4013597AF8F7A6FC014B0221CA
:10FAD8005B7E09E0B8480020A84C0020044C0020B8
:10FAE800F8F79AFC737E0321A44AD154A44D6E7E84
:10FAF800F8F7B8FB05EB86056860A14DA14A687E5A
:10FB0800A14B82180092A14A0021821803EB8003BE
:10FB180001920A46FBF77AFC9D4F687E07EB40137B
:10FB28009B69002B33D0F8F7B1FD00282FD0687EF1
:10FB380084EAE472A2EBE47207EB40139B699A42F1
:10FB480025D9FAF773FE6B7E924A0121D15407EB4F
:10FB580043139B7F93B10026B8466B7E08EB431393
:10FB68009A7FBB7F9A4205D13046FAF75FFEF0B222
:10FB7800FFF71CFE01362037032EEED1804B864A54
:10FB88005B7E0F33D15C012901D10221D1547C4D18
:10FB98006B7E022B22D80020FAF702FD95F8203060
:10FBA800C60703F0F80385F8203044BF43F001038B
:10FBB80085F8203010F0040F8DF80C00704B05D03C
:10FBC80093F8202042F0020283F82020C00605D5D1
:10FBD80093F8202042F0040283F820206F49704AED
:10FBE8000B784BB1664890F82000034204D113709B
:10FBF8006C4B1B7803B90B701378614A3BB192F8D0
:10FC080020101940994202D1674B0121197092F8CE
:10FC18002030D9070AD55A4A92F82120D20705D4AC
:10FC28005D4AD178012901D10221D1709F070AD5F7
:10FC3800534A92F82120960705D4574A1179012989
:10FC480001D10221117113F0040F4D4A09D092F825
:10FC580021104D0705D450494879012801D10220C7
:10FC68004871517E82F821300323B1FBF3F304AAD3
:10FC7800D31813F9043C002B45DA490141F0160169
:10FC88000020C9B202AAFAF790FC9DF80A3058067B
:10FC980009D53B4A4049527E52001B32885C0128F4
:10FCA80001D10220885419060AD5354A517E3A4AAC
:10FCB8000E3112F81100012802D1022002F81100B9
:10FCC800DA0609D52E4A3449527E52001B32885C26
:10FCD800012801D1022088549B060AD5284B5A7E58
:10FCE8002D4B0E3213F81210012902D1022103F80C
:10FCF8001210234B0020597E02AA490141F0160137
:10FD0800C9B2FAF78FFB1E4D214F6B7E59017A1845
:10FD18005269002A00F09D80244AD65C002E40F0EB
:10FD28009880002C00F0968041F00201C9B230465C
:10FD3800FAF72AFE8046687EF8F7C2FC697EC0EBB7
:10FD4800080807EB41135B69B8F1000FB8BFC8F1A9
:10FD5800000883EAE372A2EBE372904540F38280E5
:10FD6800002B37DD0846FAF761FD6B7E07EB43137E
:10FD78009B7F002B5DD0B8461AE000BF5D4D002088
:10FD8800B8480020004C0020244C0020A34C002040
:10FD9800A84C0020A04C0020744D0020234C0020CB
:10FDA800224C0020F04B0020A34D00201F4C0020C7
:10FDB8006B7E08EB43139A7FBB7F9A4205D130468E
:10FDC800FAF734FDF0B2FFF7F1FC01362037032EC5
:10FDD800EED12EE030460222FAF713FC697E304657
:10FDE800490141F00801C9B2FAF7C2FB6B7E07EB83
:10FDF80043139B7FEBB1B9466B7E09EB43139A7FA4
:10FE0800BB7F9A4211D15FFA86F800204146022250
:10FE1800FAF7F7FB4FEA481141F008010020C9B290
:10FE2800FAF7A6FB4046FFF7C1FC01362037032E40
:10FE3800E2D13E4B3E4A587E00F11503D15C0129C0
:10FE480001D10221D1543B4B01221A54FFF7AEFCD9
:10FE580008E03CB9590141F00801C9B20020FAF79D
:10FE6800BAFB20B1314D344B6E7E9B5D33B32F4DC1
:10FE7800324A6B7E02EB4312D28912B92E4AD35C06
:10FE88000BB3F8F7EFF96B7E0A2105EB83056A6A75
:10FE9800801A2A4A0028B8BF404202EB4312D2898E
:10FEA8004A4390420FDD264DEA5C62B91846FBF7DB
:10FEB80015FB1E4B01225B7EEA5404E0F8F7D2F9E9
:10FEC80005EB86056862194E1E4D707E002CB8BF82
:10FED800644255F830309C420AD2FBF7C9F9737E68
:10FEE80005EBC3056A7982420DD11846002108E066
:10FEF800FBF7BEF9737E05EBC3056979884202D02A
:10FF08001846FBF783F9094C607EFFF74FF9637ECB
:10FF18000133DBB2022B637601D900236376F8F74D
:10FF2800A1F9E06105B0BDE8F08300BFB848002042
:10FF3800744D00201F4C0020604D0020A84C00206C
:10FF4800634D0020044C0020084B1868024604E06A
:10FF58002C2902D100221A7004E0117813460132CC
:10FF68000029F5D1014A013313607047E8480020A1
:10FF780070B50646F9F758F90D4C054618B1002337
:10FF88002371012070BDA368E268934207D2E2188A
:10FF9800127C013301203270A360207170BD04F11E
:10FFA8001000FBF717FCA560E060284670BD00BF95
:10FFB800E848002010B50C4C0A4623791BB9BDE867
:10FFC8001040F9F717B9236DE11881F85400591C4E
:10FFD8000D28216502D03F2900D822B90348FBF734
:10FFE800DFFB0023236510BDE84800203C490020C2
:08FFF80010B50121044686B09A
:020000040801F1
:100000002020FFF7DBFF002C04DA2D200121FFF771
:10001000D5FF644200230A2100E0034694FBF1F27D
:1000200001FB124401A830341C54581C141EF4DC8B
:100030001C4601ABE05C0121FFF7C0FF14F1FF3467
:10004000F7D206B010BD2DE9F74304460DF10700C5
:10005000FFF792FF002800F0C380934B934A93F878
:10006000941019BB51789DF80700403188420DD19A
:10007000D3F89810002940F0B380012183F8941040
:10008000117931F0010140F0AB80A7E00D2801D0DB
:100090001B2802D10022844B05E0D3F898207E2A49
:1000A00000F29E800132C3F8982099E0117931F076
:1000B000010103D19DF80700FFF780FF9DF807308D
:1000C000794D1F2B0AD9D5F898207E2A77D8A91800
:1000D000013281F89C30C5F8982070E0082B07D1D8
:1000E000D5F89830002B6AD0013BC5F8983066E00F
:1000F0000D2B64D1D5F89830002B60D06B4B1A795A
:10010000112A16D1587801214030C0B2FFF756FFAE
:10011000002605F19C0704E0F05D0121FFF74EFF8A
:100120000136D5F898309E42F6D30D200121FFF715
:1001300045FF5D490023C1F81C31D1F898700D6866
:100140001A46184601F590789C4627E001280DD004
:1001500002D3022821D117E0554E965D202E1CD0E7
:10016000C81880F820610133012016E0504E965DDA
:10017000202E0DD1012B03D9C81880F820C10133DE
:1001800008EB0305022008E0494E965D202E04D0BE
:1001900001EB030989F8206101330132BA42D5D15C
:1001A000414A0021C2F81C31D31883F820110123E1
:1001B000156082F89F3182F89410C2F898109DF86B
:1001C00007301B2B0CD1384B0021C3F8981083F853
:1001D0009410364B1B79012B02D10D20FFF7EEFE58
:1001E000314B93F89F01002858D00026DFF8E080BB
:1001F00083F89F6135464FF0070909FB05872D48B5
:10020000394606F005FE28B9BE797B79F1072370DF
:1002100034D508E016F80830002B41D001350736F8
:10022000FF2DEAD13CE0FFF793FE23780546042B2F
:100230000BD1214906F0ECFDF8B128461F4906F024
:10024000E7FD68B128461E490EE00D2B13D11D496C
:1002500006F0DEFD88B128461B4906F0D9FD08B935
:10026000012305E01949284606F0D2FD10B9022302
:10027000637003E0284606F0B1FD6070B20704D554
:10028000FFF766FE06F0AAFDA070730705D5FFF71D
:100290005FFE06F0A3FDC4F803000120BDE8FE8365
:1002A00000232370F9E700BFE84800200400002085
:1002B00084490020084A00209078010894780108B9
:1002C000987801089E780108A4780108A9780108A7
:1002D0005377010838B50C4D0446A8780121403009
:1002E000C0B2FFF76BFE687801214030C0B2FFF763
:1002F00065FE2078FFF780FE6068FFF77DFE0D2029
:100300000121BDE8384059E6040000207047FEE7AF
:10031000FEE7FEE7FEE77047704770477047000052
:100320002E4B82B01A6842F001021A6000229A60D5
:10033000196821F0847121F48031196028495960CD
:10034000196821F480211960DA60009201921A681C
:1003500042F480321A601A6802F400320192009A64
:1003600001320092019A1AB9009AB2F5A06FF2D147
:100370001A4B1B6813F4003318BF01230193019B30
:10038000012B25D1154B9A689A609A6842F4004275
:100390009A609A6842F4A0529A60124A5A601A68A7
:1003A00042F080721A6019680C4A8901FBD50E4B25
:1003B00040F203711960936823F00303936093681C
:1003C00043F002039360936803F00C03082BFAD107
:1003D000064B074A9A6002B0704700BF00380240DF
:1003E00010300024081E4005003C024000ED00E0F3
:1003F00000800008154B16499868164A00F00C005A
:10040000042801D0082801D00A6013E05868596810
:100410005B6801F03F01C3F38813B2FBF1F25A436A
:100420000A4B5B68C3F3014301335B00B2FBF3F299
:10043000074B1A60054B9A68054BC2F303129A18D2
:100440001279196821FA02F21A60704700380240E6
:10045000BC0000200024F400012108B54FF4807096
:1004600001F01AFA4FF480700021BDE8084001F055
:1004700013BA43680A6823F0407323F4807313436C
:100480000A7930B543EA02234360CA680B6984687D
:100490008D681A43084B2A43234013434A7943EAA1
:1004A000420383600B7DC26A013B22F47002DBB21F
:1004B00042EA0353C36230BDFDF7FFC0002303606F
:1004C000037143718360C360036101230375704747
:1004D00010B5074A074B51680B4090E812002143C2
:1004E0008468C068214301430B43536010BD00BFC3
:1004F00000230140E030FCFF002303604360836081
:10050000C3607047836811B143F0010301E023F039
:10051000010383607047436823F4400323F40073AE
:10052000194341607047416282627047436823F01B
:100530001F03194341607047044B5A6810B142F4DD
:10054000000201E022F400025A60704700230140DB
:10055000044B5A6810B142F4800201E022F4800298
:100560005A60704700230140092970B54FF0030419
:100570000DD94C4307251E3C05FA04F503FA04F394
:10058000C66826EA050545EA0304C4600BE04C434F
:10059000072505FA04F503FA04F4066926EA0505B9
:1005A00045EA04030361062A4FF005030CD8013A1B
:1005B00053431F2202FA03F201FA03F3446B24EAC5
:1005C00002021343436370BD0C2A0DD853431F220C
:1005D000233B02FA03F201FA03F1046B24EA02025C
:1005E00042EA0103036370BD53431F22413B02FAF9
:1005F00003F201FA03F1C46A24EA020242EA0103A7
:10060000C36270BD836843F0804383607047806835
:10061000C0F380507047836811B143F4806301E0F8
:1006200023F4806383607047836811B143F0020351
:1006300001E023F00203836070474368013923F42B
:10064000604343EA413141607047436811B143F46C
:10065000006301E023F4006343607047C06C80B224
:100660007047014B1868704708230140836811B137
:1006700043F4807301E023F48073836070478368E0
:1006800011B143F4007301E023F4007383607047F9
:10069000044B5A6810B142F4005201E022F40052B7
:1006A0005A60704700230140092970B54FF00304D8
:1006B0000DD94C4307251E3C05FA04F503FA04F353
:1006C000C66826EA050545EA0304C4600BE04C430E
:1006D000072505FA04F503FA04F4066926EA050578
:1006E00045EA04030361836BC3F30154121B023216
:1006F0000524D2B262431F2404FA02F401FA02F183
:1007000023EA04030B43836370BD836B013923F435
:10071000401343EA01518163704782B00023019383
:100720000190019BC9180191019B1A6002B07047AA
:10073000836823F47023194381607047836823F42E
:100740004013194381607047836843F480038360DA
:1007500070478068C0F380507047436811B143F41C
:10076000806301E023F4806343607047436811B104
:1007700043F4805301E023F480534360704782B018
:10078000002301930190019B283359180191019B8B
:10079000186880B202B070470123C9B203FA01F1B0
:1007A00043680AB1194301E023EA0101416070473F
:1007B000036819420CBF002001207047C943016043
:1007C00070474368006810EA112007D00122C9B2BF
:1007D00002FA01F119420CBF0020012070476FEAB4
:1007E00011210160704700BF08B50B4B984207D13B
:1007F0004FF00070012101F043F84FF0007006E067
:100800004FF08060012101F03BF84FF08060002143
:10081000BDE8084001F034B800640040036823F0EC
:1008200002030360036843F0010303604FF4803365
:100830004268D20701D4013BFAD1436813F00103A7
:1008400056D08B79012B03680CBF43F0800323F053
:1008500080030360CB79012B03680CBF43F0400396
:1008600023F0400303600B7A012B03680CBF43F0B5
:10087000200323F0200303604B7A012B03680CBF95
:1008800043F0100323F0100303608B7A012B0368FD
:100890000CBF43F0080323F008030360CB7A012B5D
:1008A00003680CBF43F0040323F0040303608B7858
:1008B000CA789B0743EA02630A7943EA02434A790A
:1008C00043EA02530A88013A1343C361036823F0E1
:1008D000010303604FF480334268D20701D5013B26
:1008E000FAD1436813F0010F14BF002001207047B4
:1008F00018467047837A012101FA03F170B5354B30
:10090000CC43D3F8002242F00102C3F80022D3F80E
:100910001C222240C3F81C22027BAAB9D3F80C2265
:10092000C6882240C3F80C22827A4588483245EABC
:10093000064543F8325003888288857A43EA0242AA
:10094000254BED00EB185A60037B012B16D1214B90
:100950000688D3F80C2245880A43C3F80C22827A11
:1009600045EA0645483243F83250C3888288857A82
:1009700043EA0242184BED00EB185A60C37A154A5D
:100980001BB9D2F80432234002E0D2F804320B4300
:100990000589C2F804320F4B2DB9D2F814522C40FD
:1009A000C2F8144206E0012D04D1D3F814220A4300
:1009B000C3F81422427B012A04D1D3F81C2211432C
:1009C000C3F81C12D3F8002222F00102C3F800225F
:1009D00070BD00BF0064004040660040002383718A
:1009E000C371037243728372C3728370C370032333
:1009F0000371022343710123038070470D4BD3F829
:100A0000002242F00102C3F80022D3F8002222F4AF
:100A10007C5222F00E02C3F80022D3F8002242EAF0
:100A20000020C3F80002D3F8002222F00102C3F82C
:100A30000022704700640040036811B143F4803322
:100A400001E023F4803303607047036899B143F0F9
:100A500080030360D0F8843143F48073C0F884319C
:100A6000D0F8943143F48073C0F89431D0F8A431B5
:100A700043F4807312E023F080030360D0F88431E4
:100A800023F48073C0F88431D0F8943123F4807358
:100A9000C0F89431D0F8A43123F48073C0F8A431A5
:100AA000704770B582680346500107D49A681201F6
:100AB00006D49A68D0004AD5022002E0002000E067
:100AC000012000F1180212019C5804F001049C500E
:100AD0000C7A9D5824B90E684C7A44EA465404E0D6
:100AE0004E6844EAC6042C434D7A2C439C508A7AC3
:100AF00000F11804240102F00F028A721A195568D5
:100B000025F00F05556055688E7A354355604E7B4C
:100B10008A7B360446EA0266CA7A16430A7B46EAAC
:100B2000022603EB0012C2F8886102F5C4754A7C04
:100B30008E7C120442EA0662CE7B097C324342EA92
:100B400001226A601A5942F001021A5170BD042054
:100B500070BD012906D002D302290AD105E08268BE
:100B60000E4B04E082680E4B01E082680D4B13408F
:100B700000E00023094A93420BD001D83BB10AE0C0
:100B8000074A934205D0074A934204D101E002206C
:100B90007047012070470020704700BF0300000429
:100BA0000003000800000310012907D002D3022926
:100BB0000DD108E0836843F0800302E0836843F4CA
:100BC000004383607047836843F400038360704789
:100BD00030B501F11B042301C55805F00405EDB241
:100BE0001572C35815B95B0D136001E0DB08536043
:100BF00024010319045904F0020454725C6804F0DF
:100C00000F0494725B681B0AD37400EB0113D3F8D2
:100C1000B85103F5DC74D572D3F8B8512D0A1573A9
:100C2000D3F8B8512D0C5573D3F8B8311B0E93730C
:100C30006368D37363681B0A137463681B0C537473
:100C400063681B0E937421B9C36843F02003C3602B
:100C500030BD036943F02003036130BD21B9C3688F
:100C600043F02003C3607047036943F0200303612E
:100C7000704709B9C06802E0012903D1006900F09A
:100C8000030070470020704799B9036823F00303FD
:100C900043F0010303604FF48033426802F0030223
:100CA000012A01D0013BF8D1406800F0030001287F
:100CB00028E0012911D1036823F0030303604FF4F6
:100CC00080334268920701D0013BFAD1436813F0A8
:100CD000030F14BF002001207047022916D10368BA
:100CE00023F0030343F0020303604FF480334268B0
:100CF00002F00302022A01D0013BF8D1406800F063
:100D00000300022814BF0020012070470020704714
:100D1000036823F0030343F002030360406800F01C
:100D20000300A0F10201484240EB01007047036854
:100D300023F0020303604FF480334268920701D529
:100D4000013BFAD1436813F0020F14BF00200120C9
:100D50007047806900F0700070478069000E70472E
:100D60008069C0F30740704743690AB1194301E045
:100D700023EA01014161704711F4700F01D08369CA
:100D80000AE0CB0101D5436806E00A0101D583687A
:100D900002E08B0109D5C36823F07F4323F470037D
:100DA0000B420CBF002001207047036923F07F43F2
:100DB00023F470030B420CBF0020012070470B4B43
:100DC000994202D100238361704721F07F438A0159
:100DD00023F4700301D5C36070474A0101D5036154
:100DE00070470A014CBF8360436070477000F03069
:100DF00043690B405DD040293CD00ED804292DD04A
:100E000004D8012921D0022955D125E0102929D063
:100E100020292DD008294ED122E0B1F5006F3DD018
:100E200009D8B1F5007F33D0B1F5806F34D0B1F57A
:100E3000807F40D128E0B1F5803F1DD0B1F5003F63
:100E40001ED0B1F5004F36D12FE083681B48184003
:100E5000003018BF01207047C06804E0C0680CE093
:100E6000C0680EE0006910F0030018BF0120704751
:100E7000006902E0006904E04068C0F3C000704708
:100E80004068C0F300107047806900F001007047AF
:100E90008069C0F340007047806907E0836913F000
:100EA000700F0CBF0020012070474068C0F3800025
:100EB0007047184670470020704700BF01010100CD
:100EC000B1F5807F35D00CD8082924D004D8012969
:100ED0001CD0042934D11CE020291FD040292FD157
:100EE0001EE0B1F5006F22D006D8B1F5007F20D00A
:100EF000B1F5806F24D11CE0B1F5803F13D0B1F57E
:100F0000003F12D0B1F5004F1AD115E00D4B8360B0
:100F10007047082300E01023C3607047082300E0F7
:100F2000102303617047082304E0102302E000232C
:100F3000836104234360704700238361042343607B
:100F4000704700BF01010100036823F00103036043
:100F50000023036043608360C36003612123436116
:100F60002C4B98421CD02C4B984220D02B4B9842B3
:100F700025D02B4B98422AD02A4B98422FD02A4B6F
:100F8000984233D0294B984237D0294B984204D10C
:100F90004FF03D5243F8AC2C7047264B984203D19A
:100FA0003D2243F8082C7047234B984204D14FF45C
:100FB000746243F8202C7047204B984204D14FF4C0
:100FC000741243F8382C70471D4B984204D14FF0EF
:100FD000746243F8502C70471A4B984203D11A4A56
:100FE00043F8642C7047194B984203D1184A43F8D0
:100FF0007C2C7047174B984203D1174A43F8942C26
:101000007047164B984204BF4FF03D5243F8AC2C4A
:10101000704700BF106002402860024040600240FC
:10102000586002407060024088600240A060024048
:10103000B8600240106402402864024040640240EC
:1010400058640240706402403D0000208864024001
:10105000400F0020A064024000003D20B864024020
:101060000268134B10B51340CC680A6822434C69E0
:1010700022438C692243CC6922430C6A22434C6A86
:1010800022438C6A22434C6B22438C6B22431343D2
:10109000036042690C6BCB6A22F0070223431343BF
:1010A00043610B6943604B6883608B68C36010BD0C
:1010B0003F801CF00023036043608360C3600361D2
:1010C00043618361C361036243628362C3620363FA
:1010D000436383637047036811B143F0010301E088
:1010E00023F0010303607047036811B143F4004328
:1010F00001E023F4004303607047036811B143F03B
:10110000200301E023F02003036070474160704733
:10111000406880B27047036812B143F4002301E0D5
:1011200023F40023036001617047036811B143F4A5
:10113000802301E023F48023036070470AB101613A
:101140007047C16070470068C0F3C04070470068D6
:1011500000F001007047406900F03800704710B59A
:10116000084A094B094CA0428CBF104618468B0018
:10117000074B4CBF426802680B4013420CBF002073
:10118000012010BD00640240006002400F64024074
:101190007D0F7D0F10B5084B084A094CA0428CBF4B
:1011A00010461846074B11F0005F01EA030314BF15
:1011B000C360836010BD00BF006002400064024055
:1011C0000F6402407D0F7D0F0B0607D5436912B1F6
:1011D00043F0800301E023F080034361802909D0BC
:1011E00001F01E01036812B119430160704723EA40
:1011F000010101607047104B10B5104A104CA0421D
:101200008CBF14461C460F4B0B402BB1026802F0FA
:101210001E0202EAD12202E0426902F08002880046
:10122000094B4CBF606820680B40184002D0101C6E
:1012300018BF012010BD00BF0060024000640240E2
:101240000F6402403C0F3C0F7D0F7D0F10B5084B23
:10125000084A094CA0428CBF10461846074B11F0B3
:10126000005F01EA030314BFC360836010BD00BFC9
:1012700000600240006402400F6402407D0F7D0F59
:10128000044B00221A605A609A60DA60024A5A617E
:10129000704700BF003C0140FFFF7F00837910B51D
:1012A000002B29D01A4B01681C68CA4314401C60EB
:1012B0005C6822405A60027902F1804202F59E3257
:1012C00014682143116002689C68D1430C409C6003
:1012D000DC682140D9604179102906D19968114311
:1012E0009960D9680A43DA6010BD01F1804303F5C3
:1012F0009E3319680A4308E00379016803F18043CB
:1013000003F59E331A6822EA01021A6010BD00BF7D
:10131000003C014000230C22036003714271837181
:101320007047024B1A69104318617047003C014036
:10133000034B5B6918420CBF00200120704700BFBF
:10134000003C0140014B5861704700BF003C014028
:10135000054B1A685B69034004D010420CBF0020A3
:101360000120704718467047003C0140014B58610E
:10137000704700BF003C014008B52C4B984205D196
:101380000120014600F058FA012048E0284B98421D
:1013900005D10220012100F04FFA02203FE0254B49
:1013A000984205D10420012100F046FA042036E0DD
:1013B000214B984205D10820012100F03DFA082078
:1013C0002DE01E4B984205D11020012100F034FA87
:1013D000102024E01A4B984205D12020012100F072
:1013E0002BFA20201BE0174B984205D14020012109
:1013F00000F022FA402012E0134B984205D18020E1
:10140000012100F019FA802009E0104B98420BD11D
:101410004FF48070012100F00FFA4FF4807000212A
:10142000BDE8084000F008BA08BD00BF0000024057
:101430000004024000080240000C0240001002407C
:101440000014024000180240001C0240002002402C
:101450002DE9F0470023D1F800801A464FF0010C27
:1014600003270CFA02F404EA0805A54231D107FA71
:1014700003F40668E443264006600E79D0F8009035
:1014800006FA03FA013EF6B24AEA0909012EC0F84B
:10149000009015D891F80590866809FA03F926405E
:1014A0008660866849EA06068660466826EA05057B
:1014B00045608D79466805FA02F5ADB23543456061
:1014C000C5682C40C460CC79C56804FA03F42C4389
:1014D000C46001320233102AC3D1BDE8F0874FF651
:1014E000FF7303600023037143718371C3717047FD
:1014F00082B04FF480330193019B0B430193019B16
:10150000C361C161019BC361C3690193C369019355
:1015100002B07047036919420CBF002001207047D8
:10152000006980B27047436919420CBF0020012056
:101530007047406980B270470183704741837047AC
:101540000AB1018370474183704741617047436925
:1015500059404161704701F0070330B59B000F24EB
:1015600004FA03F402FA03F3C908083150F82150D1
:1015700025EA040440F8214050F82140234340F874
:10158000213030BD0A4B1A6842F001021A60002275
:101590009A60196821F0847121F48031196005493D
:1015A0005960196821F480211960DA60704700BF22
:1015B0000038024010300024024B00221A701870CC
:1015C000704700BF02380240034B1A6822F0F8024D
:1015D00042EAC0001860704700380240014B1860B2
:1015E000704700BF00004742064B002201281A70D6
:1015F0001A7002D0042804D101E018707047052247
:101600001A70704770380240014B1860704700BF75
:10161000800E4742014341EA8212009942EA016189
:101620005A08013A024B41EA02425A60704700BF31
:1016300000380240014B1860704700BF600047420D
:101640008001034B40EA0170C3F88400704700BF7B
:1016500000380240014B1860704700BF68004742E5
:10166000014B1860704700BF4C004742034B9A681B
:1016700022F0EC6210430843986070470038024043
:10168000034B9A6822F078421043084398607047F1
:1016900000380240034B9A6822F00302104398601E
:1016A000704700BF00380240024B986800F00C0001
:1016B000704700BF00380240034B9A6822F0F002E6
:1016C00010439860704700BF00380240034B9A688F
:1016D00022F4E05210439860704700BF0038024087
:1016E000034B9A6822F4604242EAC0009860704757
:1016F0000038024010B51A4B1A4A996801F00C01E3
:10170000042913D0082911D15C6859685B6801F07D
:101710003F01C3F38813B2FBF1F25A43104B5B68ED
:10172000C3F3014301335B00B2FBF3F20C490260E7
:101730008B680D4AC3F30313D35C046824FA03F3E4
:1017400043608C68C4F38224145D23FA04F484603B
:101750008968C1F34231525C23FA02F3C36010BDC1
:10176000003802400024F400D000002000F4407350
:10177000B3F5407F084B08D1996820F0704221F4FE
:10178000F81122F440720A439A601A6F000542EA87
:1017900010501867704700BF00380240014B1860B6
:1017A000704700BF3C0E4742014B1860704700BFB6
:1017B000400E4742014B1860704700BF5C01474232
:1017C000044B1A6B09B1104301E022EA00001863D0
:1017D000704700BF00380240044B5A6B09B11043F8
:1017E00001E022EA00005863704700BF0038024061
:1017F000044B9A6B09B1104301E022EA00009863A0
:10180000704700BF00380240044B1A6C09B1104306
:1018100001E022EA00001864704700BF003802406F
:10182000044B5A6C09B1104301E022EA00005864ED
:10183000704700BF00380240044B1A6909B11043D9
:1018400001E022EA00001861704700BF0038024042
:10185000044B5A6909B1104301E022EA00005861C3
:10186000704700BF00380240044B9A6909B1104329
:1018700001E022EA00009861704700BF0038024092
:10188000044B1A6A09B1104301E022EA0000186211
:10189000704700BF00380240044B5A6A09B1104338
:1018A00001E022EA00005862704700BF00380240A1
:1018B000044B1A6D09B1104301E022EA00001865DB
:1018C000704700BF00380240044B5A6D09B1104305
:1018D00001E022EA00005865704700BF003802406E
:1018E000044B9A6D09B1104301E022EA00009865AB
:1018F000704700BF00380240044B1A6E09B1104314
:1019000001E022EA00001866704700BF003802407C
:10191000044B5A6E09B1104301E022EA00005866F8
:10192000704700BF00380240044B1A7809B11043D9
:1019300001E022EA00001870704700BF0D38024035
:101940004309012B074A01D1136803E0022B0CBFA6
:10195000136F536F00F01F0023FA00F000F0010036
:10196000704700BF0038024007B5002301933120C3
:10197000FFF7E6FF019B01330193019BB3F5A06FD5
:1019800001D00028F3D03120FFF7DAFF003018BF74
:1019900001200EBD024B5A6F42F080725A677047A9
:1019A00000380240034BDB6818420CBF00200120C6
:1019B000704700BF00380240014B1870704700BFED
:1019C0000E38024008B5154B98420BD101214FF457
:1019D0008050FFF761FF4FF480500021BDE80840C0
:1019E000FFF75ABF0E4B984207D14FF480400121B8
:1019F000FFF746FF4FF4804009E00A4B98420BD1B5
:101A00004FF400400121FFF73BFF4FF4004000215D
:101A1000BDE80840FFF734BF08BD00BF00300140FB
:101A200000380040003C00400B8810B54C8802880C
:101A300023438C8802F441522343CC8823430C89EE
:101A400023434C8923438C892343CC892343134369
:101A50009BB20380838B23F400631B041B0C8383E2
:101A60000B8A038210BD838BF0B523F47A6323F0D5
:101A70001F031B041B0C8383022303848B68858B49
:101A8000022BADB238D0294A8E889468002E14BF3C
:101A900002260126240203D5946824F400049460ED
:101AA000D2F88440D2F884705268DFF884C002F023
:101AB0003F02BCFBF2F2C4F388145443C7F3027232
:101AC000B4FBF2F4CA88B2F5007F4FF00A0201D1EC
:101AD000240A02E07601B4FBF6F46243B2FBF3F3AE
:101AE00005330A229BB2B3FBF2F303F001021202A8
:101AF000C3F34F0392B200E000229C1EA4B2FE2C5E
:101B000028BF0022CC8828BF0223134323439BB263
:101B100003840B884A882B4343F4006313438A8869
:101B200013438A8913439BB28383F0BD003802407C
:101B30000024F4000023038043808380C38003815A
:101B400043818381C38107230382704700230222DC
:101B5000038043808380C3808260838170470388D1
:101B600019B19BB243F0400303E023F040031B0490
:101B70001B0C03807047838B19B19BB243F48063C5
:101B800003E023F480631B041B0C838370470388EA
:101B900023F400631B041B0C038003889BB21943CE
:101BA00001807047B1F5804F038803D19BB243F4A5
:101BB000804303E023F480431B041B0C0380704725
:101BC0004FF6FF639942038803D09BB243F48073BE
:101BD00003E023F480731B041B0C0380704783888D
:101BE00019B19BB243F0040303E023F004031B0488
:101BF0001B0C83807047838819B19BB243F010039C
:101C000003E023F010031B041B0C838070478089C2
:101C100080B2704781817047038819B19BB243F449
:101C2000005303E023F400531B041B0C0380704794
:101C300003889BB243F4805303807047012902D08C
:101C4000008B80B27047808A80B27047008A80B271
:101C5000704783889BB20AB1194301E023EA01016E
:101C6000818070470123090903FA01F1838889B251
:101C70009BB20AB1194301E023EA01018180704758
:101C8000038919420CBF002001207047C94389B263
:101C900001817047012301F00F0203FA02F210B52F
:101CA00084880089A4B280B2104006D0090903FAE2
:101CB00001F31C420CBF0020012010BD01F00F01F8
:101CC000012303FA01F3DB439BB20381704700BF9A
:101CD000012108B54FF48040FFF7DEFD4FF480404E
:101CE0000021BDE80840FFF7D7BD014B18607047E1
:101CF0000038014001F0030230B592000F2404FACD
:101D000002F400FA02F2074B8908023153F821501D
:101D100025EA040443F8214053F82140224343F8C4
:101D2000212030BD00380140014B1860704700BFD2
:101D3000DC002742014B1860704700BF00042742B7
:101D4000024B186AC0F30020704700BF0038014002
:101D500030B5048C24F001042404240C0484058B85
:101D6000048CADB225F0F305A4B22A4342EA031273
:101D700024F00A0343F0010392B219430283018461
:101D800030BD30B5058C25F010052D042D0C0584D3
:101D9000048B058C24F440742405240DADB244EA70
:101DA000022242EA033225F0A00343F0100343EA83
:101DB000011192B289B20283018430BD08B5474B4C
:101DC000984205D101200146FFF766FD01203DE064
:101DD000B0F1804F05D101200146FFF751FD0120F0
:101DE00076E03F4B984205D102200121FFF748FDE4
:101DF00002206DE03B4B984205D104200121FFF702
:101E00003FFD042064E0384B984205D108200121B1
:101E1000FFF736FD08205BE0344B984205D11020D7
:101E20000121FFF72DFD102052E0314B984205D1E2
:101E300020200121FFF724FD202049E02D4B98426E
:101E400009D102200121FFF727FD02200021BDE872
:101E50000840FFF721BD284B984207D14FF480304E
:101E60000121FFF719FD4FF48030EFE7234B984233
:101E700007D14FF400300121FFF70EFD4FF4003081
:101E8000E4E71F4B984207D14FF480200121FFF770
:101E900003FD4FF48020D9E71A4B984205D140202A
:101EA0000121FFF7EDFC402012E0174B984205D1CD
:101EB00080200121FFF7E4FC802009E0134B9842C9
:101EC0000BD14FF480700121FFF7DAFC4FF48070E2
:101ED0000021BDE80840FFF7D3BC08BD0000014069
:101EE0000004004000080040000C004000100040CA
:101EF0000014004000040140004001400044014043
:101F00000048014000180040001C00400020004034
:101F10001C4A038890429BB212D002F58062904224
:101F20000ED0B0F1804F0BD0A2F58032904207D096
:101F300002F58062904203D002F58062904203D1A4
:101F40004A8823F0700313430F4A904208D002F5E9
:101F50008062904204D023F440730A899BB21343F9
:101F600003804B68C3620B880385064B984203D0FD
:101F700003F58063984201D18B7A03860123838223
:101F8000704700BF00000140001000404FF0FF33D9
:101F9000436000230380038143808372704701857F
:101FA00082827047038823F070031B041B0C0B43D1
:101FB0000380704741627047C1627047406A704752
:101FC000008D80B27047038819B19BB243F00203C1
:101FD00003E023F002031B041B0C038070470388FB
:101FE00019B19BB243F0040303E023F004031B0484
:101FF0001B0C03807047038819B19BB243F0800328
:1020000003E023F080031B041B0C0380704703884C
:1020100023F008031B041B0C038003889BB21943A5
:1020200001807047038823F440731B041B0C03805A
:1020300003889BB2194301807047038819B19BB292
:1020400043F0010303E023F001031B041B0C038096
:102050007047038C70B523F001031B041B0C038431
:10206000038C8488028B0D8822F073021204120CF8
:102070002A434E888D8923F002031B0435431B0C31
:10208000ADB22B430E4DA4B2A84203D005F5806536
:10209000A8420ED1CD8923F008032B438D8823F06D
:1020A00004032B434E8A0D8A24F440743543ADB2A9
:1020B0002C43848002838A684263038470BD00BF1E
:1020C00000000140038C30B523F010031B041B0CEF
:1020D0000384038C8288048B0D8824F4E644240452
:1020E000240C23F0200344EA05241B048D891B0CD7
:1020F00043EA05134D8892B243EA0513124DA4B288
:10210000A8429BB203D005F58065A84215D1CD89C0
:1021100023F080039BB243EA05134FF6BF751D40C1
:102120008B8822F4406245EA03130D8A9BB242EA8F
:1021300085024D8A42EA850292B282808A680483CF
:102140008263038430BD00BF00000140038C30B5C2
:1021500023F480731B041B0C0384038C8288848B00
:102160000D8824F073042404240C23F400731B044E
:102170002C438D891B0C43EA05234D8892B243EA18
:102180000523124D9BB2A84203D005F58065A842F5
:1021900015D1CD8923F400639BB243EA05234FF6A2
:1021A000FF351D408B8822F4405245EA03230D8AF7
:1021B0009BB242EA05124D8A42EA051292B282802F
:1021C0008A688483C263038430BD00BF000001407D
:1021D000038C30B523F480531B041B0C0384038C45
:1021E0008488828B0D8822F4E6421204120C23F4B8
:1021F000005342EA05221B048D891B0C43EA053378
:102200004D88A4B243EA05330A4D92B2A8429BB26C
:1022100003D005F58065A84205D10D8A24F48044D9
:1022200044EA8514A4B2848082838A6802640384A9
:1022300030BD00BF00000140002303804380838045
:1022400083608381C38103824382704730B5012458
:1022500004FA01F4058C00F11803ADB225EA040478
:10226000048409B1082907D14908CC584FF68F706A
:102270002040C850C8580AE00439C1F34E01CC5878
:1022800048F6FF702040C8501202C85892B202436C
:10229000CA5030BD4163704781637047C163704766
:1022A00001647047038B23F070031B041B0C0B436A
:1022B00003837047038B23F4E0431B041B0C43EAA6
:1022C00001239BB203837047838B23F070031B04AD
:1022D0001B0C0B4383837047838B23F4E0431B0465
:1022E0001B0C43EA01239BB283837047038B23F0CB
:1022F00008031B041B0C0B4303837047038B23F45D
:1023000000631B041B0C43EA01239BB20383704749
:10231000838B23F008031B041B0C0B438383704740
:10232000838B23F400631B041B0C43EA01239BB241
:1023300083837047038B23F004031B041B0C0B43A4
:1023400003837047038B23F480631B041B0C43EA55
:1023500001239BB203837047838B23F004031B0488
:102360001B0C0B4383837047838B23F480631B0414
:102370001B0C43EA01239BB283837047038B23F03A
:1023800080031B041B0C0B4303837047038B090260
:102390005B0441EA534189B201837047838B23F088
:1023A00080031B041B0C0B4383837047838B090240
:1023B0005B0441EA534189B281837047038C23F067
:1023C00002031B041B0C0B4303847047038C23F094
:1023D00008031B041B0C0B4303847047038C23F07E
:1023E00020031B041B0C43EA01139BB203847047B8
:1023F000038C23F080031B041B0C43EA01139BB2E4
:1024000003847047038C23F400731B041B0C43EA02
:1024100001239BB203847047038C23F400631B04E5
:102420001B0C43EA01239BB203847047038C23F403
:1024300000531B041B0C43EA01339BB20384704717
:10244000012303FA01F302FA01F110B5048CA4B2DE
:1024500024EA03030384038C194389B2018410BD69
:10246000042303FA01F302FA01F110B5048CA4B2BB
:1024700024EA03030384038C194389B2018410BD49
:1024800000230122038043808280C3800381704740
:10249000406B7047806B7047C06B7047006C704733
:1024A000038B23F00C031B041B0C0383038B9BB2D5
:1024B000194301837047038B23F440631B041B0CF7
:1024C0000383038B9BB243EA012189B201837047E6
:1024D000F8B50C4605464988A288208800290CBF1B
:1024E00002270027012A14BF01260226238988B962
:1024F0002846FFF72DFCE1882846FFF7D1FF284644
:10250000394623893246FFF73CFCE1882846BDE87E
:10251000F840D0E72846FFF734FCE1882846FFF76B
:10252000CAFF2846394623893246FFF711FCE18865
:102530002846BDE8F840B3E7838B23F00C031B0467
:102540001B0C8383838B9BB2194381837047838BDE
:1025500023F440631B041B0C8383838B9BB243EAED
:10256000012189B2818370470B8870B50D460446FE
:102570004988AA883BB92B89FFF7EAFBE9882046FE
:10258000BDE870408CE7042B07D12B89FFF7F9FBDE
:10259000E9882046BDE870408DE7082B2E89038C22
:1025A0001CD123F480731B041B0C0384808B238CAD
:1025B00080B29BB220F0F30023F4206340EA0616B9
:1025C00043EA0121B6B289B2324341F48071A28359
:1025D0002184E9882046BDE87040ADE723F48053AC
:1025E0001B041B0C0384808B238C20F4407023F489
:1025F000005300055B04000D5B0C40EA022243EA35
:10260000013342EA06329BB2E98892B243F4805326
:102610002046A2832384BDE8704098E74A880B884F
:1026200013438A881343CA8813430A8913434A8988
:1026300013438A8913439BB2A0F8443070470023A8
:10264000038043808380C3800381438183817047FB
:10265000B0F8443029B16FEA43436FEA53439BB269
:1026600001E05B045B0CA0F844307047838819B12B
:102670009BB243F0040303E023F004031B041B0C90
:1026800083807047838819B19BB243F0010303E054
:1026900023F001031B041B0C8380704783899BB2CA
:1026A0000AB1194301E023EA010181817047818267
:1026B0007047038A19420CBF002001207047C943AC
:1026C00089B201827047038A828911EA030092B2BB
:1026D00003D011420CBF002001207047C94389B2CA
:1026E000018270471143A0F84810704783899BB25C
:1026F0000AB1194301E023EA01018181704783880F
:1027000019B19BB243F0080303E023F008031B0454
:102710001B0C83807047038923F007031B041B0CE9
:1027200003817047038923F070031B041B0C0B43C8
:10273000038103899BB243F007030381704738B5D7
:102740000D4611460122602D044602D1FFF719FB08
:1027500001E0FFF7FDFA238923F070031B041B0C33
:102760001D43258123899BB243F00703238138BD94
:10277000038923F070031B041B0C0B430381704778
:10278000838823F070031B041B0C838083889BB217
:10279000194381807047038923F007031B041B0C36
:1027A000038103899BB2194301817047038923F098
:1027B00080031B041B0C038103899BB21943018115
:1027C000704710B50489E4B221430A4342EA032268
:1027D00092B2028110BD10B50446FFF7F2FF2389C3
:1027E0009BB243F48043238110BD10B50446FFF72C
:1027F000E8FF238923F077031B041B0C43F07703C6
:10280000238110BD70B50589048B25F00705068C62
:102810002D0424F440742D0CB6B224F00304294393
:10282000240426F02205240C2A4344F4807442EA4E
:10283000031244F0010492B201810483028470BD4A
:10284000838819B19BB243F0800303E023F0800337
:102850001B041B0C83807047A0F85010704700BF0A
:1028600008B5234B984205D110200121FFF714F839
:10287000102037E01F4B984207D14FF40030012160
:10288000FEF7FEFF4FF4003009E01B4B98420BD1DE
:102890004FF480200121FEF7F3FF4FF48020002148
:1028A000BDE80840FEF7ECBF144B984207D14FF447
:1028B00000200121FEF7E4FF4FF40020EFE7104B6A
:1028C000984207D14FF480100121FEF7D9FF4FF451
:1028D0008010E4E70B4B984209D120200121FEF73C
:1028E000DBFF20200021BDE80840FEF7D5BF08BD72
:1028F000001001400044004000480040004C0040EF
:10290000005000400014014030B5038ACA889BB2D1
:1029100023F44053134303820D4683890989AA880F
:1029200023F4B0530A43698923F00C031B040A43C0
:102930001B0C92B213438381838AAA899BB223F42E
:102940004073134385B0838204466846FEF7D2FE87
:102950001A4B9C4203D003F580639C4201D1039B38
:1029600000E0029BA2894FF0190112B2002A01FB7C
:1029700003F12A6801DA520000E092006423B1FBFF
:10298000F2F1B1FBF3F21201100903FB1011A0895F
:1029900000B2002806DAC9003231B1FBF3F303F0CC
:1029A000070305E009013231B1FBF3F303F00F0334
:1029B0001A4392B2228105B030BD00BF0010014021
:1029C0004FF4165303600C2200238380C3800381DD
:1029D0004281838170470B8810B54C88028A23435B
:1029E0008C88C988234392B20B4322F470629BB255
:1029F0001343038210BD0023038043808380C38080
:102A00007047838919B19BB243F4005303E023F468
:102A100000531B041B0C83817047038B03F47F431B
:102A20000383038B9BB2194301837047838929B1C8
:102A30006FEA43436FEA53439BB201E05B045B0CD4
:102A400083817047838A19B19BB243F4006303E02A
:102A500023F400631B041B0C83827047C905C90D56
:102A6000818070478088C005C00D7047038A23F0BD
:102A70000F031B041B0C0382038A9BB219430182C0
:102A80007047838919B19BB243F0020303E023F03E
:102A900002031B041B0C83817047838923F40063AA
:102AA0001B041B0C838183899BB21943818170476E
:102AB000038A23F020031B041B0C0382038A9BB2AE
:102AC000194301827047038A19B19BB243F48043D2
:102AD00003E023F480431B041B0C038270478389AB
:102AE0009BB243F0010383817047838A19B19BB283
:102AF00043F0080303E023F008031B041B0C83824C
:102B00007047038BDBB20383038B9BB243EA012143
:102B100001837047838A19B19BB243F0200303E01D
:102B200023F020031B041B0C83827047838A19B196
:102B30009BB243F0100303E023F010031B041B0CB3
:102B400083827047838A23F004031B041B0C838257
:102B5000838A9BB2194381827047838A19B19BB2E1
:102B600043F0020303E023F002031B041B0C8382E7
:102B70007047838A9BB20AB1194301E023EA01013D
:102B800081827047C1F3421310B5012401F01F0187
:102B9000A34204FA01F101D10C3004E0022B01D16F
:102BA000103000E0143003680AB1194301E023EA51
:102BB0000101016010BD038819420CBF00200120F3
:102BC0007047C94389B20180704710B5C1F3421400
:102BD000012201F01F03012C02FA03F201D18389C3
:102BE00003E0022C0CBF038A838A9BB21340028845
:102BF00092B243B1090A012303FA01F111420CBF59
:102C00000020012010BD184610BD090A012303FA57
:102C100001F3DB439BB20380704700BF40F0BE600E
:102C2000024B40F42020D860704700BF00ED00E068
:102C3000C37810B503B3164B4278DB688478DB4366
:102C4000C3F30223C3F10401C9B202FA01F10F2256
:102C500042FA03F2C9B222400A430E4B0178120134
:102C6000CB18D2B283F8002303780122590903F06C
:102C70001F0302FA03F307E003780122590903F066
:102C80001F0302FA03F32031024A42F8213010BD3B
:102C900000ED00E000E100E021F0604121F07F0163
:102CA000014B08439860704700ED00E0044B1A693F
:102CB00009B1104301E022EA00001861704700BF2B
:102CC00000ED00E0044B04281A680CBF42F0040237
:102CD00022F004021A60704710E000E0D0F8E835F6
:102CE00010B51B6904469847032384F8123100206D
:102CF00010BD08B590F8123180F81331042380F824
:102D00001231D0F8E835DB689847002008BD08B5D7
:102D1000D0F8E435DB6903B19847002008BD08B559
:102D2000D0F8E4351B6A9847002008BD08B5D0F8F4
:102D3000E4355B6A9847002008BDD0F8E83510B547
:102D40005B6904469847012384F81531002010BDC3
:102D5000D0F8E83510B59B6904469847D4F8E435B7
:102D600020465B6800219847002084F8150110BDBB
:102D7000002110B5402204460B4601F06BF980217A
:102D800040220023204601F065F9012384F8123126
:102D9000D4F8E835A0785B689847002010BD13B5DB
:102DA0006946044600F078FA9DF8001001F01F0310
:102DB000012B07D0022B0AD073B92046694600F0D8
:102DC00015FB0FE02046694600F0F6FA0AE02046BF
:102DD000694600F091FA05E021F07F01C9B2204672
:102DE00001F0AAF900201CBD38B50446002948D1DD
:102DF00090F81131022B38D1D0F83821D0F8243195
:102E00009A4211D9C178D21A0129C0F8382104D1C7
:102E1000D0F82811CB18C0F8283192B22046D4F847
:102E2000281100F0F3F920E0D0F83C21B2FBF3F5D3
:102E300003FB152565B99A420AD3D0F840319A426E
:102E400006D229462A4600F0E1F9C4F840510CE0C8
:102E5000D4F8E435DB682BB194F81221032A01D1B0
:102E600020469847204600F002FA94F81631012BCC
:102E700010D1094A236912685A60002384F8163178
:102E800008E0D0F8E4355B6923B190F81221032AF9
:102E900000D19847002038BD0C59002010B50446D9
:102EA00059BB90F81131032B30D1D0F89023D0F8D2
:102EB0007C339A4214D9C178D21A0129C0F89023E0
:102EC00004D1D0F88013C918C0F880139A4228BFE3
:102ED0001A4692B22046D4F8801300F0B0F915E0FB
:102EE000D0F8E4351B6923B190F81221032A00D1F0
:102EF0009847204600F0ACF908E0D0F8E4359B692B
:102F000023B190F81221032A00D19847002010BD68
:102F10002DE9F041069F0446164698460D46F8F7FF
:102F2000C1FB20462946C4F8E485C4F8E875C4F816
:102F3000EC6501F041F8D4F8E8351B689847204665
:102F4000BDE8F041F8F700BC00207047D0F8E43548
:102F500010B51B6804469847D4F8E8359B68984735
:102F6000002010BD08B5D0F8E4355B689847002014
:102F700008BD00BF43230B800048704710010020AC
:102F800038B51D4B1A68511C052A196031D11979C1
:102F9000002201291A602CD09968B1F5006F08BF92
:102FA0009A60154B9968DC681A46A14202D100224A
:102FB0001A711EE095BFC1EB0404C1F500631461F2
:102FC000136115690C4C402D8AB205D94031403D42
:102FD000A1602561402304E06918A1600021ABB223
:102FE0002161054901240C7104498A18812101F0ED
:102FF00087F8002038BD00BF884A00209B59002078
:1030000038B5282303FB0101074C084B0546B1F8EE
:103010008C131B69204698472846012122464023ED
:1030200001F052F8002038BD53590020A8000020BC
:1030300070B50B78064613F060050C4625D0202DA0
:103040001FD1CD88B5B113F0800F487808D0224B3E
:1030500022492A469B689847E28830461F4928E063
:103060001F4B1E4958641F4B30465D612A4600F0D5
:10307000D6F820E0184B48789B6829462A4698479E
:1030800028E000F02BF9022524E04B780A2B14D01D
:103090000B2B17D0062B1DD14B881B0A212B05D1DA
:1030A000CA8811493A2A28BF3A2201E00F493A2238
:1030B000304600F09BF800250CE00D49012200F09D
:1030C00095F807E08B781BB9064A1D46936101E02D
:1030D00000F004F9284670BDA80000209359002094
:1030E00010010020884A0020220100201901002040
:1030F000A04A002010B58121044600F0CCFF012138
:10310000204600F0C8FF8221204600F0C4FF024B99
:103110005B689847002010BDA800002038B58121C9
:1031200004464022022300F095FF012140220223A1
:10313000204600F08FFF822108220323204600F062
:1031400089FF084B022200251A715D71064B1B682E
:10315000984720460121054A402300F0B5FF284644
:1031600038BD00BF44000020A800002053590020B3
:1031700010B5074C606CFF2807D0064B064A9B68C9
:10318000064952699847FF236364002010BD00BFC1
:1031900010010020A8000020884A00209359002038
:1031A00038B510490B79012B19D10C690CB90C7188
:1031B00015E0402C07D98B68403C9AB240338B60B5
:1031C0000C61402306E08D68A3B22C198C600024AA
:1031D000AAB20C6104495218812100F091FF00202D
:1031E00038BD00BF884A00209B59002010B5134607
:1031F0000C46C0F83C21C0F83821022280F8112189
:103200000021224600F07CFF002010BD10B50C46C6
:1032100013460021224600F073FF002010BD10B5B8
:1032200013460C46C0F89423C0F89023032280F87C
:1032300011210021224600F047FF002010BD10B5EB
:103240000C4613460021224600F03EFF002010BD30
:103250000021042310B50A46044680F811310B46BC
:1032600000F04EFF204600F0CFFD002010BD0021F1
:10327000052310B50A46044680F811310B4600F0CC
:1032800023FF204600F0C0FD002010BD282303FBD3
:103290000100B0F88C03704790F8CC350B7090F8B3
:1032A000CD354B7090F8CF2590F8CE3503EB022347
:1032B0004B8090F8D12590F8D03503EB02238B801A
:1032C00090F8D32590F8D23503EB02239BB2CB8044
:1032D000C0F84031012380F81131704710B58021CA
:1032E000044600F029FF2046002100F025FF20467B
:1032F000BDE8104000F088BD38B50D466B78044637
:10330000012B097910D027D3032B51D190F812311A
:10331000022B28D0032B47D16B889BB991B1802910
:1033200010D000F009FF0DE090F81231022B1AD0F6
:10333000032B39D16B88002B3AD149B1802907D0B2
:1033400000F018FFD4F8E43520469B6829469847DA
:103350002046FFF77DFF2BE090F81231022B02D0C0
:10336000032B21D106E019B3802921D0204600F09B
:10337000E3FE1DE011F0800F4FF0280306D001F0AE
:103380007F0103FB010393F81E2103E003FB01010E
:1033900091F87623074B02B101221A6020460549B5
:1033A0000222FFF723FF03E020462946FFF796FF9E
:1033B000002038BDA44A002038B590F812310446E8
:1033C000032B0D460CD10B79012B09D8D0F8E4352D
:1033D0009B689847EB883BB92046FFF739FF03E02D
:1033E00020462946FFF77AFF002038BD73B54B7899
:1033F00004460D46092B00F21C81DFE813F0CD00D6
:1034000008011A01E0001A0172000A001A01BD0049
:1034100091006B881A0A013A062A00F20A81DFE855
:1034200012F007001A00270008010801080108012E
:10343000D0F8EC350DF106011B6880789847EB88D1
:103440000146402B03D094F81231012B3AD10823C6
:10345000ADF8063036E0D0F8E4350DF106019B6A90
:1034600080789847022343700146C4F8F00529E0AC
:10347000DBB2052B00F2DD80DFE803F003080D125C
:10348000171CD0F8EC3580785B6817E0D0F8EC3585
:1034900080789B6812E0D0F8EC358078DB680DE02E
:1034A000D0F8EC3580781B6908E0D0F8EC358078EE
:1034B0005B6903E0D0F8EC3580789B690DF106017B
:1034C00098470146BDF80630002B00F0B680EA8828
:1034D000002A00F0B2809A4228BF1A46ADF80620B2
:1034E00058E0AB88002B40F0A480EB88002B40F024
:1034F000A08090F812216B88032A00F09A8003F0D4
:103500007F0580F81451294600F05EFE2046FFF743
:103510009FFE0DB1022300E0012384F812318CE0FC
:10352000A978474E0129317100F2838090F8123159
:10353000022B02D0032B7CD108E0002963D00121AB
:10354000032380F8101180F8123111E039B90223F9
:1035500080F8123180F81011FFF704FD53E090F865
:103560001011012950D0FFF7FDFC317984F81011BA
:103570002046FFF7EBFC46E0EA88012A59D190F893
:103580001231022B02D0032B53D101E02D4913E05D
:1035900000F5887120460FE090F81231023B012BB4
:1035A00047D8274B0122DA60D0F818210AB103224C
:1035B000DA60254920460222FFF718FE3DE06B88BD
:1035C000012B2DD0022B38D1AB8813F0FF0F34D153
:1035D00002691B0A013B5268042B0FD8DFE803F095
:1035E000030507090B00012306E0022304E003237F
:1035F00002E0042300E0052363F30612134B1A6074
:10360000012384F816312046FFF722FE15E090F8DA
:103610001231023B012B0CD86B88012B0DD10023FA
:10362000C4F81831D4F8E43520469B6829469847F9
:10363000E9E720462946FFF751FE00207CBD00BF88
:10364000A44A0020AC4A0020B04A00200C590020B7
:1036500030B5C8B10023DDB20133C41814F8014CF1
:10366000002CF8D16B1C5B0013800B7003234B7094
:10367000022305E0CA545A1CD2B202338C54DBB286
:1036800010F8012B002AF5D130BD00BF37B500235B
:10369000104C054601930320F8F76AF8EB68013CEB
:1036A0001A69019213D0019A002AF4DA019A42F0C1
:1036B00001020192019A1A61064A1969013A0191BF
:1036C00002D00199C907F8D40320F8F751F8002077
:1036D0003EBD00BF410D030010B5C47874B900EBC6
:1036E000820003339B10D0F8D000224603E051F84B
:1036F000044C0132046004319A42F8D1002010BD1C
:10370000033230B59210D0F8D0400B46002003E0D1
:103710002568013043F8045C04339042F8D101EB92
:10372000800030BD0122F0B50023827040220129C3
:10373000C37082800CD108230370042343704FF4BC
:10374000A073C38002230372C1724FF0A04309E04B
:1037500041B90C230370062343704FF4A063C38068
:103760001F4BC17203F500620261C36046780446D4
:1037700001461A46002508E002F5106C02F5306299
:103780000A65C1F814C001353A460431B54202F168
:103790002007F1D303F58062426103F58862C0F827
:1037A000CC20067803F5A0650146002203E0C1F8AD
:1037B0008C50013220350431B242F8D31946002230
:1037C00002E0C4F8CC1001320434B24201F5805159
:1037D000F7D303F56063C0F80C310020F0BD00BFE3
:1037E0000000044038B5037A0025012B0446C26866
:1037F0001FD1936B417A65F3104309B143F48013F1
:103800009363D36820466FF386136FF396536FF379
:1038100051436FF3D343D360FFF738FFE378012BB5
:1038200019D1052363F34405E36845F020059D6045
:1038300011E0D36843F04003D360FFF727FF637ABA
:10384000E268002B0CBF4FF450234FF4E81393634E
:103850001420F7F797FFE378012B07D1E3680522DF
:103860009D6862F3440545F020059D60002038BD49
:10387000C36800209A6842F001029A607047C368EA
:1038800000209A6822F001029A60704707B5002371
:103890000193019B43F020030193019B61F38A1381
:1038A0000193019BC2681361064B1169013B0191B1
:1038B00002D001998806F8D40320F7F759FF0020B9
:1038C0000EBD00BF410D030007B500230193019B0E
:1038D00043F010030193019BC2681361064B116909
:1038E000013B019102D00199C906F8D40320F7F7F2
:1038F0003FFF00200EBD00BF410D030008B5C268A8
:103900000129D3686FF35D736FF39E7302D143F0A7
:10391000005302E009B943F080433220D360F7F747
:1039200031FF002008BDC368586900F001007047EE
:10393000C3685B6913F0010F14BF002001207047BA
:10394000C368586900F001007047C3685A699869F4
:1039500010407047C3685868704703691A6861F37C
:1039600001021A607047C268002393614FF0FF3173
:103970006FF080435361516053610C4B9361C37886
:103980009169002B14BF4FF400634FF4016343F0BF
:10399000804343F4701343F4405343F00C0321EA93
:1039A00003010B4393610020704700BF00080080B3
:1039B000F8B5D0F80C3100221A60036915461A6870
:1039C000044665F3CC221A60C37A012B21D103216E
:1039D000FFF7C3FFE36880214FF4001261F30F0289
:1039E00059629A62A02262F30F0561F31F454FF4FA
:1039F0009072C3F8045162F30F05C0F220054FF432
:103A0000A072C3F8085162F30F056FF31F45C3F8A6
:103A10000C5110212046FFF739FF2046FFF754FFD5
:103A2000226900234FF0FF311361204653611E4687
:103A30009161FF25D361214610E082690133176847
:103A40000430C7F3076707F08007FFB2002F14BFE9
:103A50004FF0904700271760166195606278934297
:103A6000EBD300231D46FF2010E04A6D013316689A
:103A70000431C6F3076606F08006F6B2002E14BFC6
:103A80004FF0904600261660156190606278934270
:103A9000EBD323691A6942F480721A61E278012A31
:103AA00004D1054A402161F359421A632046FFF7C9
:103AB0005AFF0020F8BD00BF0301010003699B68A5
:103AC000C3F34103013B022B9ABF024AD05C03209F
:103AD000704700BF3378010810B5036981699C689D
:103AE0000A68C4F34100022802D06FF30A0202E020
:103AF000032060F30A020A605A68002042F48072D0
:103B00005A6010BD30B54D780B780022012D00EBC6
:103B1000830405D105FA03F3A46963F30F0205E0FA
:103B2000012505FA03F3646D63F31F422368C3F3B1
:103B3000072505F08005EDB26DB98D6865F30A03C0
:103B4000CD78C98865F3934361F3995343F080536B
:103B500043F40043236003690020D9690A43DA6112
:103B600030BD30B54D780B780024012D224600EB96
:103B7000830105D105FA03F3896963F30F0205E0B8
:103B8000012505FA03F3496D63F31F4203696FF3DF
:103B9000CF340C60D969002021EA0202DA6130BD1D
:103BA000F8B54F780B78012F00EB830349D19E695C
:103BB0004C69356833692A4664F3120314B967F314
:103BC000DC430BE08F68E419013CB4FBF7F7CC78D9
:103BD00067F3DC43012C08BF64F35E733361C37881
:103BE000012B06D10B780C6900EB83039B695C61A8
:103BF0000CE0CB78012B09D04B693BB10C78012745
:103C000007FA04F403695E6B34435C63CB78012BE1
:103C100007D103699B68DB0554BF45F0005245F0AE
:103C200080520B7842F0044200EB83039B691A60D8
:103C3000CB78012B38D10A788B8AC968FFF74CFD05
:103C400032E05E6D4F6935688C682A4633692FB95A
:103C500064F31203012464F3DC430AE03F19013FDB
:103C6000B7FBF4F7BF05BF0D7C4367F3DC4364F398
:103C700012033361C378012B05D10B780C6900EB7B
:103C800083035B6D5C61CB78012B06D14B7913B15B
:103C900045F0005201E045F080520B7842F00442BA
:103CA00000EB8300436D1A600020F8BD73B54D78BA
:103CB000012D3DD183694A691E681C690094E4B2F4
:103CC00042B962F306048DF800409DF8024065F3A6
:103CD000C4040EE08D68AA4286BF4D6165F30604F8
:103CE00062F306048DF800409DF80240012262F361
:103CF000C4048DF80240009A1A61C278012A05D1E5
:103D00000A780C6900EB82029269546146F0044221
:103D10001A60C378002B34D14B69002B31D00A785C
:103D2000012101FA02F20369586B02435A6328E049
:103D30000B784E6900EB83035B6D8C681A681D6914
:103D40000095EDB206B14C6164F306059DF80240A2
:103D50008DF80050012565F3C4048DF80240009CE5
:103D60001C61C378012B05D10B780C6900EB830330
:103D70005B6D5C610B7842F0044200EB8300436DA5
:103D80001A6000207CBD4B78012B0B7800EB830080
:103D90000AD182691368C3F3076101F08001C9B2D7
:103DA00021B143F0804301E0426D136843F40013F6
:103DB0001360002070474B78012B0B78C97800EB1B
:103DC00083000CBF8269426D02391368C9B26FF378
:103DD0005553012998BF43F080531360002070476A
:103DE00003699A69D8691040000C704700EB8101A3
:103DF0004B6D02699B685069184070470369986968
:103E0000DB69184080B2704782B000230093C02362
:103E10008DF803300122002362F3C4038DF80230D1
:103E200018238DF80030009A436D1A61C278012A78
:103E300007D100F5B8600C3058611A684FF0802245
:103E40001A6002B07047D0F8183110B50446D3B1EB
:103E500003699A68D20716D5827A42B1D0F80C214C
:103E6000D0F80C116FF341026FF300020A605A6838
:103E7000052042F001025A60F7F784FC23695A6872
:103E800022F001025A6010BD837A63B103699B6816
:103E9000D90708D5D0F80C31D0F80C216FF34103C5
:103EA0006FF3000313607047012310B5002280F800
:103EB000123104460346FF2104E058690132816053
:103EC000186D8160607804338242F6D32369002242
:103ED0001A615A61DA614FF0FF329A612046FFF7AA
:103EE000F3FC20461021BDE81040CFE44B78012BB5
:103EF0000B7800EB83000FD183691868C0F307408B
:103F000000F02003DBB2CBB900F00200C0B2002801
:103F10000CBF302020207047436D1868C0F3074065
:103F200000F02003DBB25BB900F00200C0B2002851
:103F30000CBF4FF440504FF40050704710207047B2
:103F40004FF4805070474B7810B5012B0B7800EB85
:103F500083030AD19C69102A236802D1BDE810406E
:103F600011E7202A0CD0302A0FE05C6DB2F5805F9B
:103F7000236802D143F400131BE0B2F5005F02D1C5
:103F800043F0006315E0B2F5405F0FD1C3F3074281
:103F900002F02002D2B222B100234B71BDE81040E2
:103FA00009E743F0806343F0802302E00AB962F33B
:103FB000CF33236010BD00BFF8B50446FFF7B2FB56
:103FC0000122002384F8122184F814312827164690
:103FD0001946402510E007FB034080F81C31A0F88B
:103FE000223180F81D6180F81F11C0F82451C0F8FB
:103FF0002811C0F83011013362789342EBD30023CB
:1040000028261946402510E006FB034080F874334B
:10401000A0F87A3380F8751380F87713C0F87C53D2
:10402000C0F88013C0F88813013362789342EBD351
:104030002046FFF724FC2046FFF7D4FB0021204652
:10404000FFF75CFC2046FFF7B3FC2046BDE8F840D4
:10405000FFF70EBC70B5CDB20C464FF0280601F04C
:104060007F0106FB010115F0800F14BF01F58E7171
:1040700001F55D7104F07F04ED090C704D708A60EC
:10408000CB7005B1CC80022B01D100230B71FFF75F
:1040900039FD002070BD10B501F07F034FF02804FA
:1040A00004FB0303CAB212F0800F14BF03F58E7332
:1040B00003F55D7301F07F01D20919705A7019463A
:1040C000FFF74FFD002010BD38B501F07F05282413
:1040D00004FB050404F55D714B6100238B614B709B
:1040E000EBB2CA6084F87433C478012C08BF0A614B
:1040F00013B9FFF7DBFD01E0FFF752FD002038BDEB
:1041000070B501F07F04282505FB040505F58E71C7
:104110000126E4B2CA600A61002285F81C414E7093
:1041200005F58C758A614B6114B9FFF7BFFD01E09D
:10413000FFF736FD002070BDCAB212F0800F10B537
:104140004FF0280306D001F07F0403FB040303F5BE
:104150008E7303E003FB010303F55D73D2090124B1
:1041600001F07F0119709C705A701946FFF70BFE21
:10417000002010BDCAB212F0800F10B54FF0280316
:1041800006D001F07F0403FB040303F58E7303E004
:1041900003FB010303F55D730024D20901F07F01E5
:1041A00019709C705A701946FFF705FE204610BD25
:1041B00008B50B0604D501F07F01FFF767FB01E0AE
:1041C000FFF782FB002008BD0369002261F30A1299
:1041D00019680A431A607047036903205A686FF32D
:1041E00041025A60F7F7CEBA036903205A6842F0D9
:1041F00002025A60F7F7C6BA11F0800F4FF0280399
:1042000006D001F07F0103FB010101F58E7103E08F
:1042100003FB010101F55D71FFF768BE11F0800F2E
:104220004FF0280306D001F07F0103FB010101F5E7
:104230008E7103E003FB010101F55D71FFF783BEA1
:104240002DE9F04F85B00446FFF772FB002800F01F
:104250005D822046FFF779FB0546002800F0568274
:10426000C0F3074000F00800C0B200285AD0204632
:10427000FFF7B6FD27468246A1464FF00008DFF85B
:1042800068B32E4649E01AF0010F3FD05FFA88F27A
:10429000114620460092FFF7A9FD10F0010F0546D8
:1042A000009A20D07B6D01259D60E178A94207D15D
:1042B0001B69D9F87C13C3F31203CB1AC9F88C33EA
:1042C000DBF8003020461B6811469847E378012B45
:1042D00009D1B8F1000F06D194F81131052B02D1A4
:1042E0002046FFF791FD05F00203DBB213B17B6DB1
:1042F00002259D6005F00805EDB23DB1DBF8003008
:1043000020469B6898477B6D0820986008F101085B
:104310004FEA5A0A043709F12809BAF1000FB2D15D
:1043200035460120C5F3074303F00403DBB2002B3D
:1043300000F0A1802046FFF761FD274683464FF03D
:104340000008019591E01BF0010F00F089802369BE
:104350005FFA88F919695D6B04EB890225FA09F5A2
:104360009269ED019268EDB20D431540EA071CD544
:10437000012000FA08F15A6B054622EA01025A634D
:10438000BB69994A9860136820465B68494698471C
:10439000E378AB4209D1B8F1000F06D194F811319E
:1043A000042B02D12046FFF72FFD05F00803DBB2F6
:1043B00013B1BB6908259D6005F01003DBB213B192
:1043C000BB6910259D6005F04003DBB213B1BB69EA
:1043D00040259D6005F00203DBB213B1BB690225E5
:1043E0009D6025F07F0515F0FF0F39D0282505FBCE
:1043F000084505F58E75AB696A69C246C3EB020CC8
:10440000AB68A0469C4528BF9C460CF1030CBB69D9
:104410004FEA9C0C9B69664614E0AA681C1B9442F8
:1044200028BF1446A3B24046E9684A46FFF754F94C
:10443000EB68E61C1B19EB60AB69B6081C19AC6194
:10444000BB699B699BB2B34205D9AC696B699C425D
:1044500001D2002BE1D1BB69802544469D60D04646
:1044600008F101084FEA5B0B0437BBF1000F7FF442
:104470006AAF019D012005F00203DBB213B1E368CE
:1044800002225A61C5F3076303F08003DBB2CBB1AC
:10449000A37A43B1D4F80C31D4F80C216FF3410363
:1044A0006FF300031360236920465A6822F001026B
:1044B0005A604D4B1B689B699847E3684FF0004278
:1044C0005A610120C5F3072303F00803DBB2002B78
:1044D0002ED000238DF80F3094F8123120468DF83D
:1044E0000F30414B1B685B6998472369E2684FF4C2
:1044F00000619B685161A27ACAB1DB0717D594F8B5
:104500001501012813D19DF80F30032B10D1D4F8D9
:104510000C311A6842F001021A601A6842F0030274
:104520001A60324B1A6942F006021A6100E001205B
:1045300005F00803DBB243B12B4B20461B68DB6858
:104540009847E36808225A61012005F01003DBB2A6
:10455000002B34D0E36828269A6922F010029A6171
:104560001F6A07F00F0306FB0346C7F34343022B02
:1045700006F55D7602D0062B1BD10EE047F6F073F0
:104580003B40B3B1C7F30A172046F1683A46FFF73C
:10459000B7F8F368DB19F36008E004F5B8610C3193
:1045A00020460822FFF7ACF8C7F30A17B369DF19F2
:1045B000B761E36801209A6942F010029A61C5F37D
:1045C000072303F01003DBB2002B38D02369002649
:1045D0005A68314622F001025A602046FFF756F928
:1045E00023463246FF2108E0E000002000ED00E015
:1045F000586901328160186D8160607804338242AD
:10460000F6D3236901274FF0FF3267F30F069A6153
:1046100067F31F460B22DE615A611A611A68204651
:104620006FF30A121A60FFF7EFFBE3684FF4805252
:104630005A61384B20461B681B6998473846C5F3BA
:10464000072303F02003DBB2EBB12046FFF744FA67
:10465000E3682046DE68FFF731FA032806D100231D
:10466000A3704FF40073A380092304E00123A37017
:104670004023A380052363F38D26E3684FF40052A3
:10468000DE6001205A61C5F3074303F01003DBB27B
:104690004BB1204B20461B68DB699847E3684FF419
:1046A00080125A610120C5F3074303F02003DBB2F7
:1046B0004BB1184B20461B681B6A9847E3684FF4C0
:1046C00000125A610120C5F3076303F04003DBB217
:1046D0004BB1104B20461B685B6A9847E3684FF06C
:1046E00080425A61012005F00405EDB275B1E3681E
:1046F0005D6805F00403DBB223B1064B20461B685E
:104700009B6A9847E36801205D60FFE705B0BDE85C
:10471000F08F00BFE000002081F0004102E000BF08
:1047200083F0004330B54FEA41044FEA430594EA71
:10473000050F08BF90EA020F1FBF54EA000C55EAAC
:10474000020C7FEA645C7FEA655C00F0E2804FEA7D
:104750005454D4EB5555B8BF6D420CDD2C4480EA5F
:10476000020281EA030382EA000083EA010180EA8F
:10477000020281EA0303362D88BF30BD11F0004FDD
:104780004FEA01314FF4801C4CEA113102D0404213
:1047900061EB410113F0004F4FEA03334CEA13334E
:1047A00002D0524263EB430394EA050F00F0A78066
:1047B000A4F10104D5F1200E0DDB02FA0EFC22FA61
:1047C00005F2801841F1000103FA0EF2801843FA55
:1047D00005F359410EE0A5F120050EF1200E012A46
:1047E00003FA0EFC28BF4CF0020C43FA05F3C01884
:1047F00051EBE37101F0004507D54FF0000EDCF1FD
:10480000000C7EEB00006EEB0101B1F5801F1BD3A5
:10481000B1F5001F0CD349085FEA30004FEA3C0CA9
:1048200004F101044FEA445212F5800F80F09A809F
:10483000BCF1004F08BF5FEA500C50F1000041EBA3
:10484000045141EA050130BD5FEA4C0C404141EBA7
:10485000010111F4801FA4F10104E9D191F0000FCE
:1048600004BF01460020B1FA81F308BF2033A3F151
:104870000B03B3F120020CDA0C3208DD02F1140C48
:10488000C2F10C0201FA0CF021FA02F10CE002F183
:104890001402D8BFC2F1200C01FA02F120FA0CFC7C
:1048A000DCBF41EA0C019040E41AA2BF01EB0451C5
:1048B000294330BD6FEA04041F3C1CDA0C340EDCC3
:1048C00004F11404C4F1200220FA04F001FA02F306
:1048D00040EA030021FA04F345EA030130BDC4F1C4
:1048E0000C04C4F1200220FA02F001FA04F340EAB9
:1048F0000300294630BD21FA04F0294630BD94F06A
:10490000000F83F4801306BF81F480110134013D50
:104910004EE77FEA645C18BF7FEA655C29D094EAC1
:10492000050F08BF90EA020F05D054EA000C04BF3F
:104930001946104630BD91EA030F1EBF002100202A
:1049400030BD5FEA545C05D14000494128BF41F0C9
:10495000004130BD14F580043CBF01F5801130BD2D
:1049600001F0004545F0FE4141F470014FF00000B8
:1049700030BD7FEA645C1ABF194610467FEA655C69
:104980001CBF0B46024650EA013406BF52EA03350B
:1049900091EA030F41F4002130BD00BF90F0000FF9
:1049A00004BF0021704730B54FF4806404F1320435
:1049B0004FF000054FF0000150E700BF90F0000FEE
:1049C00004BF0021704730B54FF4806404F1320415
:1049D00010F0004548BF40424FF000013EE700BFE5
:1049E00042004FEAE2014FEA31014FEA02701FBF75
:1049F00012F07F4393F07F4F81F06051704792F047
:104A0000000F14BF93F07F4F704730B54FF46074C0
:104A100001F0004521F0004120E700BF50EA01020B
:104A200008BF704730B54FF000050AE050EA0102B8
:104A300008BF704730B511F0004502D5404261EB28
:104A400041014FF4806404F132045FEA915C3FF469
:104A5000DCAE4FF003025FEADC0C18BF03325FEA02
:104A6000DC0C18BF033202EBDC02C2F1200300FAB7
:104A700003FC20FA02F001FA03FE40EA0E0021FADC
:104A800002F11444C1E600BF70B54FF0FF0C4CF4C6
:104A9000E06C1CEA11541DBF1CEA135594EA0C0F7C
:104AA00095EA0C0F00F0DEF82C4481EA030621EAB7
:104AB0004C5123EA4C5350EA013518BF52EA0335F2
:104AC00041F4801143F4801338D0A0FB02CE4FF0A4
:104AD0000005E1FB02E506F00042E0FB03E54FF0D4
:104AE0000006E1FB03569CF0000F18BF4EF0010ECC
:104AF000A4F1FF04B6F5007F64F5407404D25FEAC8
:104B00004E0E6D4146EB060642EAC62141EA55517A
:104B10004FEAC52040EA5E504FEACE2EB4F1FD0CBC
:104B200088BFBCF5E06F1ED8BEF1004F08BF5FEA3A
:104B3000500E50F1000041EB045170BD06F00046EC
:104B400046EA010140EA020081EA0301B4EB5C0499
:104B5000C2BFD4EB0C0541EA045170BD41F4801191
:104B60004FF0000E013C00F3AB8014F1360FDEBFB6
:104B7000002001F0004170BDC4F10004203C35DA92
:104B80000C341BDC04F11404C4F1200500FA05F315
:104B900020FA04F001FA05F240EA020001F00042B6
:104BA00021F0004110EBD37021FA04F642EB06012C
:104BB0005EEA430E08BF20EAD37070BDC4F10C0456
:104BC000C4F1200500FA04F320FA05F001FA04F21A
:104BD00040EA020001F0004110EBD37041F1000106
:104BE0005EEA430E08BF20EAD37070BDC4F1200511
:104BF00000FA05F24EEA020E20FA04F301FA05F279
:104C000043EA020321FA04F001F0004121FA04F220
:104C100020EA020000EBD3705EEA430E08BF20EAF0
:104C2000D37070BD94F0000F0FD101F0004640002A
:104C300041EB010111F4801F08BF013CF7D041EAAC
:104C4000060195F0000F18BF704703F000465200B0
:104C500043EB030313F4801F08BF013DF7D043EA81
:104C60000603704794EA0C0F0CEA135518BF95EA37
:104C70000C0F0CD050EA410618BF52EA4306D1D1BE
:104C800081EA030101F000414FF0000070BD50EADD
:104C9000410606BF1046194652EA430619D094EA67
:104CA0000C0F02D150EA013613D195EA0C0F05D151
:104CB00052EA03361CBF104619460AD181EA0301A5
:104CC00001F0004141F0FE4141F470014FF000005D
:104CD00070BD41F0FE4141F4780170BD70B54FF0F8
:104CE000FF0C4CF4E06C1CEA11541DBF1CEA135578
:104CF00094EA0C0F95EA0C0F00F0A7F8A4EB05045A
:104D000081EA030E52EA03354FEA013100F0888050
:104D10004FEA03334FF0805545EA131343EA126319
:104D20004FEA022245EA111545EA10654FEA0026CE
:104D30000EF000419D4208BF964244F1FD0404F587
:104D4000407402D25B084FEA3202B61A65EB0305E3
:104D50005B084FEA32024FF480104FF4002CB6EBA0
:104D6000020E75EB030E22BFB61A754640EA0C0020
:104D70005B084FEA3202B6EB020E75EB030E22BF60
:104D8000B61A754640EA5C005B084FEA3202B6EBA1
:104D9000020E75EB030E22BFB61A754640EA9C0060
:104DA0005B084FEA3202B6EB020E75EB030E22BF30
:104DB000B61A754640EADC0055EA060E18D04FEAEE
:104DC000051545EA16754FEA06164FEAC30343EA8E
:104DD00052734FEAC2025FEA1C1CC0D111F4801F5B
:104DE0000BD141EA00014FF000004FF0004CB6E754
:104DF00011F4801F04BF01430020B4F1FD0C88BFF3
:104E0000BCF5E06F3FF6AFAEB5EB030C04BFB6EBFD
:104E1000020C5FEA500C50F1000041EB045170BDF0
:104E20000EF0004E4EEA113114EB5C04C2BFD4EB1D
:104E30000C0541EA045170BD41F480114FF0000EA1
:104E4000013C90E645EA060E8DE60CEA135594EA1D
:104E50000C0F08BF95EA0C0F3FF43BAF94EA0C0F20
:104E60000AD150EA01347FF434AF95EA0C0F7FF495
:104E700025AF104619462CE795EA0C0F06D152EAE9
:104E800003353FF4FDAE1046194622E750EA4106CD
:104E900018BF52EA43067FF4C5AE50EA41047FF4DE
:104EA0000DAF52EA43057FF4EBAE12E74FF0FF3C43
:104EB00006E000BF4FF0010C02E000BF4FF0010C14
:104EC0004DF804CD4FEA410C7FEA6C5C4FEA430C8D
:104ED00018BF7FEA6C5C1BD001B050EA410C0CBFDC
:104EE00052EA430C91EA030F02BF90EA020F00203E
:104EF000704710F1000F91EA030F58BF994208BFA5
:104F000090422CBFD8176FEAE37040F00100704761
:104F10004FEA410C7FEA6C5C02D150EA013C07D1B8
:104F20004FEA430C7FEA6C5CD6D152EA033CD3D003
:104F30005DF8040B704700BF8446104662468C46FD
:104F40001946634600E000BF01B5FFF7B7FF002830
:104F500048BF10F1000F01BD4DF808EDFFF7F4FF59
:104F60000CBF012000205DF808FB00BF4DF808EDE4
:104F7000FFF7EAFF34BF012000205DF808FB00BF07
:104F80004DF808EDFFF7E0FF94BF012000205DF829
:104F900008FB00BF4DF808EDFFF7CEFF94BF0120DE
:104FA00000205DF808FB00BF4DF808EDFFF7C4FFD7
:104FB00034BF012000205DF808FB00BF4FEA41022A
:104FC00012F5001215D211D56FF47873B3EB62525B
:104FD00012D94FEAC12343F0004343EA505311F082
:104FE000004F23FA02F018BF404270474FF0000014
:104FF000704750EA013005D111F0004008BF6FF052
:10500000004070474FF00000704700BF4FEA410278
:10501000B2F1E04324BFB3F5001CDCF1FE5C0DD916
:1050200001F0004C4FEAC0024CEA5070B2F1004F60
:1050300040EB830008BF20F00100704711F0804F63
:1050400021D113F13872BCBF01F00040704741F428
:1050500080114FEA5252C2F11802C2F1200C10FA2C
:105060000CF320FA02F018BF40F001004FEAC12310
:105070004FEAD32303FA0CFC40EA0C0023FA02F3B4
:105080004FEA4303CCE77FEA625307D150EA01338A
:105090001EBF4FF0FE4040F44000704701F000405A
:1050A00040F0FE4040F40000704700BF80F0004038
:1050B00002E000BF81F0004142001FBF5FEA4103F0
:1050C00092EA030F7FEA226C7FEA236C6AD04FEAF0
:1050D0001262D2EB1363C1BFD21841404840414035
:1050E000B8BF5B42192B88BF704710F0004F40F4E7
:1050F000000020F07F4018BF404211F0004F41F403
:10510000000121F07F4118BF494292EA030F3FD0CE
:10511000A2F1010241FA03FC10EB0C00C3F12003E1
:1051200001FA03F100F0004302D5494260EB400070
:10513000B0F5000F13D3B0F1807F06D340084FEADB
:10514000310102F10102FE2A51D2B1F1004F40EBD0
:10515000C25008BF20F0010040EA03007047490038
:1051600040EB000010F4000FA2F10102EDD1B0FA03
:1051700080FCACF1080CB2EB0C0200FA0CF0AABFF8
:1051800000EBC25052421843BCBFD0401843704796
:1051900092F0000F81F4000106BF80F4000001329C
:1051A000013BB5E74FEA41037FEA226C18BF7FEA73
:1051B000236C21D092EA030F04D092F0000F08BFB5
:1051C0000846704790EA010F1CBF0020704712F09C
:1051D0007F4F04D1400028BF40F00040704712F1DB
:1051E00000723CBF00F50000704700F0004343F040
:1051F000FE4040F4000070477FEA226216BF084676
:105200007FEA23630146420206BF5FEA412390EA38
:10521000010F40F4800070474FF0000304E000BF2E
:1052200010F0004348BF40425FEA000C08BF7047DF
:1052300043F0964301464FF000001CE050EA0102A3
:1052400008BF70474FF000030AE000BF50EA0102B8
:1052500008BF704711F0004302D5404261EB4101A5
:105260005FEA010C02BF84460146002043F0B643CA
:1052700008BFA3F18053A3F50003BCFA8CF2083AEF
:10528000A3EBC25310DB01FA02FC634400FA02FCF8
:10529000C2F12002BCF1004F20FA02F243EB0200FF
:1052A00008BF20F00100704702F1200201FA02FC61
:1052B000C2F1200250EA4C0021FA02F243EB020054
:1052C00008BF20EADC7070474FF0FF0C1CEAD05298
:1052D0001EBF1CEAD15392EA0C0F93EA0C0F6FD059
:1052E0001A4480EA010C400218BF5FEA41211ED037
:1052F0004FF0006343EA501043EA5111A0FB013123
:105300000CF00040B1F5000F3EBF490041EAD371F7
:105310005B0040EA010062F17F02FD2A1DD8B3F173
:10532000004F40EBC25008BF20F00100704790F0E2
:10533000000F0CF0004C08BF49024CEA502040EA34
:1053400051207F3AC2BFD2F1FF0340EAC2507047FA
:1053500040F400004FF00003013A5DDC12F1190F38
:10536000DCBF00F000407047C2F10002410021FAAA
:1053700002F1C2F1200200FA02FC5FEA310040F1C2
:10538000000053EA4C0308BF20EADC70704792F03B
:10539000000F00F0004C02BF400010F4000F013A73
:1053A000F9D040EA0C0093F0000F01F0004C02BF6E
:1053B000490011F4000F013BF9D041EA0C018FE7DD
:1053C0000CEAD15392EA0C0F18BF93EA0C0F0AD0E3
:1053D00030F0004C18BF31F0004CD8D180EA010009
:1053E00000F00040704790F0000F17BF90F0004FA2
:1053F000084691F0000F91F0004F14D092EA0C0F84
:1054000001D142020FD193EA0C0F03D14B0218BF16
:10541000084608D180EA010000F0004040F0FE405C
:1054200040F40000704740F0FE4040F440007047F8
:105430004FF0FF0C1CEAD0521EBF1CEAD15392EA77
:105440000C0F93EA0C0F69D0A2EB030280EA010C67
:1054500049024FEA402037D04FF0805343EA111100
:1054600043EA10130CF000408B4238BF5B0042F15E
:105470007D024FF4000C8B4224BF5B1A40EA0C0003
:10548000B3EB510F24BFA3EB510340EA5C00B3EB35
:10549000910F24BFA3EB910340EA9C00B3EBD10F23
:1054A00024BFA3EBD10340EADC001B0118BF5FEA75
:1054B0001C1CE0D1FD2A3FF650AF8B4240EBC2509E
:1054C00008BF20F0010070470CF0004C4CEA50205F
:1054D0007F32C2BFD2F1FF0340EAC250704740F4AE
:1054E00000004FF00003013A37E792F0000F00F0A0
:1054F000004C02BF400010F4000F013AF9D040EA1E
:105500000C0093F0000F01F0004C02BF490011F4B1
:10551000000F013BF9D041EA0C0195E70CEAD153A9
:1055200092EA0C0F08D142027FF47DAF93EA0C0F90
:105530007FF470AF084676E793EA0C0F04D14B0274
:105540003FF44CAF08466EE730F0004C18BF31F026
:10555000004CCAD130F000427FF45CAF31F0004320
:105560007FF43CAF5FE700BF4FF0FF3C06E000BFB9
:105570004FF0010C02E000BF4FF0010C4DF804CDDC
:105580004FEA40024FEA41037FEA226C18BF7FEAEC
:10559000236C11D001B052EA530C18BF90EA010FEE
:1055A00058BFB2EB030088BFC81738BF6FEAE1707D
:1055B00018BF40F0010070477FEA226C02D15FEA19
:1055C000402C05D17FEA236CE4D15FEA412CE1D085
:1055D0005DF8040B704700BF844608466146FFE74C
:1055E0000FB5FFF7C9FF002848BF10F1000F0FBD2E
:1055F0004DF808EDFFF7F4FF0CBF012000205DF827
:1056000008FB00BF4DF808EDFFF7EAFF34BF0120AB
:1056100000205DF808FB00BF4DF808EDFFF7E0FF44
:1056200094BF012000205DF808FB00BF4DF808ED95
:10563000FFF7D2FF94BF012000205DF808FB00BFF8
:105640004DF808EDFFF7C8FF34BF012000205DF8DA
:1056500008FB00BF42000ED2B2F1FE4F0BD34FF059
:105660009E03B3EB126209D44FEA002343F00043D8
:1056700023FA02F070474FF00000704712F1610FFB
:1056800001D1420202D14FF0FF3070474FF00000CD
:10569000704700BF73B96AB9002908BF0028BCBFB2
:1056A00000204FF00041C4BF6FF000414FF0FF30C9
:1056B00001F072B882B0EC462DE9005000F006F817
:1056C000DDF804E002B00CBC704700BF2DE9704368
:1056D0001546804689461C4601F060F805FB01F638
:1056E000A5FB002300FB0464E318069CB8EB020250
:1056F00069EB0303C4E90023BDE87083F8B51446E1
:1057000006460F461D4601F0ADF900FB05F5A0FB6E
:10571000042304FB0154E318069CB21A67EB03034D
:10572000C4E90023F8BD00BF036803B11B18184685
:10573000704700BF03685A004CBF43F0004323F09A
:105740000043C018704700BF2DE9F84F044691464A
:1057500041B301F1FF3BDA46002707EB0A0000EBFB
:10576000D0756D1004EBC5063046FFF7E3FFAB457F
:10577000804610D0691C04EBC100FFF7DBFF013845
:10578000C84504D9BD4209D005F1FF3AE5E74845CF
:1057900005D26F1CE1E74FF0FF30F1E700263046FD
:1057A000BDE8F88F0E463046BDE8F88F30B52B4B7C
:1057B00083B004468D1E002B49D0284601A9AFF3C3
:1057C00000800346002822D02A4618460199FFF798
:1057D000BBFF054600281DD0FFF7ACFF6B68A06437
:1057E000012B10D0281D002B22DBFFF7A3FF002187
:1057F000E06421650368002B0FDBFFF79BFF20614E
:10580000002003B030BD002323610520F9E72061AB
:105810000920F6E720610920F3E7C3F3036058B1DC
:1058200001280CD002280ED0002020610920E8E7D2
:105830000122E0642265DDE7094B2361E1E7094AC3
:1058400000202261DDE7084900202161D9E7074AED
:1058500007491346881AC2100192B5E700000000FC
:10586000715D01086D5D0108695D01080C7A010830
:10587000F47A0108036810B50446D80706D49907DE
:1058800004F1480009D500F009FD23685A0709D53D
:1058900018070ED5D90613D510BD00F0F7FC236804
:1058A0005A07F5D404F1D00000F000FD2368180772
:1058B000F0D404F5D87000F001FD2368D906EBD4CC
:1058C00004F50C70BDE8104000F03CBD2DE9F04738
:1058D000ADF5916D02AC0F1D261D054691460FCF0B
:1058E0000FC60FCF0FC60FCF0FC697E80F00D5F822
:1058F0000C800027D5F818A086E80F00216C2846F8
:105900002760FFF753FF0646B94514BF4FF00A0959
:105910004FF00909FEB1A16B49F010096164012043
:105920008DE8100449462A462B46C04700282BD153
:10593000002E2AD1204692A94FF4107201F052FE97
:10594000082F28D1216C2846FFF730FF06464FF07C
:105950000909002EDFD1206C21464FF410726861D6
:1059600092A801F03FFE2F69294692AA4846B847FF
:10597000A09B0746636401208DE8100449462A462F
:105980002B46C0470028D3D00926304622B00DF55B
:10599000806DBDE8F087072FF6D1201D00F06AFC6E
:1059A00038B504460D46296C2046FFF7FFFE50B976
:1059B0002A6C01206261236921462A4698470828FB
:1059C000F1D0072801D001F005FE281D00F052FC9F
:1059D00011B933B10220704704298CBF0220012085
:1059E00070470F2A01D90220704700EB82004268FD
:1059F0001846009B1A60704710B50A4684B0002113
:105A00000B4603AC0094FFF7E3FF039804B010BD0E
:105A100011B933B10220704704298CBF0220012044
:105A200070470F2A01D902207047009900EB8202CB
:105A3000096818465160704700B585B004AB43F85B
:105A4000042D0A46002100930B46FFF7E1FF05B045
:105A500000BD00BF2DE9F04FCD6C0C4655F8041B7E
:105A60008BB0174600F008021E46039200F00308B0
:105A70000795002B40F0E08009020691216D8DF81A
:105A800021300323B8F1020F8DF8203008BFA56B39
:105A900011F0010340F0E480019304F158030293F4
:105AA000D5F80090B9F1000F00F0DC80022E00F074
:105AB000BF80B5F80090B5F802A00435A26C0F21A4
:105AC0002AF0010B38469344FFF796FF834518D818
:105AD00029F0010CE3440AF0010A09F001035845DA
:105AE00043EA4A092CBF00200120B9F1010F12D06E
:105AF00032D2B8F1000F02D0002840F017810435EF
:105B0000CEE70AF0010A09F0010343EA4A0900203E
:105B1000B9F1010FECD1B8F1000F40F0C880C8B165
:105B20006B68D5F800909A1C19D0029A013309923B
:105B30000DD0281DFFF7F8FD4FEAD972014609ABD9
:105B40002046AFF30080002800F0EC80099A002A7C
:105B500040F0CC800835A3E7B9F1020F03D009204B
:105B60000BB0BDE8F08F2B6823F000420092B8F133
:105B7000000F40F08380002853D00398002840F0A5
:105B8000B2800098002800F0B180009B05F1040A63
:105B9000DB07DDF80C9010D4029950460991FFF70D
:105BA000C3FD039A014609AB2046AFF300800028ED
:105BB00033D10AF1040A4FF00109CDF81080AB4649
:105BC000B84650460596029F11E000998E4200F0BB
:105BD000C0800997FFF7A8FD5246014609AB204651
:105BE000AFF30080B14698B9281D06F10109051DE3
:105BF0000997FFF799FD09AB014600222046AFF354
:105C00000080824609F101062846BAF1000FDCD077
:105C10004746059EDDF810805D46009A4A4565D0EE
:105C20002B68002B7CDB0099481C05EB800537E7CF
:105C3000D5F804A0083541E70B04C1F30740216DF6
:105C40000222B8F1020F069305EB800508BFA56B91
:105C500011F001038DF821008DF820203FF41CAFD6
:105C600000200190384606A900F004FC00287FF4CB
:105C700076AF019A002A43D1082071E70D213846FA
:105C8000D4F82090FFF7B8FE8145C9D1A26A9542A9
:105C9000C6D10098291D00220423A062E26223637A
:105CA00061632868002857DB01220192BBE70D21C0
:105CB0003846D4F82090FFF79FFE81457FF44AAF25
:105CC000A16A8D427FF446AF2846FFF733FD0F21CE
:105CD00002463846FFF7B0FE384600212246FFF75D
:105CE000ABFE07203CE7009900299AD138460D21E8
:105CF000FFF782FE099B20626362A56206202FE700
:105D00000F213846FFF778FE0E2102463846FFF78E
:105D100093FE38460F21134AFFF78EFE07201FE738
:105D2000043580E7CDF824800835B9E62846FFF72A
:105D300001FD04350646A5632046AFF30080002828
:105D40003FF40DAF38460F213246FFF775FE0720AE
:105D500006E75D464746C9E7009B591C05EB8100F5
:105D6000B3E700BF00000000022373E6012371E6E1
:105D700000236FE62DE9F0470446E8B004290CD86B
:105D8000DFE801F0390392940F00150C012B96B255
:105D900000F07881052B00F0C880022068B0BDE8D3
:105DA000F087002BF9D1102AF7D82368D90600F123
:105DB000738164A8019200F0CFFA019AA36BD00717
:105DC00044BF53F8040B6490910744BF53F8041B7D
:105DD0006591500748BF53F8041B64A848BF6691FB
:105DE000110748BF53F8042BA36348BF679200F024
:105DF000A9FA0020D2E7002BCFD1A36BD00791B234
:105E000044BF53F8042B62608A0744BF53F8042B45
:105E1000A260480744BF53F8042BE2600A0744BF5E
:105E200053F8042B2261C80644BF53F8042B626167
:105E30008A0644BF53F8042BA261480644BF53F8B6
:105E4000042BE2610A0644BF53F8042B2262C80502
:105E500044BF53F8042B62628A0544BF53F8042BF5
:105E6000A262480544BF53F8042BE2620A0544BF0E
:105E700053F8042B2263C80444BF53F8042B626315
:105E800011F400501CBF53F8042BA2634A0444BF12
:105E900053F8042BE2630A0444BF53F8042B226432
:105EA000002840D1A36379E7012077E7032B7FF433
:105EB00074AF160C95B2AA19102A3FF66EAF23687C
:105EC000180700F10A8144A800F01AFAA76B4FEAFC
:105ED000450E3B460DB30EF1FF3C44A953F8040BAD
:105EE00001EBC60662460CF0010146F8040B92B1C4
:105EF00029B153F8041B013A46F8041B0BD018468D
:105F000050F8045B314641F8045B5D68031D756021
:105F10000E1D023AF3D107EB8E0344A8A36300F0F1
:105F2000CDF900203AE7002038E777192022BA425D
:105F3000FFF433AF012B00F0A8800F2D40F2A880B2
:105F40003746F6B1052B7FF428AF0F2D11D8226804
:105F5000D0070ED522F00101052B216000F0DA8078
:105F600022F00302204640F8482B019300F092F9FA
:105F7000019B1FB12268510700F1B780012B00F08F
:105F8000BE800F2D74D9002F40F09F80D4F8389038
:105F9000002EC8462EDD49464FEA46080DF1080C92
:105FA00051F8046B0CEBC50208F1FF3000F0010A58
:105FB00042F8046BA8F1020CD0B1BAF1000F08D07E
:105FC00051F8040B0CF1FF3CBCF1FF3F42F8040B0D
:105FD0000ED00E4656F804AB104640F804AB4968A4
:105FE000ACF1020C5160311D021DBCF1FF3FF0D13C
:105FF00009EB88089FB3102D2CBF2E46102668AAE7
:10600000414602EBC60A4FEA470951F8046BAAF56C
:10601000C87209F1FF3000F0010A42F8046BA9F1DF
:10602000020CD0B1BAF1000F08D051F8040B0CF1FA
:10603000FF3CBCF1FF3F42F8040B0ED00E4656F871
:1060400004AB104640F804AB4968ACF1020C516057
:10605000311D021DBCF1FF3FF0D108EB8908012B77
:106060002BD00F2DC4F8388008D9FFB9384695E6F3
:1060700002A8019300F016F9019B84E702A800F042
:106080000DF9F2E77719102251E70F2D3FF685AE93
:10609000102F10D9103F55E723F01003236004F5AB
:1060A0000C70019200F058F9019A82E624A800F0E1
:1060B000FDF8002072E6002747E708F1040302A874
:1060C000A36300F0E3F8002068E624A80193C5F17B
:1060D000100600F0EFF8019B58E723F0080704F5DD
:1060E000D870276000F00CF9EDE622F0040120469C
:1060F00040F8D01B019300F0DDF8019B3EE702A8B9
:10610000019300F0C7F8019B002F3FF43FAFC5F1AA
:1061100010063BE741F00201204640F8481B01937E
:1061200000F0C0F8019B24E7406C7047F0B50D46C5
:10613000C96BADF5117D296401AE2F1D04460FCF4B
:106140000FC60FCF0FC60FCF0FC697E80F0086E818
:106150000F004FF0FF33009310992046FFF726FB06
:1061600058B9266921466A46B04708280646F3D042
:106170006846FFF77FFB062E03D009200DF5117D41
:10618000F0BD20462946FFF70BFC00BF10B4DC6BC6
:10619000C1608261194600221C6410BCFFF796BBE7
:1061A00038B54269C36804460D460A6423B101222A
:1061B000FFF78CFB01F00EFA0369214602202A4604
:1061C0009847072803D0082804D001F003FA281DB7
:1061D00000F050F820462946FFF7E2FBC36823B1E0
:1061E000CA6B0A640022FFF771BB9FE7704700BFCC
:1061F00008B5836801460BB10120984708BD00BF70
:10620000F0B5D46BADF5277D146401AE171D0546BE
:106210000C460FCF0FC60FCF0FC60FCF0FC697E894
:106220000F0086E80F004FF0FF330093109990A8FD
:10623000FFF7BCFA034690AA68460C21BBB9FFF7EA
:10624000FBFB21466846A847064690A908206A46F7
:106250006EB9949B98470528064601D00928E5D1D8
:106260006846FFF707FB30460DF5277DF0BD092690
:10627000F6E700BF00F1340191E838009C46A646DD
:106280004CF8045D90E8FF0FE54600BD90EC210B53
:10629000704700BF80EC210B704700BF90EC200BD3
:1062A000704700BF80EC200B704700BFD0EC200B84
:1062B000704700BFC0EC200B704700BFF0EC02013C
:1062C000F0EC0211F0EC0221F0EC0231F0EC0241B2
:1062D000F0EC0251F0EC0261F0EC0271F0EC0281A2
:1062E000F0EC0291F0EC02A1F0EC02B1F0EC02C192
:1062F000F0EC02D1F0EC02E1F0EC02F1704700BFEB
:10630000E0EC0201E0EC0211E0EC0221E0EC0231F1
:10631000E0EC0241E0EC0251E0EC0261E0EC0271E1
:10632000E0EC0281E0EC0291E0EC02A1E0EC02B1D1
:10633000E0EC02C1E0EC02D1E0EC02E1E0EC02F1C1
:10634000704700BFB0FC0181B0FC0191B0FC01A11D
:10635000B0FC01B1704700BFA0FC0181A0FC01911D
:10636000A0FC01A1A0FC01B1704700BFEC4600B544
:106370002DE900502DE9FF1F4FF000032DE90C001F
:1063800001A9FFF7D3FEDDF840E012B0704700BF6F
:10639000EC4600B52DE900502DE9FF1F4FF000033A
:1063A0002DE90C0001A9FFF7FBFEDDF840E012B07B
:1063B000704700BFEC4600B52DE900502DE9FF1FE6
:1063C0004FF000032DE90C0001A9FFF707FFDDF8EE
:1063D00040E012B0704700BFEC4600B52DE9005018
:1063E0002DE9FF1F4FF000032DE90C0001ABFFF773
:1063F000CDFEDDF840E012B0704700BFEC4600B5BE
:106400002DE900502DE9FF1F4FF000032DE90C008E
:1064100001AAFFF7F5FEDDF840E012B0704700BFBB
:10642000027A03461AB9427A42B9B020704700682E
:10643000013A01021A72000E196070474168501E3D
:10644000587251F8040B0322596001021A72000EAF
:106450001960704710B5002184B00C220DEB0204C6
:106460000B460094FFF7B4FA039804B010BD00BFC8
:10647000F0E700BF2DE9F043064685B00D464FF02A
:1064800000094FF47F672846FFF7CAFFB02804468B
:1064900000F0B18010F0800120D000F0F003802BDC
:1064A00075D0902B37D0A02B45D0B02B56D0C02B19
:1064B00000F0868000F0F800D0280BD104F007032C
:1064C0005A1C42F40022304601210523FFF752FCFA
:1064D0000028D8D0092005B0BDE8F0834FEA80023B
:1064E00003A85FFA82F800900D220B463046FFF7B2
:1064F0006FFA039B600608F104084CBFC8EB030366
:10650000434403AC03930094002130460D220B4614
:10651000FFF77EFAB7E700F00F020D2ADAD00F2A54
:10652000D8D0002103AC009430460B4603ACFFF7F3
:106530004FFA0094E8E7C24302F0070C47FA0CF068
:10654000210700F47F6248BF42F4804200213046B8
:106550000B46FFF70FFC0028BCD194E7B1285ED0B2
:10656000B2286FD0B32800F0968000F0FC0CBCF18C
:10657000B40F46D000F007014A1C42F4002201216A
:1065800030460B46FFF7F6FB0028A3D17BE72846F1
:10659000FFF746FF210240EA0104B4F5004F99D00D
:1065A000230500211A0C30460B462401FFF7E2FBBD
:1065B00000288FD114F4004F18BF4FF0010962E793
:1065C000C62873D0C72800F0848000F0F801C029E5
:1065D00000F09280C82800F0A680C9287FF47AAF26
:1065E0002846FFF71DFF00F00F0100F0F0024B1CE2
:1065F00043EA023267E7B9F1000F00F08380002020
:1066000069E700F00300431C022143F48022304676
:106610000B46FFF7AFFB00287FF45CAF33E728465B
:10662000FFF7FEFE024600283FF454AF10F0F001E1
:106630007FF450AF30460B46FFF79CFB00287FF4F9
:1066400049AF20E700210D220B4603AC30460094F1
:10665000FFF7BEF92846FFF7E3FE022402060DD538
:1066600000F07F0000FA04FE039B284603EB0E01B6
:106670000391FFF7D5FE07340306F1D400F07F0E37
:106680000EFA04F4039903AB01F5017C0CEB040250
:106690000093039238E72846FFF7C2FE00F00F018F
:1066A0004A1C00F0F00042EA003268E72846FFF793
:1066B000B7FE00F00F02531C00F0F00043EA003276
:1066C000032130460B46FFF755FB00287FF402AF4D
:1066D000D9E62846FFF7A4FE024600283FF4FAAEAA
:1066E00010F0F0037FF4F6AE30460421FFF742FBD2
:1066F00000287FF4EFAEC6E600F00F03581C40F40C
:106700002022DDE703AC49460E224B46304600947A
:10671000FFF75EF9304649460F224B460094FFF7DB
:1067200077F94846D7E62846FFF77AFE00F0F002F0
:1067300000F00F001032411C41EA0232C3E600BFF4
:1067400010B5C26C84B0032054688DF80C00D37966
:1067500024020832084601A9019402928DF80D30F6
:10676000FFF788FE04B010BD08B5FFF781FE806C0E
:1067700008BD00BF08B5FFF77BFEC16CC87901EB0F
:10678000800303F1080008BD08B500F023FF00BF37
:1067900008B500F01FFF00BF704700BF2DE9F00FE4
:1067A00000291D46C0F29D800024002DC0F2948077
:1067B00007460D4616469C46002B3DD18A4253D9CA
:1067C000B2FA82F343B1C3F1200620FA06F501FACA
:1067D00003F19A4098402943130CB1FBF3F697B2AA
:1067E00003FB161107FB06F54FEA104C4CEA01417A
:1067F0008D4209D9891806F1FF3C80F014818D4241
:1068000040F21181023E8918491BB1FBF3F503FBED
:10681000151307FB05F780B240EA03439F4207D9EF
:10682000691E9B1880F005819F4240F20281023D63
:1068300045EA0642002303E08B420AD900231A46A8
:106840001046194614B1404261EB4101BDE8F00F1A
:106850007047B3FA83F3002B40F087808C4501D357
:106860008242ECD80122EBE712B90127B7FBF2F222
:10687000B2FA82F6002E3AD1891A150C1FFA82FC60
:106880000123B1FBF5F705FB17110CFB07F64FEAE7
:10689000104848EA01418E4207D9891807F1FF38AC
:1068A00002D28E4200F2DA804746891BB1FBF5F630
:1068B00005FB16110CFB06FC80B240EA0140844542
:1068C00007D9711E821880F0B080944540F2AD80E7
:1068D000023E46EA0742B3E7E443524263EB430316
:1068E00066E7404261EB41014FF0FF345DE7B240A3
:1068F000C6F1200521FA05F320FA05F901FA06F19F
:10690000150CB3FBF5F805FB18371FFA82FC0CFBDE
:1069100008F349EA01094FEA194141EA0747B04043
:10692000BB420AD9BF1808F1FF3180F09580BB4205
:1069300040F29280A8F10208BF18FE1AB6FBF5F3E8
:1069400005FB13670CFB03F61FFA89F949EA0741B7
:106950008E4206D95F1E891878D28E4276D9023BC4
:106960008918891B43EA08438BE7C3F1200122FA07
:1069700001F80CFA03F725FA01FB20FA01F205FAF7
:1069800003F548EA070C4FEA1C48BBFBF8F908FB83
:1069900019B71FFA8CFA0AFB09FB15432A0C42EAC5
:1069A0000747BB4506FA03F609D917EB0C0709F1AF
:1069B000FF324FD2BB454DD9A9F102096744CBEB59
:1069C0000701B1FBF8F208FB12170AFB02FAADB29D
:1069D00045EA07418A4507D9551E11EB0C0137D20C
:1069E0008A4535D9023A614442EA09421FFA86F8DB
:1069F0004FEA124C08FB0CF7360C95B208FB05F871
:106A000006FB057506FB0CFC05EB1845AF4288BF7D
:106A10000CF5803CCAEB01010CEB1546B14212D3D8
:106A200009D000230CE76646EEE60E4646EA07422A
:106A300006E70D46FCE600FA03F31FFA88F808EBB8
:106A40000545AB42EDD2013A0023F9E63B4688E723
:106A50002A46C9E79146B2E788466EE7023F8918A1
:106A600023E700BF2DE9F007144605460E46002B2C
:106A70003FD18A424AD9B2FA82F343B1C3F120002E
:106A800025FA00F201FA03F69C409D401643230CC0
:106A9000B6FBF3F1A0B203FB116C00FB01F22F0C6B
:106AA00047EA0C46B24208D94F1E361980F0FF80E3
:106AB000B24240F2FC8002393619B61AB6FBF3F244
:106AC00003FB126300FB02F0ADB245EA03439842B8
:106AD00007D9561E1B1980F0EC80984240F2E980DD
:106AE000023A42EA0142002310461946BDE8F00787
:106AF00070478B4243D8B3FA83F4002C42D18B42C7
:106B0000234601D382423BD80122EDE712B9012787
:106B1000B7FBF2F4B4FA84F2002A40F08A80091B31
:106B2000260CA7B20123B1FBF6F006FB101107FB00
:106B300000F24FEA154C4CEA01418A4207D9091983
:106B400000F1FF3C02D28A4200F2D4806046C2EBE0
:106B5000010CBCFBF6F206FB12C107FB02F7ADB25B
:106B600045EA0145AF4207D9511E2C1980F0A38098
:106B7000A74240F2A080023A42EA0042B4E7002372
:106B80001A46B1E7C4F1200703FA04F822FA07F322
:106B900021FA07F920FA07FA01FA04F143EA080397
:106BA0001E0CB9FBF6FC06FB1C991FFA83F808FBC8
:106BB0000CF74AEA010A4FEA1A4545EA0945AF428D
:106BC00002FA04F905D9ED180CF1FF32C0F0878004
:106BD0009446EA1BB2FBF6F706FB172608FB07F8FC
:106BE0001FFA8AFA4AEA0641884503D97A1EC9186B
:106BF00070D3174647EA0C42170C1FFA89FC0CFBAE
:106C000007F695B24FEA19430CFB05FC03FB05653B
:106C100003FB07F305EB1C45AE4288BF03F5803349
:106C2000C8EB010103EB1543994250D347D0002331
:106C30005AE79440C2F1200621FA06F520FA06F937
:106C400001FA02F1260CB5FBF6F806FB1855A7B2BF
:106C500007FB08F349EA01094FEA194141EA054CEB
:106C6000634500FA02F509D91CEB040C08F1FF3268
:106C70003ED263453CD9A8F10208A444C3EB0C0200
:106C8000B2FBF6F306FB132007FB03F21FFA89F9A8
:106C900049EA00418A4206D9581E091926D28A4279
:106CA00024D9023B0919891A43EA08433BE73946CC
:106CB00003E7324615E70A4642EA004214E700FAC3
:106CC00004F01FFA8CF101EB0545A842AFD2013A5E
:106CD000002309E788458CD9023FC9188AE7AF42EB
:106CE0007FF676AFACF1020CED1872E70346DAE7F7
:106CF0009046C3E70238091929E700BF002103E0E5
:106D00000A4B5B584350043109480A4B42189A42D7
:106D1000F6D3094A02E0002342F8043B074B9A42AB
:106D2000F9D3F9F7FDFA00F00DF87047007B010880
:106D300000000020BC050020C0050020A06200204B
:106D4000FEE7000010B562B6F1F796FAF2F792FD91
:106D5000F1F778FAF2F76CFFF3F702FAF1F7FEFFBA
:106D6000194C28B1F1F7FAFF6070F1F7F7FFA06056
:106D70002078F2F723F922696079A168F2F7B4FB71
:106D8000F4F752FDF3F73EFEF4F7BEF8F1F782FD9B
:106D9000F7F78CFCF8F7E6F9F8F71AFD0B4B1C2215
:106DA0005A83F7F7A1FDF8F7DEF9F8F725FDF1F7BB
:106DB00041FCF1F763FC0028F3D0F4F7A5F8F7F7EE
:106DC00075FCF8F705FDECE7040000200010024018
:106DD000014600200246034600F0DAB800210A22EC
:106DE00000F0C8B838B5084D084C641BA41006D094
:106DF00005EB840555F8043D9847013CFAD1BDE800
:106E0000384000F0E5BD00BFFC7A0108007B0108B6
:106E10000F4B70B41E68054615F8013B11F8014B85
:106E2000F21850781A4600F00300012808BF03F159
:106E3000200233195878234600F00300012808BFC8
:106E400004F12003D01A01D1002BE5D170BC7047AA
:106E5000B40500202DE9F00F454C82B02468019064
:106E6000084605780646671997F801A001301AF020
:106E7000080A0746F5D12D2D5BD02B2D04BF757860
:106E8000B71C002B42D0102B40D099466619BAF19E
:106E9000000F76780CBF6FF0004B4FF0004BBBFB40
:106EA000F9F84FF0000C16F0040F09FB18BB604610
:106EB00013D0303DAB421ADDBCF1FF3F06D0404558
:106EC0002ED82BD009FB00504FF0010C17F8015BB6
:106ED0006619767816F0040FEBD116F0030606D08B
:106EE000012E14BF57263726AD1BAB42E4DCBCF1A4
:106EF000FF3F23D0BAF1000F19D11AB1BCF1000F36
:106F000013D1116002B0BDE8F00F7047302D20D0D2
:106F1000002BBAD1302D27D00A23B6E75D45D1DD4D
:106F20004FF0FF3C17F8015BD2E7791EE9E74042DA
:106F3000E3E77578B71C4FF0010AA2E7BAF1000F3A
:106F4000019C0CBF6FF000404FF0004022232360F3
:106F5000D3E73878782801D05828D9D14FF01009D4
:106F60007D784B46023791E7082399468EE700BFAC
:106F7000B405002030B440F2B053C2F200031D68E3
:106F80000C46134601462246284630BCFFF762BF36
:106F90002DE9F0410546274884B00468D4F848013B
:106FA000002841D046681F2E1CDD234810B94FF041
:106FB000FF301EE04FF4C870039102920193AFF3CB
:106FC00000800399029A019B0028F0D0D4F8486110
:106FD000002780E8C000C4F848013E46C0F8887128
:106FE000C0F88C7145B9B31C013640F823104660D7
:106FF000002004B0BDE8F081012404FA06F4D0F8C2
:10700000887100EB860847EA040C022D4746C8F851
:107010008820C0F888C1C8F80831E4D1D0F88C3194
:107020001C43C0F88C41DEE704F5A670C4F84801A3
:10703000B8E700BFB478010800000000024B13B1AC
:107040000248FFF7C5BE704700000000E56D01086B
:107050002DE9D0438AB006460F4600F079F8384C47
:10706000804694F900308946013336D0304639469F
:1070700000F06EFA002830D0304639460022002356
:10708000FDF792FF002828D12E4B2478019300238E
:107090000893CDE90267CDE90467002C22D04FF0B8
:1070A00000094FF00008CFF6F0793046394600224B
:1070B0000023CDE90689FDF74FFF002822D00223E7
:1070C0009C42009331D0684600F076FA00282CD01C
:1070D000089B002B24D1DDE90689404649460AB0C9
:1070E000BDE8D0834FF6FF794FF06048CCF2EF79DE
:1070F0003046394600220023CDE90689FDF72CFFF2
:107100000028DCD10123022C009313D0684600F044
:1071100053FA78B10C4800F051FACDE90601D7E7EF
:1071200000F052FA089B0360D5E700F04DFA2223E5
:107130000360CDE700F048FA21230360EAE700BFCF
:10714000B8050020BC790108C079010800000000E2
:107150002DE9F04FB1F5801F87B00B460C465FDA82
:1071600021F00043034300F0FD800029C0F2AC8110
:1071700000230022C4F25033FDF786FC4FF6FF7265
:107180000B46C7F6EF7293426FF035074FDC23F0E2
:107190007F4545F6647425F47005C0F209042C1986
:1071A00004F4801484F07E521E1582F4E002002361
:1071B00042EA0501C3F6F0730022FDF7B1FAA6F525
:1071C0007E76AB1C073E23F47003F6190022022BD7
:1071D00006EB145482468B4630DC0023FDF7BCFEE0
:1071E000002800F0C880002C00F077812046FDF7D1
:1071F000E5FBA1A3D3E9002304460D46FDF744FCBB
:107200009FA3D3E9002306460F4620462946FDF7F3
:107210003BFC02460B4630463946FDF783FA0AE04E
:107220004FF6FF72C7F6EF7200279342AFDD0246BA
:107230000B46FDF777FA07B0BDE8F08F4FF08043BB
:10724000FDF770FA02460B4650465946FDF746FDDB
:10725000CDE900012046FDF7B1FBCDE90201DDE9F2
:10726000000102460B46FDF70FFC02460B46804626
:107270008946FDF709FC84A3D3E9002306460F469F
:10728000FDF702FC82A3D3E90023FDF74BFA324657
:107290003B46FDF7F9FB80A3D3E90023FDF742FA53
:1072A00032463B46FDF7F0FB7DA3D3E90023FDF713
:1072B00039FA42464B46FDF7E7FB7BA3D3E90023AF
:1072C0008046894630463946FDF7DEFB78A3D3E990
:1072D0000023FDF727FA32463B46FDF7D5FB76A3A0
:1072E000D3E90023FDF71EFA32463B46FDF7CCFBFF
:1072F00002460B4640464946FDF714FA4EF68633E1
:107300004BF65102CFF6F973C0F20602EB18521B8E
:107310001343002B06460F4656DD00230022C3F61A
:10732000E07350465946FDF7AFFB52465B46FDF70A
:10733000ABFB80468946002C6AD132463B46FDF7BE
:10734000F1F9DDE90023FDF79FFB02460B464046BD
:107350004946FDF7E5F902460B4650465946FDF70A
:10736000DFF968E70021002000220023CCF2503131
:10737000FDF7B4FC5FE752465B4650465946FDF7C1
:1073800083FB4FA3D3E9002306460F4650465946D8
:10739000FDF77AFB0B4600210246C3F6E0710020A0
:1073A000FDF7BEF902460B4630463946FDF76CFB49
:1073B00006460F46002C40F0938050465946324610
:1073C0003B46FDF7ADF936E7002C00F0AD802AA36F
:1073D000D3E90023DDE90201FDF756FB32463B46C7
:1073E0008046894650465946FDF79AF9DDE9002363
:1073F000FDF74AFB22A3D3E9002304460D46DDE94D
:107400000201FDF741FB02460B46204629467EE07D
:1074100019A3D3E90023DDE90201FDF735FB32466C
:10742000CDE904013B4640464946FDF77BF9DDE9DD
:107430000023FDF729FB12A3D3E9002304460D46E0
:10744000DDE90201FDF720FB02460B4620462946F6
:10745000FDF768F902460B4640464946FDF760F9DC
:1074600052465B46FDF75CF902460B46DDE9040136
:10747000FDF756F9DFE600BF0000E0FE422EE63FD2
:10748000763C7935EF39EA3D44523EDF12F1C23F96
:10749000DE03CB966446C73F599322942449D23FDA
:1074A000935555555555E53F9FC678D0099AC33F2A
:1074B000AF788E1DC571CC3F04FA97999999D93F41
:1074C000555555555555D53F02460B46FDF728F9FC
:1074D00000220023FDF702FCADE600200021AAE611
:1074E0002046FDF76BFA16A3D3E9002304460D46A8
:1074F000FDF7CAFA14A3D3E9002380468946204643
:107500002946FDF7C1FA02460B4630463946FDF7DB
:1075100007F952465B46FDF703F902460B46404623
:107520004946FDF7FDF886E632463B465046594649
:10753000FDF7F6F8DDE90023FDF7A6FA0BE700BF3B
:107540000000E0FE422EE63F763C7935EF39EA3D19
:107550000B4661B1B1F1004F09D04FF6FF72A3F5B0
:107560008011C7F6DF72914205D8042070470028C9
:10757000F3D10220704703F1FE4101F57001914201
:10758000F3D94FF6FF72C0F20F02934201D80320E5
:10759000704703F100419142F9D90022C7F6F07219
:1075A000934204D013F5801F01D000207047D0F122
:1075B000010038BF002070470020704700210020E4
:1075C000C7F6F871704700BF40F2B053C2F2000333
:1075D0001868704708B5062000F072F80120F1F72E
:1075E000E9FC00BF0F2AF0B43AD941EA00039B0737
:1075F00038D10C46034615462668103D1E60666865
:107600005E60A6689E60E6681034DE6010330F2D61
:10761000F2D8A2F1100424F00F0402F00F0210348B
:10762000032A00EB0403214411D90E461D461446DB
:1076300056F8047B043C032C45F8047BF8D8141F4F
:1076400024F00304043402F0030209191B192AB1BF
:1076500011F8014B013A03F8014BF9D1F0BC704726
:107660000346F4E70346F3E71F2938B50C46054601
:1076700020D8D0F8DC229AB152F8213083B1012B06
:107680000CD0591C06D00025204642F824509847BB
:10769000284638BD16230360012038BD002038BDC0
:1076A000284600F02BF8224601462846BDE838401F
:1076B00000F010B8162303604FF0FF3038BD00BF54
:1076C00040F2B053C2F200031B6801461846FFF7B0
:1076D000CBBF00BF38B5084C00230546084611460D
:1076E0002360F1F768FC431C00D038BD2368002BF1
:1076F000FBD02B6038BD00BF9C620020F1F75CBC62
:10770000F40100006400000001800808000000008F
:10771000000001000000000000000000C8000000A0
:107720000000000000000000010003E8000000006D
:1077300000000003E800000000000200FA06000359
:1077400000000000003706000000000000000000FC
:10775000010203524F5200000106524F4C0000023A
:10776000064D5354000003024D56500000040753C9
:1077700041500000050747415000000603535441A3
:107780005000070352534150000803534750000074
:10779000090747475000000A0353544750000B03A2
:1077A00052534750000C0352465300000D035349F7
:1077B0004F00000E0747494F00000F03534143009D
:1077C000001D0753434F00001E0747434F00001F93
:1077D0000343434F0000200341434F00002703555C
:1077E00046300000400755463100004107554632FB
:1077F0000000420755463300004307554634000059
:1078000044075546350000450755463600004607F3
:107810005546370000470752554E00008105535426
:107820004F5000800042494E00008B0000000000D5
:10783000000000020102333131305631303700563A
:10784000435020496E74657266616365005643500B
:1078500020436F6E66696700544D43333131300009
:107860005472696E616D6963204D6F74696F6E202B
:10787000436F6E74726F6C00544D434D2D33313134
:107880003020287669727475616C20434F4D290051
:107890004142530052454C00434F4F524400535411
:1078A0004152540053544F500053544154555300C7
:1078B00043000000880100200020202020202020FC
:1078C0002020282828282820202020202020202090
:1078D00020202020202020202088101010101010A0
:1078E00010101010101010101004040404040404EC
:1078F0000404041010101010101041414141414186
:107900000101010101010101010101010101010167
:107910000101010110101010101042424242424277
:107920000202020202020202020202020202020237
:1079300002020202101010102000000000000000DF
:107940000000000000000000000000000000000037
:107950000000000000000000000000000000000027
:107960000000000000000000000000000000000017
:107970000000000000000000000000000000000007
:1079800000000000000000000000000000000000F7
:1079900000000000000000000000000000000000E7
:1079A00000000000000000000000000000000000D7
:1079B0000000000000000000000000006C6F670085
:1079C00000000000F8B500BFF8BC08BC9E46704738
:0C79D000F8B500BFF8BC08BC9E4670472C
:1079DC00A1B20181B0B0AE010000000008B101817C
:1079EC00B0B000840000000008B10181B0B0008488
:1079FC000000000008B10181B0B00084000000005C
:107A0C00C0DCFF7FB0378480E8DCFF7FAB08B1803F
:107A1C000CDDFF7F0100000088DDFF7FB0A9028034
:107A2C0048DEFF7FB0B0A88098DEFF7FA4FFFF7F09
:107A3C0064DFFF7FA908B1808CDFFF7F01000000AD
:107A4C0008E0FF7FB0AF0A8014E3FF7F0100000065
:107A5C0018E3FF7FAE3F2780C4E6FF7F01000000E4
:107A6C00C0E6FF7FAB10B28018E7FF7F010000007B
:107A7C0024E7FF7FA908B18058E7FF7F01000000D1
:107A8C0064E7FF7F58FFFF7F6CE7FF7FAB26B28078
:107A9C00D8E7FF7F01000000B0E9FF7FB0A80380AA
:107AAC00C4E9FF7F01000000C0E9FF7FB0AD048096
:107ABC0084ECFF7FB0A80380A4ECFF7F2CFFFF7F3A
:107ACC00A8ECFF7F30FFFF7FB4ECFF7F01000000CC
:107ADC00C0ECFF7FB0B0A78080EFFF7FB0B0A68076
:087AEC0010F2FF7F0100000011
:087AF4003D700108AD8100089E
:047AFC008981000874
:107B000036780108000102000008000001000000B2
:107B10000200000000000000000000000000000063
:107B20000000000000000000000000000000000055
:107B30000000000000000000000000000000000045
:107B4000000000001201100202000040D016CC0616
:107B500000020102030104030904000000C2010045
:107B60000000080073B5000881B5000815B60008CC
:107B700031B60008F9B50008DDB50008C1B5000848
:107B800065B5000867B5000869B500086BB5000861
:107B90006DB500086FB5000871B500080A0600024F
:107BA00000000040010000008DB5000891B50008FC
:107BB0004DB6000895B5000899B50008000E2707D6
:107BC000000000000000000001020304060708098D
:107BD0000000000001020304010203040607080973
:107BE000E40000209D2E0108E92D01089F2D0108C9
:107BF0000F2D0108712D0108F32C0108DD2C01085F
:107C00001F2D01082D2D01083B2D0108512D0108C4
:107C100009024300020100C032090400000102020F
:107C200001000524001001052401000104240202C2
:107C30000524060001070582030800FF090401006E
:107C4000020A00000007050102400000070581024A
:107C500040000000FF0000001D310108F530010860
:107C6000313001080000000071310108A131010824
:107C700001300108812F0108000000000000000011
:107C8000752F0108000000000000000074040020AF
:107C9000DC0400204405002000000000000000007B
:107CA00000000000000000000000000000000000D4
:107CB000000000000000000000000000B078010893
:107CC00000000000000000000000000000000000B4
:107CD00000000000000000000000000000000000A4
:107CE0000000000000000000000000000000000094
:107CF0000000000000000000000000000000000084
:107D00000000000000000000000000000000000073
:107D10000000000000000000000000000000000063
:107D20000000000000000000000000000000000053
:107D300001000000000000000E33CDAB34126DE6F0
:107D4000ECDE05000B000000000000000000000059
:107D50000000000000000000000000000000000023
:107D60000000000000000000000000000000000013
:107D70000000000000000000000000000000000003
:107D800000000000000000000000000000000000F3
:0C80B00088010020B878010801000000E1
:0400000508016CFD85
:00000001FF
